:020000024000BC
:100000006FD0A23400000000001801180028012859
:100010000228032800290129022903290429052986
:10002000062907290829002A012A022A032A042A64
:10003000052AA62A78DF06008C3F0400B4040020BD
:100040003605002034040020F40300208C03002037
:100050002440040066400400884104001E4404005B
:1000600038450400EA3E0400983E0400EC020020FB
:100070008C020020144A04006C080020FA3F04009F
:1000800010470400967906007C7B0600E27B0600A0
:10009000AE530600E8530600A483050082780500ED
:1000A000B47306003E470400625B0600DAF8040001
:1000B00068F90400C6F9040008520400465204001E
:1000C000BC500400F4BA0400DAB504005A29002038
:1000D00018C704006ACA04007CA804001EA8040013
:1000E000EAAB0400C8A80400FCA7040074A804003C
:1000F000B2A704004AA90400A2A9040052A904005E
:1001000056A90400E4A90400AAA90400DAA904007D
:10011000BCAE0400C0AE040046A904004EA9040011
:10012000E2A90400BEAE040090AA04001CB00400C2
:1001300018D804008AD80400C4D804003ABD0400CA
:1001400050BD04008ABD0400949D04009A9F0400E1
:1001500062A00400A46F0400EE690400A8930400E8
:100160006A6A04005E8F0400C4B80600FAB0060094
:1001700000B6060024CD0600EECB060042D00600F5
:10018000FECF06003AD006008ED10600B69F0600CC
:100190001ED106008CC30600B2C30600D2C30600FF
:1001A000FED10600E2C906007AC906006ED206003A
:1001B0003AA20600D2A20600F2A20600A4A20600FD
:1001C000E05B050082460500FE490500BE470500CC
:1001D00008520500587406004C730600EA9F06009A
:1001E000964B0400FE540600425B06003A5C060093
:1001F000486A0600CA6A06002C6C0600F4C00400B7
:10020000E25A0500B052050052440500565505005B
:10021000324605002C0A0020D655060068D006009C
:1002200002D0060036D0060032D006009E430400FD
:1002300072BE040070D00600BE5E0600845F060039
:10024000EC5F060068B606006CD00600B6D006006B
:1002500004780500BAD00600B62000207C200020DB
:1002600048B60600DEB70600BED0060012D1060072
:1002700016D1060074D00600AED00600B2D006003B
:100280001AD10600985B0500000000000000000085
:10029000000000000000000000000000000000005E
:1002A000000000000000000000000000000000004E
:1002B000000000000000000000000000000000003E
:1002C00017470000130757BB974700009387973ED7
:1002D000014663ECE70097470000938727BA17466B
:1002E00000001306663D1D8E719A8145174500007A
:1002F0001305C5B8174304E0670023D7174700006C
:10030000130717AA97470000938757B7014663EC76
:10031000E700974700009387E7A8174600001306F9
:1003200026B61D8E719A97E506E09385252D174513
:0E0330000000130525A7174304E06700A3D1C2
:100340004111B7E700E022C480433707200006C60A
:10035000798C23A0E7180F10000011C199E5B7E7C9
:1003600000E023A08710014579A80D053345050855
:10037000130740037199B34705086366A702174541
:100380000000032525B09746000083A626AF6391A1
:10039000A60217470000032767D171D3C207DD8D7E
:1003A000054502976DBF17450000032565ADE1BF08
:1003B0007A2131EF5A21636CF704B306F7402148E4
:1003C00017460000130606C96375D8028328050086
:1003D00003586600938687001D8FAA966117DAA2DC
:1003E00023A016012393060014C15EA1130788FF02
:1003F0007AA27A226EA12105B307F7407EA2B7E761
:1004000000E023A08710B2402244410182800841CD
:10041000BDBFB7E700E08C433707200023A0E718F3
:10042000F98D0F10000001E523A0B710828017435B
:100430000000032323A59748000083A828A49A87D7
:10044000814663FE170903A80700636DF508636B17
:10045000A808138787006364E508F223216705076E
:100460006319E60017460000130636B01822050788
:1004700018A2174500001305E5BDD2237A21239366
:1004800007003297334707087AA16385670217434D
:1004900000000323E39E630FF30003D36600631B96
:1004A0000300DE2223A0060121073E962106D2A2E8
:1004B0007AA1B6879843630417039746000083A682
:1004C000269C630ED700762399EAD623522318433D
:1004D000A106B296D6A398C37E21A1077EA1B7E755
:1004E00000E099B7BE86C287A9BFAA871747000058
:1004F000032747991746000003264698B305B540E1
:100500006314E6003E8529A8930687001843E3E9B3
:10051000D7FEE3F7E7FE2E85E3E4D5FEE3F2E5FE42
:10052000828023AC05FE1C4199E30CC182803E878A
:1005300083A787FFEDFF232CB7FE8280411126C2DF
:10054000B7E400E04AC003A90400B707200006C6CC
:1005500022C43379F90023A0F4180F10000009E534
:1005600023A0241101452DA09565938505D0C98D43
:100570002A842105B3C5050833450508D1336DD15B
:10058000FD572320050042A17CA123A024112105B1
:10059000B240224492440249410182804111B7E7AE
:1005A00000E04AC003A9070026C23707200006C69C
:1005B00022C4AA843379E90023A0E7180F100000B1
:1005C0009747000083A7478C0144014695E311C873
:1005D000A285174500001305258B974004E0E780AE
:1005E00000B5A1652685974004E0E780800E2DA028
:1005F00003C7E7FF631D970221C0A28517450000CE
:1006000013058588974004E0E78060B2A1652685E0
:10061000974004E0E78040CCB24022852244B7E70F
:1006200000E023A02711924402494101828011E099
:100630003E8683A787FF59BF3E84E5BF37E700E0CA
:100640001C43B70620002320D718F58F0F10000099
:1006500019C191C111E637E700E02320F71082802D
:100660002E960F70B650D5BF37E700E01C43B70693
:1006700020002320D718F58F0F10000019C1014763
:1006800085E137E700E02320F7108280B386E5009C
:1006900003A80600B306E5007D1623A00601110796
:1006A00075F6C5B7411126C2B7E400E022C4804008
:1006B000B706200006C6758C23A0D4180F100000C2
:1006C00011C111EAB7E700E023A08710B24022442D
:1006D000924441018280974004E0E780009923A082
:1006E0008410EDB7411122C437E400E026C2044073
:1006F00006C6B7072000FD8C2320F4180F10000059
:1007000097D006E0E780C031B24023209410224405
:100710009244410182800111B7E700E026CA844378
:100720004AC83707200006CE22CC2A892E86F98CAB
:1007300023A0E7180F1000009305F00432C63345DC
:100740000608FD3E2A8401C53246CA85C53DF240F1
:1007500022856244B7E700E023A097104249D244C3
:100760000561828037E700E01C43B70620002320A4
:10077000D718F58F0F10000001C599C1014711EA84
:1007800037E700E02320F710054582800507E309DD
:10079000E6FE3308E500B386E5000348080094222E
:1007A000E306D8FE37E700E02320F71001458280FA
:1007B00037E700E01C43B70620002320D718F58F49
:1007C0000F1000001307F6FFBA952A966317C500AD
:1007D00037E700E02320F71082809821FD150505FA
:1007E000A30FE5FEE5B737E700E01C43B70620009E
:1007F0002320D718F58F0F10000001C53307C5005F
:1008000019E637E700E02320F71001458280142124
:100810000505E398B6FEE31CE5FE37E700E023207C
:10082000F71005458280797126D2973400009384B1
:10083000246722D4804006D64AD04ECE52CC56CA27
:100840005AC85EC662C45DC837C9C901814B973AB0
:100850000000938A6A641309F937174B0000130BE1
:10086000EB81973900009389E97E174A0000130A4B
:10087000EA853E2091EF5C4463990B009CC0032CF9
:10088000C400228579366284B9A823A6FB00C5BFBF
:1008900083A70A0082971C443307F5406376F5006E
:1008A00003278A001D8F2A97636DE906973700009A
:1008B00023AA077A2E200820974004E0E780C0A1F1
:1008C0005C405844A1CB0C441746000003268680A8
:1008D000AE97BE8663E4B70063E4C700B386C74043
:1008E00014C4A28B3A8451F417370000130787769B
:1008F0001C4B854663FBF604FD171CCBB2502254FB
:1009000092540259F249624AD24A424BB24B224CAB
:100910004561828063940B0098C095B723A6EB00D5
:10092000B9BF03274B0219CB63EDA7003385A7405E
:1009300083A709016374F50023A8A900A28B404492
:100940005DB703278A00BA97D5B79737000023AB66
:1009500007706DB70111B7E700E04AC803A90700A7
:100960003707200006CE22CC26CA4EC652C43379A1
:10097000E90023A0E7180F100000973400009384CB
:10098000E4749C288844B9CF97470000938787A5D3
:1009900003D7C70A21CB03A4870A6305A4049739A8
:1009A00000009389296B83A709016380A710173A78
:1009B0000000130A6A4E83270A0082976364A40E1C
:1009C00083270A00098C829783A70901984433542E
:1009D000F40AB307A4003E8563E4870063E4E700FC
:1009E0003385E740B7E700E023A027119C44639DCF
:1009F000A702173400001304E46518489737000075
:100A000083A787496315A70A82979444374736FE20
:100A1000130707C83697B307A7003E8563E4E700CE
:100A200063E4D7003385D74017440000130484BE25
:100A30005C5C99CB9736000083A6C6589C46370766
:100A4000CDFF7D17F98F9CC611E1884485475CD0A6
:100A50009737000083A7C764829715E15C5C99CF44
:100A60005C5089CF975006E0E7808062975006E09F
:100A7000E78040D59747000023A007BC6D335C5C3E
:100A800091CB173700000327E7531C47B706330005
:100A9000D58F1CC7F2406244D2444249B249224A2F
:100AA000056182809C443E9421BF228525BF8297A8
:100AB00014489844B387A6003E8563E4D700E3E575
:100AC000E7F63385E7408DB79737000023A0A73CB2
:100AD00011C5854717370000230CF73A82809737F6
:100AE000000083A7A73A85C3411106C682979737AE
:100AF000000083C7E73989E79737000023A8073844
:100B0000B240410182809737000083C7673891E780
:100B10009737000023AC073682808280411122C4BF
:100B200026C206C64AC0974400009384A4AE83C779
:100B300034021734000013042458B9C717340000D6
:100B400013044451173900001309C935032709005C
:100B50001C2014300146B3A5E7208E21A5CD11C27B
:100B60001CA00820636FD506973700002384074E2A
:100B70009737000083A74732C5EFB2402244924422
:100B800002494101828082971C40F5FF973700009F
:100B900083C7C75485E3DC48858B89CFD84C9947F8
:100BA000631EF7009747000023A007A8EF10701DF1
:100BB0005C4482971C44D9D3829749B7D84C9D474F
:100BC000E31AF7FE9747000023A007A6EF10701B5B
:100BD0001C48C5B7850793F7F70F0546E3EDD7F631
:100BE00041B73327E5200E23231007009737000075
:100BF0002391072A9737000083A7472AB347F52098
:100C00009C4382971C208326090017370000035756
:100C100047283377E540B3A6D7209222518F9AA276
:100C200099C385071CA018201C30E368F7F42DBF7A
:100C30009737000083A7074A1CC8F53683C73402DC
:100C40008DFF83C7140299CBDC4C89EB97470000DA
:100C5000A382079E975006E0E780A0E39737000045
:100C600083A7074499DBD84C9147E3E8E7F097372F
:100C7000000083C7A775918BE39107F097370000B9
:100C800083C70721E39B07EE18308326090063C85A
:100C9000E7002244B24092440249410165B933A6BB
:100CA000D7201222E31B06EC8507D5B7B7C7004053
:100CB0001387C72014431396264910C3010001006F
:100CC00093878726173500000325853A9C436A05DC
:100CD00014C393C7F7FF99835D8D82809737000017
:100CE00083A7C71C91C382871305F00F8280173634
:100CF00000001306E66A973600009386666CDC36C1
:100D0000383E4C4ABA97FD8B33D7F5001CB2DCB69F
:100D1000058B0DE7943A13050002B3F7D70281461D
:100D200033D8E548630908006394D70018B282807D
:100D3000850693F6F60F0507E314A7FE8280974712
:100D4000000083A7678EC1E741114AC097370000B2
:100D500083A7871406C622C426C2829717390000CB
:100D60001309096683278900638DA7046363F5046B
:100D70001D8D973400009384A462BC2C135455003D
:100D80006361F404AD37BC2C0327890093965700A8
:100D900036971D8C2324E900E376F4FE2244883044
:100DA000B2409244024981454101173305E0670092
:100DB000232C173700000327E731B307F7403E9590
:100DC0004DBFB24022449244024941018280828058
:100DD000011126CA9737000083A7070C06CE22CC44
:100DE0004AC84EC652C48297973400009384445D2B
:100DF0009844AA870145630DF70463E3E706998FDA
:100E0000173900001309C95993F9F70113D4570092
:100E10008347A901636AF402173A0000130A0A2BF8
:100E2000F9350347A9018C4403268A00931757001C
:100E3000AE97198CBE8663E4B70063E4C700B3863F
:100E4000C74094C4E37EE4FC1315540033653501B8
:100E5000F2406244D2444249B249224A056182804A
:100E60009736000083A606273387E640BA9749BF26
:100E7000411126C2973400009384C4799C4422C453
:100E800006C6858B173400000324045CA1C718280C
:100E90009737000023A407788947630DF7020146BE
:100EA000930550020145EF10501A01468145054552
:100EB000EF101002DC44858B91CF2244B240924463
:100EC0008145177505E01305E5A34101174304E0CB
:100ED0006700C39BEF20D05622852244B240924443
:100EE00041016F10D05E9737000083A7A759639F19
:100EF000071C011122CC2A84094506CE26CA4AC8FD
:100F00004EC6973400009384E40AEF20905B904033
:100F10009307800717390000130909097CD283273A
:100F20000900973900009389E909B7053300D857BC
:100F30002285719B13671700D8D798431377F7CF93
:100F400098C398431377F7CF1367072098C303A775
:100F500009001447CD8E14C7B70603009386862573
:100F600034CA5457F59A54D798433424137707F862
:100F700093F6F607558F98C3EF10706A94403705C3
:100F800000827D15DC4293E71700DCC203260900CE
:100F9000030784065C569375F703E605E98FCD8F4A
:100FA0005CD69305A00383A7090063D9E50AF84F2F
:100FB000B70500074D8FF8CFB7C7898E938767EDC8
:100FC0001CC6B7575500938757555CC28347A40684
:100FD00083494406B3E9F9008947173700002329FC
:100FE000F7649737000023AD07627C44BCDE973777
:100FF000000083C7A70ED9CFFC52FDFF0C384E85E9
:101000009737000023AC0760EF10E06318289D4776
:10101000172500001305E5206306F70017050000FB
:10102000130545E55534832709009843131777299D
:1010300098C3D857719BD8D79737000023A6075E6F
:101040009737000023AA075C9C40F240624409479E
:1010500098C3D2444249B249056182809305200277
:1010600063DAE500F84FB70500F9FD156D8FB70598
:10107000000589B7B70500F96945FD156357E50017
:10108000F84F6D8FB705000335B7F84F6D8F131705
:10109000872915B718289D47814517250000130596
:1010A00045186306F700170500001305A5DC973007
:1010B00004E0E780A07D10386244F240D244424907
:1010C000CE85B249014505616F10806082809737F7
:1010D000000093872731E853054754256390E602C3
:1010E00003C747079147631AF700011106CE2AC6C6
:1010F000EF1070393245F2400561F5B382808327E5
:101100008511E5CB411122C406C658258345E50467
:101110009437D2272A841377C70F1395466063F755
:10112000C50663510506882793F6F60794B705466A
:10113000936627006314C5009366170054A4D84330
:101140000907D8C3032504114CB82E86CC430905E2
:10115000EFF0CFCE832784115438D8433697D8C3C5
:10116000DA27158FDAA789473CBC03476403973712
:10117000000083C7C7F16369F706B2402244014506
:10118000410182801367170058A46DBF9376F60F54
:101190006355050288278545136627006314B5004B
:1011A0001366170050A454B8A384070085473CBCBD
:1011B000832784119C43D5FBC9B71367170058A434
:1011C00054B8A384070003250411CC430905EFF0AC
:1011D000EFC6832784115438D8433697D8C3DA270B
:1011E000158FDAA78D47E1B75C2493E707015CA46C
:1011F00069B70545828041119737000083A707D959
:1012000022C406C6858B2A84C5E74165130525F5EA
:10121000978005E0E780C03B41CD3C253EA5832774
:101220000412ADE32320A4122322A4128547231124
:10123000F404232005007C2854415EA5583418A5E9
:10124000054718B5138517021737000003274740D5
:1012500015811C437D151375F50F9CC25C43DCC2E0
:101260001C479CC65C47DCC61C4B9CCA5C4BDCCA5A
:101270001C4F9CCE5C4FDCCE0DC19386060213073B
:101280000702C1BF8327441288C383572404232243
:10129000A4128507B3C7070859BF17370000130703
:1012A00067141E2785071EA7B24022444101828091
:1012B0005C2423090400054593C747005CA4EDB7EF
:1012C000142D854763EED70A1C3D2A870145DDEBC7
:1012D0005C2713F507013C2B99CB834667039737AF
:1012E000000083C7D7DA63ECF60001E5828059E598
:1012F00082808357271E0357671EBA9721A0835702
:10130000271E75F90145BDCF9387C7121735000019
:10131000035585DCB3B5A70237460F00411113060C
:101320000624814622C426C206C67D543385A70200
:1013300097C006E0E78020359734000083C494D539
:10134000AA949737000083A7271303A707099C4394
:101350003354E40AFDFB9737000083A7E7B3829775
:1013600081476364A400B307A440B240224433B56C
:101370009700134515009244410182808147A5BF23
:10138000014582808280173700000327A7C23C5B9B
:10139000FDFF01000100828035C901116C0022CCE3
:1013A00006CE2A84EF20406429C9FD57630CF5045A
:1013B00017370000130787CC5453B2479DC2254707
:1013C000637BF700938567FF034594026244F24014
:1013D00005616F100076173700000327A7CFBA9773
:1013E000D5B70C3F63E5B700B385B740F1BF1737FA
:1013F0000000032727CEBA97C5BF6244F2400561BB
:101400006F200022F24062440561828082807971FF
:1014100052CC173A0000130AEAFC26D283244A0968
:1014200006D622D44AD04ECED5C89737000093872F
:10143000671ED44F15476386E604DC532A8989CF9B
:10144000975006E0E780C0C4974006E0E780803709
:101450009737000023A2071EFD596C002685EF2058
:10146000A0580DE9172500001305C51BEFF0CFE5C7
:101470009737000083A707B43707100098C70547C0
:10148000B8DB0D45B250225492540259F249624AD7
:1014900045618280637435013244AA898440D5FC59
:1014A000FD571305F00FE38FF9FC914763F18702B5
:1014B0009307B4FF2320F9002324FA0A99E797370A
:1014C000000083A727C12320F900014565BF973796
:1014D000000083A727C0ED17A297E9BF09455DB7B4
:1014E000797126D206D622D44AD04ECE52CC56CAD4
:1014F0005AC85EC68347550303447513AA843E94B5
:101500001374F40F9307400263F687001304B4FDCD
:101510001374F40F03A9841383A9C413A38B841237
:1015200022864A85CE8597C006E0E78000110589AE
:1015300015E503CBD412014A814A337B6403930B34
:10154000500252864A85CE8597C006E0E780E00EBD
:1015500005890DC563916A031374FA0F238B8412F6
:10156000B250225492540259F249624AD24A424B32
:10157000B24B45618280850A939A4A60050AE3125C
:101580007AFDE9BF8327850903560504797193D64F
:101590000701BD8EB3C60608358E93575640898B1A
:1015A000135776485D8F93573640918B5D8F9357D5
:1015B0001640A18B5D8F93171600C18B5D8F93171B
:1015C000360093F707025D8F9317560093F70704D1
:1015D0005D8F9317760093F7F70F22D45D8F2A84DF
:1015E0009357D6001355B6001189898B9355860001
:1015F000C98F1355F6002582C98F218AD18F139682
:101600001500418AD18F1396350013760602D18FCB
:101610001396550013760604D18F13967500137632
:10162000F60FD18FA207C5455D8F3307B70226D2CB
:101630004AD04ECE032984138329C4135AC806D630
:1016400052CC56CA36973347070813565740098A73
:1016500093577748D18F13563740118AD18F13563D
:101660001740218AD18F13161700418AD18F131684
:10167000370013760602D18F13165700137606042F
:10168000D18F131677001376F60FD18F1358B7004A
:101690001356D70013784800098A1355870033661C
:1016A00006011358F700258333660601218B518FFD
:1016B00013161500418A518F131635001376060252
:1016C000518F1316550013760604518F13167500AB
:1016D0001376F60F518F2207D98FB387B7025EC6F4
:1016E000B697B3C7070813D55740098913D777486A
:1016F000498F13D537401189498F13D51740218958
:10170000498F139517004189498F13953700137539
:101710000502498F1395570013750504498F1395DA
:1017200077001375F50F598D13D8B70013D7D7006D
:1017300013784800098B13D687003367070113D845
:10174000F700A58333670701A18BD98F1317160004
:10175000418BD98F1317360013770702D98F1317D0
:101760005600137707041E06D98F1376F60FD18F14
:10177000A2073367F5003307B702130650024A8504
:10178000CE853697B98EB3C4060833F6C402137BF0
:10179000F60F97C006E0E78040EA058905E9834A2D
:1017A000D412014A930B5002B38A9A02814493DA0D
:1017B0000A0126864A85CE8597C006E0E780E0E7E5
:1017C00005890DC563914A0313FBF40F230B6413C2
:1017D000B250225492540259F249624AD24A424BC0
:1017E000B24B45618280050A137AFA0F8504E392B1
:1017F00074FDE9BF8327C50803568508797193D620
:101800000701BD8EB3C60608358E93575640898BA7
:10181000135776485D8F93573640918B5D8F935762
:101820001640A18B5D8F93171600C18B5D8F9317A8
:10183000360093F707025D8F9317560093F707045E
:101840005D8F9317760093F7F70F22D45D8F2A846C
:101850009357D6001355B6001189898B935586008E
:10186000C98F1355F6002582C98F218AD18F13960F
:101870001500418AD18F1396350013760602D18F59
:101880001396550013760604D18F139675001376C0
:10189000F60FD18FA207C5455D8F3307B70226D259
:1018A0004AD04ECE0329040A8329440A5AC806D6D0
:1018B00052CC56CA36973347070813565740098A01
:1018C00093577748D18F13563740118AD18F1356CB
:1018D0001740218AD18F13161700418AD18F131612
:1018E000370013760602D18F1316570013760604BD
:1018F000D18F131677001376F60FD18F1358B700D8
:101900001356D70013784800098A135587003366A9
:1019100006011358F700258333660601218B518F8A
:1019200013161500418A518F1316350013760602DF
:10193000518F1316550013760604518F1316750038
:101940001376F60F518F2207D98FB387B7025EC681
:10195000B697B3C7070813D55740098913D77748F7
:10196000498F13D537401189498F13D517402189E5
:10197000498F139517004189498F139537001375C7
:101980000502498F1395570013750504498F139568
:1019900077001375F50F598D13D8B70013D7D700FB
:1019A00013784800098B13D687003367070113D8D3
:1019B000F700A58333670701A18BD98F1317160092
:1019C000418BD98F1317360013770702D98F13175E
:1019D0005600137707041E06D98F1376F60FD18FA2
:1019E000A2073367F5003307B702130650024A8592
:1019F000CE853697B98EB3C4060833F6C402137B7E
:101A0000F60F97C006E0E78040C3058905E9834AE1
:101A10001408014A930B5002B38A9A02814493DA64
:101A20000A0126864A85CE8597C006E0E780E0C099
:101A300005890DC563914A0313FBF40F230F640757
:101A4000B250225492540259F249624AD24A424B4D
:101A5000B24B45618280050A137AFA0F8504E3923E
:101A600074FDE9BF8327450903568508797193D62C
:101A70000701BD8EB3C60608358E93575640898B35
:101A8000135776485D8F93573640918B5D8F9357F0
:101A90001640A18B5D8F93171600C18B5D8F931736
:101AA000360093F707025D8F9317560093F70704EC
:101AB0005D8F9317760093F7F70F22D45D8F2A84FA
:101AC0009357D6001355B6001189898B935586001C
:101AD000C98F1355F6002582C98F218AD18F13969D
:101AE0001500418AD18F1396350013760602D18FE7
:101AF0001396550013760604D18F1396750013764E
:101B0000F60FD18FA207C5455D8F3307B70226D2E6
:101B10004AD04ECE0329040B8329440B5AC806D65B
:101B200052CC56CA36973347070813565740098A8E
:101B300093577748D18F13563740118AD18F135658
:101B40001740218AD18F13161700418AD18F13169F
:101B5000370013760602D18F13165700137606044A
:101B6000D18F131677001376F60FD18F1358B70065
:101B70001356D70013784800098A13558700336637
:101B800006011358F700258333660601218B518F18
:101B900013161500418A518F13163500137606026D
:101BA000518F1316550013760604518F13167500C6
:101BB0001376F60F518F2207D98FB387B7025EC60F
:101BC000B697B3C7070813D55740098913D7774885
:101BD000498F13D537401189498F13D51740218973
:101BE000498F139517004189498F13953700137555
:101BF0000502498F1395570013750504498F1395F6
:101C000077001375F50F598D13D8B70013D7D70088
:101C100013784800098B13D687003367070113D860
:101C2000F700A58333670701A18BD98F131716001F
:101C3000418BD98F1317360013770702D98F1317EB
:101C40005600137707041E06D98F1376F60FD18F2F
:101C5000A2073367F5003307B702130650024A851F
:101C6000CE853697B98EB3C4060833F6C402137B0B
:101C7000F60F97C006E0E780409C058905E9834A96
:101C8000F408014A930B5002B38A9A02814493DA12
:101C90000A0126864A85CE8597C006E0E780E0994E
:101CA00005890DC563914A0313FBF40F230F6407E5
:101CB000B250225492540259F249624AD24A424BDB
:101CC000B24B45618280050A137AFA0F8504E392CC
:101CD00074FDE9BF411126C206C622C44AC097243A
:101CE000000083A4A4756389041003A4C40AAA860F
:101CF000054525C43C241307700A6392E708583051
:101D00001C34172900001309693C03268900B38796
:101D1000E7020357C900B387E7021307003293872E
:101D20000719B3D7E70203A744093E97BA8463644F
:101D3000F7006364C700B304C7409727000083A778
:101D4000A71584C28297B387A44063F5A400032734
:101D50008900BA9789EB1305F00FB24022449244F0
:101D600002494101828058309306204E3307D70242
:101D7000E3F3E7FE930780FA3CA40145F9BF13079C
:101D8000800AE39AE7FC9727000083A7E710829771
:101D90002A893545EF10F072AD4717370000232927
:101DA000F78858301C341726000013062632B387F4
:101DB000E7025A261046B387E702130700329387DB
:101DC0000719B3D7E70203A744093E97BA866364AD
:101DD000F7006364C700B306C740E31ED9F617D502
:101DE00005E01305E58AEFE03FCE9727000083A7C3
:101DF000671C0947F8D785B7054585B7397156D2AD
:101E0000973A0000938A0A8183A70A0337070800DC
:101E100026DA06DE22DC4AD84ED652D45AD05ECE1E
:101E200062CC66CA6AC86EC6F98F9724000083A484
:101E3000E460638A071C83A9C40A83C7990003A4CA
:101E4000C90092073E942820B14705053305F502E5
:101E50005E203E9533450508EFE04FEEAA8C630FF8
:101E6000051A130DC5002324A50134203146370B74
:101E70000300B386C602231304000149172A000099
:101E8000130A4A13972B0000938B0B12972D000017
:101E9000938D4D13130B8B15054CEA9654C483C6D2
:101EA00079009307D00783250A00B386F602C1673D
:101EB0009CC5370833008606B4D183A60B00904238
:101EC0001376F6CF90C290421376F6CF13660620B3
:101ED00090C203A50D0010453366060110C503A688
:101EE000090023A865059305500290C6722054444A
:101EF000B2962324DD0014300146CA96A301DD000A
:101F000003C504089726000023A80670EF00F0130D
:101F100083260A00CC4613961549D0C60F10000040
:101F200083260A003706020090C61306000823A87D
:101F3000CA0003A60B00104213567648631E860B98
:101F40001306E018F0D2CCC617260000232E066C2C
:101F5000172600002322066C23A086011D25EF1002
:101F6000304E83A64A00858AD9CAEA85268597D04D
:101F700005E0E780007A0DE903465D0049C276205E
:101F80004E20B29663DDB606B428AC4803258D001A
:101F9000918E8906B695EFE06FEA23020D000346A5
:101FA0005D007620B29676A003260A00310D3452E9
:101FB000FDFE342005091379F90FE362D9EE9C2464
:101FC0006685A381FC001C20A3820C002383DC0017
:101FD0002382FC006254F250D2544259B259225A20
:101FE000925A025BF24B624CD24C424DB24D21618F
:101FF000172305E06700C3931306E01AA1B7FD5647
:102000002302DD0055B79727000083A7A7FAFC57E6
:1020100091C7854717270000230CF7E6F25062545A
:10202000D2544259B259225A925A025BF24B624C34
:10203000D24C424DB24D21618280797122D426D298
:102040002E84AA84414697C506E0938565A00A853B
:1020500006D6972004E0E780E0FF414697C506E0FA
:102060009385059F0808972004E0E780A0FE3C3098
:1020700010088A85DC875C2026855C875C30DC86DE
:10208000973006E0E780202E0347F1011C20014530
:10209000631EF7000347E1011C3001456318F70098
:1020A0000345D1013C201D8D13351500B25022543B
:1020B000925445618280011122CC26CA4AC84EC67C
:1020C00006CEAA84172400000324043E1309250029
:1020D000854905C09C303830858B6304F700405C2F
:1020E000CDBF1946930544004A85EFE0AFE7E318FA
:1020F00035FFF24022856244D2444249B24905612B
:102100008280411122C426C24AC006C6172400009C
:102110000324843993042500054901E8B24022854F
:1021200022449244024941018280A6851305A402FB
:102130002937E30525FF405CCDB7411122C426C2F3
:102140004AC006C617240000032404369304250061
:10215000054901E8B24022852244924402494101E6
:102160008280A6851305A401C93DE30525FF405CD7
:10217000CDB7011126CA644122CC4AC84EC652C40A
:1021800006CE2A841D4993096505054A3C4463E44B
:10219000F4000545A1A05834DC2063192705034746
:1021A00084026304F7008440D5B7D83083475405D0
:1021B000E31BF7FE19469305640513856400EFE001
:1021C0006FDA8547E311F5FED82483479402E31CB8
:1021D000F7FCFA243E34E318F7FC0145F240624470
:1021E000D2444249B249224A05618280E31DF7FA8E
:1021F000D83083475405E318F7FA1946CE8513857E
:102200006400EFE02FD6E31045FBC1BF411122C4AB
:1022100006C626C24AC017240000032424245DC831
:102220008347840B1307700A6393E7080347140E70
:102230008347A40B17290000130949E98326890065
:10224000B387E7020357C900B387E70213070032D9
:1022500093870719B3D7E7020327440A3E97BA8446
:102260006364F7006364D700B304D7409727000086
:1022700083A787C204C18297B387A44063F5A400F3
:1022800003278900BA9785CB0347140E9306204E87
:102290003307D70263F1E702930780FA230CF40AAD
:1022A0000145B24022449244024941018280130711
:1022B000800A639EE700172506E013056526EFE018
:1022C000BF809727000083A7E7CE0947F8D71305FB
:1022D000F00FC1BF0545F1B7011122CC26CA06CEC9
:1022E0002AC42EC6172400000324841B854419E049
:1022F00001450DA09C841830858B6304F7000044D1
:10230000FDB719469305A10013052400EFE08FC522
:10231000E31795FEF2406244D244056182800000DA
:10232000EFE0EFFB730000000000000097220000C8
:10233000938202B60383020023800200630F03002E
:10234000F32510342EC0970500009385A5FD7390EA
:102350001534EF00C0577300203086DCEF002057A3
:10236000E6508280000041114AC01729000013097D
:10237000A9C30327090026C206C61C5F22C49724EE
:102380000000938424C293D76748C1C7930700060F
:102390001CDF172400001304E427184C93070008DF
:1023A0006317F7009C409C4393F707041CCC1C4028
:1023B00093F7070499CB9727000083A7E7AD82978F
:1023C00048D81C4093F7F7FB1CC01C4093F707024A
:1023D00099CF1C40172700000327C7BDB706080088
:1023E00093F7F7FD1CC05C5414C786077CD71C48C4
:1023F00093F7070499EF85475CC8370702009727D2
:10240000000083A727BB98C71307000C18C81854EF
:10241000F8D383270900985F1357474805C3985F8F
:102420001367070198DF9727000083A7A7B823A2A7
:1024300007068547172700002326F71E9C40D84330
:102440001357174819C7D843759BD8C3D843799BEE
:10245000D8C3B240224492440249410182802137CC
:1024600073002030972700009387C71A37070400AE
:1024700088DB698F11CF172700000327A7B3FD560C
:1024800034D7972600009386E6BCD84E0507D8CEF1
:102490001377850001CB98471367170098C7130778
:1024A000000898CB1377150009C7D84313671700A6
:1024B000D8C3137765000DC31377450059C79843F8
:1024C0001367170098C39726000083A6E6ADD85679
:1024D000719B13671700D8D64167698F0DC3972684
:1024E000000083C666F7C18A17270000130787EF2D
:1024F000B5C28346470793E60602230AD706370785
:102500000200698F11CF984B1377070819C305474D
:1025100098CB9727000083A7E7A93707020098C741
:10252000B70708007D8D0DC1172700000347D7F2BC
:10253000058B972700009387E7EA1DCB03C7570752
:1025400013672700A38AE7068280D847136717001E
:10255000D8C795BF834647070946BD8A6388C6002A
:10256000834647070D46BD8AE39BC6F8914671B77F
:1025700003C75707118B69DB03C75707136787002A
:10258000D1B79726000083A6E6A29727000093877D
:1025900067089843058B19E7D843058B01E7F85284
:1025A0006DFBDC4B9727000023A00708828097264D
:1025B00000009386669F2A8788421C5D93D7574800
:1025C000C9E381C51C59BD839CA115C69C42945B7F
:1025D000C60693D7660163D6060093E707C0B3C764
:1025E00007088316060093975760B1CABE968947BD
:1025F000B3C6F60216A29727000083A7A79BBC4B81
:10260000014593D757489DCF08330DCD972700003C
:1026100083A7C70193F707049306950009459DC357
:1026200036971C230547194593F6F706639CE60089
:1026300001459397476063D70700394582801EA202
:102640005DBF054582809727000083A7279699CB19
:10265000944BD04B9842518F98C294439C479842D8
:10266000D98F9CC2172600001306C694054818424D
:102670009726000083A6469397270000938787F943
:10268000631D050388421365050888C283C62702B7
:10269000B3C5D5209385A50C54471395164948C753
:1026A0000F100000184237060200860510C71306F7
:1026B000000890CB6CD354C7828088421375F5F71D
:1026C00088C283C62702B3E5D5209385E50EE9B716
:1026D000411126C2AA8706C622C42E85972400006F
:1026E0009384448DB285C9EF9C40F8537DFF370732
:1026F000020098C79727000023A207F2B7E700E07F
:102700003707200037F400E023A0E728130404D0A3
:102710001C48ED9B1CC81C4893E787031CC873002A
:10272000501015379727000083A707889843131781
:10273000772998C3D857719BD8D79727000023A52E
:1027400007EE9727000023A907EC9C40094798C390
:102750001C4893E787001CC873005010944017274B
:102760000000130727EB1C47858B91E75C47858B9F
:1027700099E3FC52EDFBB240224492444101828035
:102780000D47639AE7049727000023A907E89727D6
:10279000000023A707E8B7E700E03707200037F479
:1027A00000E023A0E728130404D01C48ED9B1CC8BC
:1027B0001C4893E787031CC87300501069359717AE
:1027C000000083A7677E98431317772998C3D857CB
:1027D000719BD8D7B5BF0547E392E7F837F700E01C
:1027E000130707D0144BED9A14CB144B93E68603D2
:1027F00014CB73005010984050479316164954C795
:102800000F1000009840B706020014C79306000896
:102810009725000023A8D5E09716000083A6C67868
:10282000944293D67648639FF6009307E0187CD3D2
:1028300050C737F700E0832707D193E787002328A5
:10284000F7D019BF9307E01ADDB79717000083A7E9
:10285000E77589CFD44303A88700984233670701FF
:1028600098C2D447DC4B9842D98F9CC20547971732
:10287000000083A767739505631BE5029843136700
:10288000070898C3984F137707C01367A71398CF0B
:1028900013078007B8BB939735009387C70319C206
:1028A0009317160017270000232AF7D88280984331
:1028B0001377F7F798C3984F137707C01367271359
:1028C00098CF1307F007B8BB93974500F9B7971750
:1028D000000083A7276E8847D847798D01C988C72C
:1028E0009717000083A7C76C91C38287828089678E
:1028F000171700000327076C938707F47CD39716FC
:10290000000083A6266C83A7060993D7A74991C721
:1029100083A7060993D7974999E37C53EDF7828003
:10292000AA87171500000325A55711E182803A21D7
:102930006315B7001821E30BF7FE4845FDB74111B9
:1029400022C406C626C24AC02E849DCD13F91500A6
:102950008147414763040904131745003E97B14678
:102960003307D7029714000083A40454B317F02848
:1029700033C90708BA949C40C840829723A004003A
:1029800023A2040033448900B240228522449244A9
:10299000024941018280B356F448DDFE8507E39C7D
:1029A000E7FECDB7011126CA06CE22CC4AC84EC6D4
:1029B000AE84B1C593F7150001444147A1CF9317E9
:1029C0004500A2973147B387E70297190000938922
:1029D000A94D03A909003E998327090081C7032552
:1029E0004900829731473307E40283A70900BA9769
:1029F0009C478DC733148028B3470408BD8CF24030
:102A000062444249B2492685D24405618280B3D6E8
:102A10008448D5F60504E31CE4FECDB72320090065
:102A200023220900C1BF7971B7E700E022D48043B7
:102A300052CC06D626D24AD04ECE56CA5AC85EC608
:102A400062C43A8A37072000798C23A0E7180F1058
:102A5000000005E123A087100945B250225492548A
:102A60000259F249624AD24A424BB24B224C45616A
:102A700082809717000083A72742B6892A89AE8AE9
:102A8000328B971B0000938B2B42829703A70B007E
:102A90008144B146C147338CD402330687011042CA
:102AA00041E2C165938505F04145EFD07F8919ED7D
:102AB0009717000083A7875F81C7814511458297DB
:102AC000B7E700E023A087102D4541BF171700008E
:102AD0001307073D1C43A1E308C323000500B317F8
:102AE00090283EA183A70B0023260500232465011F
:102AF00023224501E29723A0270123A2570123A403
:102B000047016384090023809900B7E700E023A010
:102B10008710014599B73E87DC47F5FF48C775BF69
:102B20008504E39AF4F6B7E700E023A08710214577
:102B30002DB70111B7E700E022CC80433707200012
:102B400006CE26CA4AC8798C23A0E7180F100000C9
:102B5000BD4763E9A70431473307E5029717000033
:102B600083A78734BA979C4395CF3315A0282E8925
:102B7000B345050801452EC66533AA8409C9B24587
:102B80000145971004E0E780407923A42401B7E7CA
:102B900000E023A087100145F2406244D24442493C
:102BA00005618280B7E700E023A087100945EDB7F3
:102BB0009716000083C6867E9717000083A74737C5
:102BC00001476394E600014582808E2313868702C5
:102BD0006394A5003E85828005071377F70FB287BF
:102BE000CDB79717000083C7777BAA86850717158F
:102BF00000000325A534014712216307D60005070D
:102C00001905E36BF7FE014582802A87171500003E
:102C10000325453311E182801C45B227636BC70051
:102C200003584500B306C8006355D7008146639436
:102C300006010841C5B703D3A700938807016316AF
:102C4000E30091C192A13E8582808506C687B3C606
:102C50000608F1BF9716000083C646749717000058
:102C600083A7073101476394E60001458280AE23C4
:102C70001386C7036394A5003E85828005071377FA
:102C8000F70FB287CDB7411122C406C697170000CF
:102C90002384077C171400000324842E05C06C399C
:102CA0000145B315B028B3C50508972004E0E780B7
:102CB000E0B3930710273305F50202942244B24093
:102CC000814501454101172304E0670023BC383DDD
:102CD00009C734256312D7027DB73C2DF5DF3825AF
:102CE000E30CF7FE3CA5814517E5FFFF1305653EA4
:102CF000172304E0670083B93C2D89C7E394F6FEEF
:102D000038A5D5B7F1FAEDBF41114AC01729000027
:102D1000130949908327890022C426C206C6971446
:102D200000009384246C858BE0509DCB9727000096
:102D300023A6078E83C74407C18B85CFEF00507051
:102D400083C7440793F70702E5DF83C7440722855B
:102D500093F7F70C238AF406974005E0E78060D9E3
:102D6000EF00106E22852244B24092440249410194
:102D700019BF83C75407858B91CBEF00706C8D47CB
:102D8000230EF406BC5822858297D9BF83C7440717
:102D90001547BD8B6393E7048347B40603453406A8
:102DA0000146930550025D8D4D3401468145054530
:102DB00005328327C900858BC5D722859727000058
:102DC00023A00786974005E0E780C0BA51F9B240DA
:102DD0002244924402494101828083C74407194733
:102DE000BD8BE39FE7F68347B406034534060146EF
:102DF000930550025D8D913C014681450545EFF0FC
:102E00003F8D8327C900858BA1DF2285972700008E
:102E100023A80780974005E0E780608F45BF4111F8
:102E200022C426C206C67C2578452A84BD8B1CA9EF
:102E30001CA31D476445639BE7340547B8A083473F
:102E4000F5058D466395D7185E2DCDE37C49114776
:102E5000B18B638DE70831476398E7000347150698
:102E60008347F5076304F7088547BCB01946930507
:102E7000640313854400EFD06FFCBC20990793F7DF
:102E8000F70FBCA0034704061377070401CFB8303F
:102E900013670704B8B07844BA975838B8B3BC2061
:102EA0008507BCA0971700002388075ABC2013F79A
:102EB000F703050718B80347E4051A07D98FBCA024
:102EC00083475403858B91E703474403894763177E
:102ED000F70078441C2393E707041CA37C441838AC
:102EE00098B3B2402244924441018280A147BCB0D1
:102EF0008357C406971500009385C54E171600002A
:102F00001306460BDCA08357C4060347140674441B
:102F1000A1831207BD8BD98FDCB2B4208547890607
:102F200093F6F60FB4A0171700000347E752631E8D
:102F3000F706183C9387E6008E07231AF40693875A
:102F4000C708B387E702794510420948238A050775
:102F5000C1650CC6938707FBB3C70708938777162D
:102F6000B3C7A70233C70708B387A70286073CD2B7
:102F7000BC3093E70701BCB07C44B6978346240677
:102F800093E60604B4B3B4207C44B697D8A3B42027
:102F90007C4421837D8BB697834634069606558FF5
:102FA000D8B3BC208D07BCA011B71042F9473852E6
:102FB00005833357F7023C5268528583FD8BAA97ED
:102FC0007CD28D47238AF5063347070855B7194643
:102FD000639DC7125E2DC1E393056503B8B01385E9
:102FE0004400EFD0AFE5BC201385A4009907BCA036
:102FF000BC3093E72700BCB083475403898B95CF3F
:103000000C58BC299DCB1946D105EFD02FE378444D
:103010001C2393E707F81CA3BC20990793F7F70F2D
:10302000BCA00347040613770704E30D07E6B4309A
:10303000784493E60604B4B085B58347D40391C7BA
:1030400078441C2393E707F81CA319469305E4036F
:10305000EFD0CFDED1B7A147BCB08357C506DCA007
:103060008357C506034615066C45A1831206BD8B22
:10307000D18FDCB1B020171500001305A5369715C8
:103080000000938525F309061376F60FB0A0971775
:10309000000083C7673C6398E704183C9307E60089
:1030A0008E07231AF4069387C708B387E702794887
:1030B0008946230AD5069441C1658CC6938707FBD0
:1030C000B3C7070893877716B3C7070333C7070843
:1030D000B38707038607BCD2BC3093E70701BCB0B7
:1030E0007C44B29761BD8C41B851F9470583335791
:1030F000F702BC5103A845068583FD8BC297FCD11E
:10310000230AD50633470708C1BFA147BCB0835780
:10311000C506DCA08357C506034615066C45A1838A
:103120001206BD8BD18FDCB1B0201715000013053E
:10313000652B09061376F60FB0A09717000083C71A
:10314000A7319715000083A5E5E6E39FE7F8183C53
:103150009307E6008E07231AF4069387C708B38700
:10316000E702F9460948230A0507416588C59387A0
:1031700007FBB3C7070893877716B3C7D70233C7D0
:103180000708B387D7028607BCD1B9B70547639E46
:10319000E706B1471CB983475503898BA1CB0C596E
:1031A000BC29A9C71946D10513858400EFD00FC9E2
:1031B00078441C2393E707F81CA368441946930539
:1031C00064030905EFD08FC711679717000083A725
:1031D000672EF98FE38607CE7C24B98BE39207CE66
:1031E00078441C2393E707021CA3D9B98347D4036F
:1031F00089C79C2093E707F89CA06844194693056B
:10320000E4032105EFD08FC34DBF522D0C5593071A
:10321000660093F7F7031CB913858400E5B7011125
:1032200026CA971400009384E43E9C4422CC06CE28
:10323000171400001304041B858B6850D9C32AC6D9
:103240009717000023AC073CEF00901F034744078B
:10325000894732456307F700034744078D47631EDC
:10326000F7029716000083A6E6D4BC520357450721
:1032700085831307C71263F2E702BC528583B1C38B
:10328000914703474407E31EF7FE6244F240D244ED
:103290000561174305E06700A3AE382D3C3D09CF1B
:1032A00034256309D7026388F60238A56244F240E8
:1032B000D24405616FD03FC399CF382509EF3CA5B3
:1032C000F5B72AC6EF00D01762443245F240D24427
:1032D000056155BAEDF7DC4CEDF703474407894724
:1032E0006307F700034744078D47E31CF7FC91474A
:1032F00003474407E31EF7FE49BF6302053201118D
:1033000022CC06CE26CA4AC84EC652C456C258253A
:1033100085472A84631AF72C971700009387872F15
:10332000D44F1547638AE600D44F0D476386E60005
:10333000D84FAD476314F7026C386244F240D24470
:103340004249B249224A924A01450561B315B02863
:10335000B3C50508171304E0670003F81631130717
:103360000064971400009384E4073347D7029C203D
:10337000E8D0850793F7F70F9CA063CAE700972072
:1033800004E0E780A08E97170000238D07047824BF
:103390009D47631FF70483479406B1C38356040710
:1033A00063ECF6020C24930730041CAC13053004C4
:1033B00093F6F60F0146977006E0E78080B7228506
:1033C0006244F240D2444249B249224A924A0561DB
:1033D000174305E06700034A85062318D4069305C2
:1033E00030020545972004E0E78080802301A40691
:1033F0000549238A2407183C8D47631CF70E971054
:1034000004E0E780E0E30D89630F051463162517D8
:10341000930760023CA4930750023CAC93077002F0
:1034200078243CBC85476302F70889659385F5706D
:1034300013051027171A0000130A4AC9834974019B
:10344000971004E0E780407D0E30835ACA002A8935
:1034500013060064B3855503814613850532B335E1
:10346000B50097A006E0E7800022AA84B33559038F
:1034700037460F001306062481463305590397A0EB
:1034800006E0E780402083270A00AA948297B307CA
:10349000950003278A00BE8563E4A70063E4E70084
:1034A000B385E7404E85EFF0CFE883475403898B1F
:1034B000E9CB8347C403F1C70C58E1C5BC25F1C370
:1034C0008947230AF4021946B10513056403EFD0B6
:1034D000EF960347C407894763E9E70A22856244F8
:1034E000F240D2444249B249224A924A05616FD021
:1034F0009F9F89467C346315D70213F7170019CBB9
:10350000898B1307500291EB9307700238A43CACEF
:10351000814739B713076002C5BF93076002FDB743
:1035200099CF93F617001307500291E6898B13B7D2
:1035300017001307670238A4230D0400D1BF3C2CE9
:10354000130740026368F700930750023CAC3C2C21
:103550003CA47DBF850793F7F70F3CAC13077002BF
:10356000E364F7FEEDB713077002930750023CAC1B
:1035700038A4930760026DB51307500293077002D9
:10358000FDB78547230AF402A9B70327C40A971693
:10359000000083A666903C27ADC31C3758339714B0
:1035A00000009384A4B29044B387E702DA24B3877F
:1035B000E7021307003293870719B3D7E7020327FF
:1035C00044093E973A896364F7006364C70033098E
:1035D000C7408296B307A9406374A9009844BA977C
:1035E00003576407E3FCE7EEF2406244D2444249E9
:1035F000B249224A924A05618280832484098296D4
:1036000063E9A400835764073385A440E378F5ECAD
:10361000E1BF9717000083A7E7ABBE94E5B78280B0
:1036200001114EC6971900009389C9DB22CC03A46F
:10363000C90926CA97140000938444A9DA244AC809
:10364000035964088327040906CE3309E902374782
:103650000F009306F7231307072452C456C25AC01B
:1036600036993359E90263E02705171A0000130A57
:10367000AA823389274183270A0082976368A902B7
:103680003305A9406347050283570404A30F0400D0
:1036900085072310F40483470414639707102285D9
:1036A000EFD01FE429A29844BA97C1B79C443E9931
:1036B000C1BF83270A008297032784086363E50A52
:1036C000198D7E3CDA248E07B387E7021307003298
:1036D00093870719B3D7E70263E9A708B74A0F0032
:1036E000138BFA23938A0A24835704048507231033
:1036F000F4048347041481E72285EFD07FDE22851E
:10370000975005E0E78040FF631305240326040972
:103710000327C40894443297BA876364C70063647C
:10372000D700B307D740783CD2242328F4080507F4
:1037300078BC035764083307C7025A9733575703B7
:103740003389E74063F5E700998E3389F6008327D4
:103750000A0082976365A9043305A940E34605F88A
:1037600025B79C44998F3E95A9BFA14522859750C6
:1037700005E0E78080F0A305A4029717000083A767
:10378000E7926386071C6244F240D2444249B24940
:10379000224A924A024B89451545056182879C441D
:1037A000CA973385A7405DBF2285EFD0BFDD228554
:1037B000975005E0E78040F4631B0518CA2483573F
:1037C0006408B7460F001386F623B387A7029386D3
:1037D000062403270409230B040283AA8400B2975A
:1037E000B3D7D702636FF716B307F7408326C40831
:1037F0002324F408014BB387E6003E8963E4D70035
:1038000063E45701338957411E3023282409A1CB93
:10381000835604045A3037460F0056B03387E640CB
:10382000B387E7023A301306062481468145BA97EA
:10383000B3C707083385A7023EB097A006E0E7802C
:1038400080E411CD4A9533392501CA95AA876314BE
:10385000BB0063645501B30755412328F40883274F
:103860000A0082972A8983270A008297E30D25FFA1
:1038700083270A000329840882976369A90E330508
:10388000A9406306051003DAC4008357640837496A
:103890000F001307F923B387470313090924BA97C5
:1038A000B3D72703170700000347D77EBA9763E013
:1038B000A70EB3352503035B2402528681463305E8
:1038C000250397A006E0E78000DCB30AAB003305D0
:1038D0004B0337460F00130606248146814597A007
:1038E00006E0E78040DA15C1B337250352868146EA
:1038F000B305B9023305A902BE9597A006E0E7809B
:1039000080D8330BAB402311640335455D2E23AEC5
:10391000890838348547631EF704930700FD7CA4AB
:1039200017050000032585679C28A1CFEFD0CF990C
:10393000954717170000232DF7CE3707100097077C
:10394000000083A7276798C7860A23A85707F24075
:103950006244D2444249B249224A924A024B05612A
:103960008280B3065701B387F64049B59C443E991F
:1039700039B7930710FC7CA4170500000325856167
:1039800065B78145971004E0E78040F055B7971779
:10399000000023A707AE9C2885C717050000032554
:1039A000655E971004E0E780C02B6244DC40F24083
:1039B000D2444249B249224A924A024B0561828767
:1039C000834594026244F240D2444249B249224AB9
:1039D000924A024B01450561B315B028B3C50508ED
:1039E000171304E06700438F011122CC26CA4EC68C
:1039F00006CE4AC852C456C25AC0383585478324B9
:103A000005092A84AE896314F70C83570508835A85
:103A1000C503170A0000130A6A6B035BCA0063FE42
:103A200057191429639BE618032785116317071894
:103A30000327450A6313071874351D47639FE6166D
:103A40002A3DB38AFA409307204E330555030329D4
:103A5000440937460F001306062481463305F50254
:103A60009707000083C7076333592503B335AB02BB
:103A70003E9933490908231324093305AB0297A063
:103A800006E0E78040C0B307950033B5A7002E9548
:103A900003278A00BE8419E163E4E700B384E740AA
:103AA000B307690337470F009306F723130707246B
:103AB00023A09900B697B3D7E702D69763E4F40042
:103AC0009D8C31A003278A00B307F740BE941709E5
:103AD00000001309693C8327090023A099008297FD
:103AE00063E2A4103385A440635D050A83270900BF
:103AF000170B0000130B8B5D829703A70900636906
:103B0000E50E198D7E3C0357CB008E07B387E70285
:103B10001307003293870719B3D7E70263EFA70CA7
:103B2000374A0F00930AFA23130A0A24835704041E
:103B300085072310F4048347041481E72285EFD01E
:103B40003F9A2285975005E0E78000BB61E5832618
:103B500004098327C40803278B00B697BE8463E457
:103B6000D70063E4E700B384E7407C3C8356CB0096
:103B70002328940885077CBC83576408B387D70241
:103B8000D697B3D7470363E6F40A9D8C83270900D1
:103B900023A09900829763E1A40A3385A440E347F8
:103BA00005F89707000083C7F74E63E6A706971747
:103BB000000023A7878C0145B9A8835764083747BD
:103BC0000F009306F723B387670313070724B697FD
:103BD000B3D7E702E3F6F4EE03278A002697B3048F
:103BE000F740F5B59707000083A7C74EBE94DDBD2B
:103BF00083278B00998F3E9531B7A1452285975039
:103C000005E0E78080A7A305A4029707000083A72B
:103C1000E74981EF7D55F2406244D2444249B249BE
:103C2000224A924A024B0561828089451545829756
:103C3000D5B71D8FBA9499BF83278B00BE94B1BFAF
:103C400097060000938606379C42B84B1377F78F90
:103C5000B8CB98431367870098C39C4393D73748E2
:103C600089C70100010001000100170700000327B8
:103C7000A7331C4393F7F7CF93E707101CC317062E
:103C80000000032626341C463707CEFF7D17F98F28
:103C90001CC69C4237070300B8CB9707000083A7D8
:103CA000E73099CBD44390479842518F98C2944BB8
:103CB000DC4B9842D98F9CC29717000023AA079625
:103CC00082809707000083A7E72E9C438D8BF9C75E
:103CD0004111B7E700E04AC003A9070026C2370731
:103CE000200006C622C4AA843379E90023A0E7187D
:103CF0000F100000171400001304C491584C8D4796
:103D0000631AF7009707000083A7876A0146814579
:103D10004545829719476393E4048347140289CB8E
:103D2000834704026396970097170000A3840790C7
:103D3000584CA1476315F700930780101EB09707F2
:103D4000000023870714ED3DB2402244B7E700E0AE
:103D500023A0271192440249410182809D47639B21
:103D6000F40083471402E9D7034704028D47E311A7
:103D7000F7FC5DBF544C6389E600584C6306F700BE
:103D8000584CA147E31DF7FA83471402CDFB5C4C66
:103D90002300F4028547A300F40255B78280000097
:103DA0002A8309CA83830500230073007D16050357
:103DB00085056DFA82802A8311C62300B3007D1623
:103DC000050365FE82809707FC1F83A7A7E01707FE
:103DD000FC1F0327A7DF01456313F7008280F6234A
:103DE00099E2D62336959C43C5BF1707FC1F1307DE
:103DF000E7FD1C435A23411193860711E117BA9737
:103E000085651706FC1F2327D6DC1706FC1F232F0A
:103E1000F6DA06C69D051356370063F4E50013066F
:103E200000203387C6009705FC1F23A3E5DA61163F
:103E300098C2D2A2239306001CC3998FE1175EA3F8
:103E4000231307004937B2409707FC1F239FA7F4AD
:103E5000410182809707FC1F83A7C7D71707FC1F64
:103E60000327C7D601456313F7008280F62381E656
:103E7000D6233375D50A9C43FDB7184183A785FF28
:103E80006319B7001CC1FD5723AC05FE238FF5FE57
:103E90008280232CF6FEC5BF411122C437E400E026
:103EA00026C204403707200006C6F98C2320E418F8
:103EB0000F10000009E9232094101545B240224458
:103EC0009244410182800347E5FF9307F00F6306A8
:103ED000F700232094101145D5B797C0FB1FE7804A
:103EE0008028014523209410D1BF41114AC037E9F1
:103EF00000E022C403240900B707200006C626C23A
:103F00007D8C2320F9180F10000089E523208910EB
:103F1000154515A0AA849707FC1F83C7B7E82E850F
:103F200063F5F400894763EE9700BD37B7E700E01B
:103F300023A087100D45B24022449244024941011A
:103F4000828083A785FF99E703C7E5FF9307F00FFA
:103F50006308F7009137B7E700E023A087104DBF53
:103F6000238F95FE1705FC1F130505C797C0FB1F80
:103F7000E7806030A16526857520014523208910E2
:103F80005DBF9707FC1F23A907C482804111B7E7D3
:103F900000E026C284433707200006C622C4F98CFD
:103FA00023A0E7180F1000009707FC1F83A707E462
:103FB0001704FC1F130484B991C782971C40AA9769
:103FC0001CC031A09707FC1F83A707C2FDF708405C
:103FD000B74703009387D73F3305F502B7A72600FD
:103FE000938737ECB2403E9508C02244B7E700E023
:103FF00023A09710924441018280411122C406C639
:104000009707FC1F83A707BE1704FC1F130484D95E
:1040100089C782975C48AA975CC84848B240224446
:1040200041018280B7E700E09843B706200023A053
:10403000D718758F0F1000009706FC1F83C696D601
:10404000637FD5009706FC1F83A6C6BA3325D5200B
:104050001621D58D0EA123A0E7100145828023A053
:10406000E7100D458280B7E700E09843B7062000CF
:1040700023A0D718758F0F1000009706FC1F83C66A
:1040800076D26370D5029706FC1F83A6A6B63325A9
:10409000D5201621B3F5B6400EA123A0E7100145A7
:1040A000828023A0E7100D4582807971B7E700E098
:1040B00026D284433707200006D622D44AD04ECEDB
:1040C00052CCF98C23A0E7180F100000930705FFCE
:1040D00093F7F70F7D476363F70A31473307E5022C
:1040E0009707FC1F83A747B1BA979C43C1CB1354D2
:1040F00045003D893315A028AE89B34505082285C2
:104100002EC697E0FB1FE780E0562A8939C9B245E1
:104110002285170AFC1F130A6AD0B1379707FC1FC4
:1041200083A787AC82978357CA002A848146338746
:10413000370313060064B3B7370313050732B335EB
:10414000E500BE95EF90E228B307850083268A003C
:104150003E8763E4A70063E4D7003387D740232476
:10416000E900B7E700E023A097100145B2502254C0
:1041700092540259F249624A45618280B7E700E0F1
:1041800023A097100945DDB7797122D437E400E008
:104190004AD003290400B707200006D626D24ECE07
:1041A00052CC56CA5AC85EC63379F9002320F41897
:1041B0000F1000009707FC1F83C7D7BE6378F50078
:1041C000970BFC1F83AB4BA263970B00B7E700E094
:1041D00023A0271199A0970AFC1F938A2AC403AB36
:1041E0008A00B74736FE938707C83E9B83D7CA002D
:1041F0002E8AAA84B385C702B2898146B3B7C702A3
:1042000013850532B335B50013060064BE95EF90F3
:10421000421C6370AB02232024110145B25022548A
:1042200092540259F249624AD24A424BB24B45611A
:104230008280829B83D7CA002A8413060064B385D8
:1042400037038146B3B7370313850532B335B5005D
:10425000BE95EF900218B307850003A78A003E843D
:1042600063E4A70063E4E7003384E740D285268552
:1042700097E0FB1FE780004001C900C5B7E700E0F9
:1042800023A02711054559BF93E504F04145B3C567
:10429000050897C0FB1FE780E0DF11E99707FC1FC7
:1042A00083A7C7B585D7A6851145829705B7170798
:1042B000FC1F1307E7931C4389EF08C38547232698
:1042C000050000C52311450104A11CB123220500EE
:1042D00075B73E87DC47F5FF48C7CDB77971B7E7BB
:1042E00000E026D284433707200006D622D44AD0E5
:1042F0004ECE52CC56CA5AC85EC662C466C2F98C4B
:1043000023A0E7180F10000035C12A892E8AB28A2F
:10431000B6894144B14C170BFC1F130BEB8D130CEA
:104320000003B30B940383270B00DE979C43B9EF84
:10433000135544409375F40056861375F50FB31565
:10434000B028B3C50508893531C183270B00DE9736
:1043500023A0270123A24701638409002380890049
:10436000B7E700E023A09710014521A023A09710F4
:104370000945B250225492540259F249624AD24A33
:10438000424BB24B224C924C456182800504E31AA9
:1043900084F9B7E700E023A097102145D9BF0111A8
:1043A00022CC37E400E026CA04404AC84EC652C4B4
:1043B00006CEB70720002A892E8AB289FD8C2320D9
:1043C000F4180F100000C933D2854A8597E0FB1F0F
:1043D000E780402A01ED232094102145F2406244F9
:1043E000D2444249B249224A056182809707FC1FA4
:1043F00083D787A3B38537032A89130600648146D0
:10440000B3B7370313850532B335B500BE95EF80DA
:10441000527C2322A900232094100145C1B7011129
:1044200026CAB7E400E04AC803A9040022CC4EC65D
:10443000B707200006CE52C4AA892E843379F9002A
:1044400023A0F4180F10000097E0FB1FE7808022E4
:10445000170AFC1F130A0A951DE1A2854E8521311A
:1044600083470A006382370523A024111945F240CF
:104470006244D2444249B249224A056182802311F2
:104480000500A2854E85C53683470A00638637013D
:1044900023A024110145E1BF17F7FB1F1307677421
:1044A0001E23C18F1EA3EDB797F7FB1F938767737A
:1044B0009A23598C82A34DBF01114AC837E900E005
:1044C00022CC03240900B707200006CE26CA4EC618
:1044D0007D8C2320F9180F1000009307F00263E78A
:1044E000A704B144B304950297F9FB1F9389C970DF
:1044F00083A70900A6979C4395CB9375F50011817E
:10450000B315B028B3C50508193F83A709000145B5
:10451000A69723A0070023A2070023208910F240BA
:104520006244D2444249B24905618280B7E700E063
:1045300023A087100945E5B74111B7E700E026C27F
:10454000844306C622C437072000F98C23A0E7184D
:104550000F10000097E0FB1FE780C01119E901452B
:10456000B2402244B7E700E023A0971092444101F3
:104570008280004597F7FB1F83A7076782979707FD
:10458000FC1F9387A7896367A4029847B74636FE46
:10459000938606C83305A4403697E372E5FC1307FB
:1045A0000064B335E502D22781463305E502EF808A
:1045B00052627DB798473A94C9BF411106C697F732
:1045C000FB1F23A1A7620295B24097F7FB1F23A709
:1045D000A77E014541018280914763E9B7009707B3
:1045E000FC1F93876782B3C5F52088C18280411183
:1045F000514681451705FC1F1305058106C622C4D7
:1046000026C297F7FB1F23A5075E97F7FB1F23AB77
:10461000075C97F7FB1F23A9075C97F7FB1F238114
:10462000075C97F7FB1F23AB075A97C0FB1FE78078
:10463000A0DC13068002814517F5FB1F1305857664
:1046400097C0FB1FE78040DBEFF02FFA97F7FB1FC7
:104650009387C777E82BFC3B17F4FB1F1304847484
:1046600085453E958D473305F502994797F4FB1F25
:104670009384845839051375F50F28A03305F50286
:10468000130505243345050897C0FB1FE78080A06C
:1046900088C035C93020994781453306F602130694
:1046A000062497C0FB1FE78020D59C40382097F454
:1046B000FB1F9384A453938707249CC0B347F72020
:1046C00017F7FB1F2328F7526D381D211C3094402B
:1046D00017E6FB1F1306460233C7D72010C3138704
:1046E00017001377F70F17E6FB1F130686FA3347F9
:1046F000D72010C313873700890718B093F7F70F37
:10470000B3C7D72090C3B240224492444101828073
:1047100097F6FB1F938606692A87BC228832637D41
:10472000F5001306150097F7FB1F83A7274C90B2DF
:10473000B347F52098C382801305F00F82801C4197
:10474000E5CB370700F07D8FB7060020894763125D
:10475000D70E5A21411122C406C62A8469C71946B8
:104760009305F00F690597C0FB1FE78000DD054743
:104770008D47630AE50A1C4491C75858994745C7B5
:10478000185C55C31306C003814517F5FB1F1305BD
:10479000E56397C0FB1FE78020C61306C003A28510
:1047A00017F5FB1F1305856297C0FB1FE78040BE0E
:1047B00097F7FB1F93878761DA2701E7130700103C
:1047C000DAA7F82719E30547F8A79A2B19E36D47ED
:1047D0009AABF83719E31547F8B7B82B19E3054733
:1047E000B8ABB83B19E3F837B8BBD83B11C79376E1
:1047F00037000983F4ABF8BBD82B19E35547D8AB86
:10480000182C01E71307C00398AF9C5791C78297F4
:1048100097F7FB1F239CA758FD5717F7FB1F230192
:10482000F758F1338147B24022443E8541018280EE
:1048300089473E85828079714ECE97F9FB1F938917
:10484000E95D83A7090006D622D426D24AD052CCED
:10485000829713090064B335250303D6C900814646
:1048600017FAFB1F130A0A5432C633052503EF80DB
:10487000523683248A012A840145638684023246A3
:104880003305944063EF840003A589008146B33566
:10489000A9023305A902EF80D233B30795403385CF
:1048A0008700232C8A00B250225492540259F249B4
:1048B000624A45618280011122CC0A852E844146DC
:1048C000979502009385C5EB06CEEFF06FCD1808E3
:1048D0003324E420035704FFF240624497F7FB1FA0
:1048E00083D7A75437450F00BA97130505243355CE
:1048F000F5020561828097F7FB1F83D70753514765
:104900001D45637CF702794719456378F702130761
:10491000200315456373F7021307B0041145637E46
:10492000F700130740060D456379F7001307600988
:1049300009456374F70013B5B70F8280411122C493
:1049400026C22E84AA8406C6058CEFF02FE4B32776
:10495000A402B2402244338597001375F50F9244A8
:1049600041018280411122C426C22E84AA8406C637
:10497000058CEFF0AFE1B327A402B24022443385A7
:10498000970033450508924441018280411122C4B9
:1049900026C22E84AA8406C6058CEFF02FDF33359D
:1049A000A402B2402244269592444101828097F7A6
:1049B000FB1F23A5A724828041114AC017F9FB1FC2
:1049C0001309C9408327890206C622C426C28DCF97
:1049D000829797F4FB1F9384E43C9E242A848DC71E
:1049E00033F7A70A33470708B3D7A70AB3C707089F
:1049F000B307F74051476359F7008327C90291C3B2
:104A00008297EF10822382A4B2402244924402494A
:104A100041018280011122CC97F7FB1F23A0071EC2
:104A200017F4FB1F1304843A5C5406CEAA8581C791
:104A30002AC68297B245C1C19C410545ADCB9C4574
:104A4000BDC7DE25ADC7FE25BDC39C2981CB7C2813
:104A50007838BA97634DF504DC41B1CB13064002B8
:104A600017F5FB1F1305853B97C0FB1FE78040929E
:104A700097F7FB1F9387873A984397F6FB1F23A569
:104A8000E616183C19EFCA279307805737460F00E0
:104A90003305F5021306062481468145EF80721323
:104AA00008BC17050000130545D9013E0145F24039
:104AB00062440561828097F7FB1F23A3073097F7B5
:104AC000FB1F9387A73517C7FB1F130767F398C30F
:104AD00037873200FD56130727A194C7D8C797F729
:104AE000FB1F23850734B7C7004023A4D72649B747
:104AF000011122CC17F4FB1F1304442D084406CEE9
:104B000026CA4AC801E90545F2406244D2444249F6
:104B1000056182805C58E5DB185C75D770008545BF
:104B200082971844B247E300F7FE4A249305E00455
:104B300017F9FB1F1309092797B0FB1FE780805562
:104B40002320A90269D152249305F00F814497C014
:104B5000FB1FE780608A7C240326090263C1F402FC
:104B6000328597B0FB1FE7800060014597F7FB1F78
:104B700023AA072497F7FB1F23A8072471B74E2405
:104B80001844B3879502898185043385E7001C5C4E
:104B900008C28297C9B7011122CC17F4FB1F130476
:104BA000E4221C4426CA4EC656C206CE4AC852C487
:104BB0005AC0AA84AE89B28A6388071A585839CB7A
:104BC0001307F01F6366A71017FAFB1F130A8A1D4D
:104BD00003290A02631209044A249565938515E0A6
:104BE00097B0FB1FE780004B2320AA022A861DC135
:104BF0004E245C580844898182971C4403290A0288
:104C00002322FA028947639EF402C1479305090CE7
:104C10006381F9042945BDA003274A02E384E7FE26
:104C20004A249565938525E097B0FB1FE780804671
:104C30002A896DD14E242A865C580844898182973E
:104C4000D1B78D47639AF404C1479305490DE393A7
:104C5000F9FCB8219307A0056312F7069E21639F14
:104C600097044E869105568597B0FB1FE7804072EA
:104C700083270A02638727014A8597B0FB1FE780D5
:104C8000804E0145F2406244D2444249B249224A30
:104C9000924A024B0561828091476397F400930525
:104CA000890EE39999F675B793070010E394F4F62B
:104CB000A147E3E137F79305090F61BF83270A0294
:104CC000E38A27F54A8597B0FB1FE780C04999B76B
:104CD0001D67637FE506130705E099463347D70252
:104CE000562417FBFB1F130BEB0B3307D702330ABA
:104CF000F70083274B026396470103290B026311D8
:104D000009024A249305E00497B0FB1FE78080382E
:104D10002A8909D14E245C582A8689815285829736
:104D200091451307A00593F5C50FB307B900B42348
:104D30006399E60296236394960291054E86CA957E
:104D4000568597B0FB1FE780A06483270B021DB731
:104D5000A166F916E3E0A6EC3307E54051B7AC33A2
:104D6000D9B783270B02A9BF97F5FB1F83A585053C
:104D7000E38205EA91479306A00593F7C70F3387AF
:104D8000F5003023E318D6E81223631B9600910741
:104D90004E86BE95568597B0FB1FE780605FD5B500
:104DA0003C33E1BF97F7FB1F93874702984721C722
:104DB000985F31C385466310D504411122C417F4AE
:104DC000FB1F130424FE105006C615C2CE27485000
:104DD00089810297085097B0FB1FE780C03897F78A
:104DE000FB1F23A107FE97F7FB1F23AF07FCB24071
:104DF000224441018280828001114AC817F9FB1FB9
:104E00001309C9FC4EC68329890022CC26CA52C484
:104E100006CE56C2AA842E84328A638B091A83274F
:104E2000890399EB2945F2406244D2444249B24990
:104E3000224A924A0561828083274903E5D7930776
:104E4000F01F63E0A70C97F9FB1F9389A9F583A7CF
:104E5000090295CF0325890083A749026395A7041A
:104E60008947639FF404C147E31EF4FA03A50902CE
:104E70001305050C9307A0053CA106A12286D28547
:104E8000110597B0FB1FE780A050014569BF03558E
:104E9000C9009305E00497B0FB1FE780A01F23A083
:104EA000A9024DF941B78355C9008327490303A6D9
:104EB0000902898182978327890023A2F9024DB7CD
:104EC0008D47639AF400C147E31EF4F403A5090279
:104ED0001305450D45B791476399F400E31494F425
:104EE00003A509021305850E71B793070010E39B14
:104EF000F4F2A147E3E887F203A509021305050FC1
:104F000095BF9D676373F506930705E01947B3C71F
:104F1000E7020357C90097FAFB1F938AAAE8B387F1
:104F2000E702BE9983A70A02A1CB83A74A02639135
:104F3000370703A50A0291479305A0051308F00F50
:104F400013F7C70FB306E500B0226313B60683D884
:104F50000600B032639C9804B307F64063C687042A
:104F600011072286D2853A9529BF21677917E36B0D
:104F7000A7EAB307F54071BF0355C9009305E004E4
:104F800097B0FB1FE780001123A0AA0259FD59BD6D
:104F90008355C9008327490303A60A0289814E85E8
:104FA000829723A23A0371B723900601B28749BFC3
:104FB0003386870011061308F00BE365C8E6ACA240
:104FC00013063400719A1106B29786A2BCB249BF8B
:104FD00097F9FB1F938909DD83A709029DCB03A5E0
:104FE000090291471308A0059305F00F13F7C70FA7
:104FF000B306E500B0226310060583D80600B03280
:1050000063979800B307F640E3DC87F48EA2B2877B
:10501000F1BF8347E9000355C9009305E004330558
:10502000F5023345050897B0FB1FE780A00623A0D3
:10503000A90255F5C5BB0356C9008345E900B385F0
:10504000C502338687001106E3EEC5DC2381060125
:1050500085BF014582809C211CA1BE211CB1BE21BF
:10506000A1833CA1DC213CB11145828097F7FB1F55
:1050700023AA07B897F7FB1F23A407B882800DCD9A
:10508000411122C426C206C6AA842E84014585C1C8
:1050900022854146978502009385857197B0FB1F55
:1050A000E780002F9C2005455CA49C305CB4B24096
:1050B000224492444101828001458280011122CC28
:1050C00026CA06CE8947AA843284639EF50063838C
:1050D000B602414781476395E6048A854D374146CC
:1050E0008A8522850DA841476392E504638FF60007
:1050F000639EB6022E86A2856244F2402685D24483
:10510000056117B3FB1F6700233B8A853285853F06
:1051100041468A85268597B0FB1FE780E039AA873C
:10512000F2406244D2443E85056182808147CDBF12
:1051300097F7FB1F23A6A7AC828097F7FB1F23A33B
:10514000A7AC8280011122CC622106CE26CA4AC8B1
:105150004EC63DC8832985002A88AE8403C909004C
:1051600081471317496063550702B147054563F648
:105170008704035528005114334404084E863387AE
:105180008900A2868545EFB03000B337A0008507BF
:10519000135569487D141379F903334404089CA01E
:1051A00088B023812401C2A0014719C013871900C8
:1051B00098C409476383E7000145F2406244D24442
:1051C0004249B249056182800545C5BFC167F917EB
:1051D000630AF502D94763F7B702011122CC2EC644
:1051E00006CE2A84EF902006B2456368B50022857A
:1051F0006244F24005616FA0407AF2406244054586
:105200000561828005458280C167F9176314F50046
:105210006F906003411106C6EFA0C06611E15D45C5
:10522000B240410182809147639DF5001C211CA280
:105230003C211831A207D98F3EA23C3101455CA226
:105240008280114582804111814522C426C206C652
:10525000AA849D232A8409E997F7FB1F83A7479A0D
:1052600081C7F94526858297B2402285224492441F
:105270004101828039714ED652D45AD05ECE06DEBC
:1052800022DC26DA4AD856D22A8A2E8BB289B68BED
:105290000DE79D3F9145EF9020092A844D49854AAD
:1052A00019EDF2506254D254B259225A925A025B0A
:1052B000F24B4A854259216182803A84814A230017
:1052C00034018544630A0B00DE8513051400029B3C
:1052D00093041500B3C404089399496063D3090289
:1052E000C1455285EFA04068654915E53306940035
:1052F000A6852285EFB0602F2A8911EDB104B3C4D1
:10530000040891472C0052857C8422C66485EF9066
:10531000707D2A8959D5E3860AF8228597B0FB1F4C
:10532000E78060E4BDBF011122CC26CA4AC84EC640
:1053300006CE2A893284B689353FAA840DE197F7D3
:10534000FB1F83A7278C81CF05476317E40003C4A5
:10535000090005041374F40FA2854A858297F24070
:1053600062444249B2492685D24405618280AE86B4
:105370000147054697050000938525CE6DB79E2110
:105380001CA19E21A1831CB1094582809E211CA1E4
:105390009E21A1831CB1BE213CA1BE21A1833CB1B1
:1053A000114582809E211CA19E21A1831CB1BE219A
:1053B0003CA1BE21A1833CB1DC315CA1FC215CB1EC
:1053C0008A2519053345050882809E211CA19E214E
:1053D000A1831CB1094582809E211CA19E21A1832D
:1053E0001CB1BE213CA1BE21A1833CB111458280EC
:1053F000CA2106053345050882809E211CA19E21F5
:10540000A1831CB1AA2109053345050882809E218C
:105410001CA19E21A1831CB1BE213CA1BE21A18360
:105420003CB1CA2111053345050882809C211CA18D
:10543000054582809E21411122C406C61CA19E21E1
:105440002E841105A183A30EF5FEBE219505230F21
:10545000F5FE83D7D5FFA183A30FF5FE03C6F5FFA5
:1054600097B0FB1FE780C0F24820B24022441105EC
:105470004101828089476399F5001C31182101455B
:10548000A207D98F1EA28280114582809A21011124
:1054900006CE22CC2EC6D94763F4E7022A84EF80D9
:1054A000905AB2469E22636DF50022856244F24016
:1054B00001470946970500009385A5EC05615DBB92
:1054C000F2406244094505618280AA87A9C114217E
:1054D000FD150547B3C505086398E60013D72500F9
:1054E0008D89114589CD8280094711456392E60275
:1054F000494533D7A502B3F5A502114591E91145F8
:1055000001CB850734A21AA25CC2014582801145F5
:105510008280AE860147114697050000938545E7D6
:1055200091BB13F73500AA8701EB8981114591C51D
:105530000EA25CC20145828011458280D821894734
:10554000631BF702011122CC2A84C84506CEAE8621
:1055500001C92EC69D4597B0FB1FE78040CEB246DD
:105560002A8722856244F2401946970500009385F8
:10557000A5E3056101B30945828099E11145828067
:105580001C2105473EA2E37BF7FEFD1593F5F50FC1
:1055900033D7F502B387E702E392F5FE050548C26B
:1055A0001AA201458280DC210947AE866385E700A7
:1055B00041476399E700014721469705000093851D
:1055C000A5E74DB9094582800EA291E1014548C287
:1055D00001458280AE8601472946970500009385E4
:1055E00005DF49B90EA291E1014548C2014582801B
:1055F000AE860147314697050000938525DE9DB9AB
:105600000EA291E1014548C201458280DA21854719
:1056100063FFE702011122CC2A84884106CE2EC600
:1056200015C1854597B0FB1FE78060C12A87228599
:105630006244B246F240394697050000938585DB07
:1056400005610DB9F2406244094505618280094552
:105650008280AA878DC518218D46114563F2E60226
:10566000FD15B3C50508B3C6E5023308D702639933
:105670000501850716A23AA25CC201458280114548
:105680008280DC210947AE866385E7004147639944
:10569000E70001474146970500009385E5D9D9BE4B
:1056A000094582803335B0000A058280011122CC81
:1056B00026CA06CE98258547AA842E844946631FAC
:1056C000F70099363E2049151306200963C8A70044
:1056D000F2406244D244094505618280183485470E
:1056E0006314F70013660604484001C98D4532C6AD
:1056F00097B0FB1FE780A0B43246A2866244F24016
:105700002A872685D24497050000938545CF0561F9
:1057100095B68D4763F7B7021C311821F115A20722
:10572000D98F1EA23C313821B3C50508A207D98FF5
:10573000014799C1130745003EA24EA218C6014574
:10574000828011458280011122CC2A84884506CEB0
:10575000AE8601C92EC6954597B0FB1FE78020AEE7
:10576000B2462A8722856244F240594697050000D6
:10577000938525CA0561FDBC3335B0000A058280DA
:10578000AE860147614697050000938565CADDB482
:105790008547114563F1D7021C320C220945A20747
:1057A000CD8F81456384A60093052600F9161EA3BC
:1057B00036A34CC301458280014781467946814525
:1057C00055BC9E211CA19E21A1831CB1094582804C
:1057D000BC2105471CA18A216397E7000A0505053E
:1057E000334505088280C9473305F502CDBF8A21BC
:1057F0000A05334505088280BE211CA18A21BE21ED
:105800003305F50205053345050882808A2182802B
:105810008A2182808A218280BE211CA18A21BE2108
:105820003305F50205053345050882809E211CA13C
:105830009E21A1831CB1BE213CA1BE21A1833CB10C
:10584000CA2111053345050882809E211CA19E2195
:10585000A1831CB1AA210905334505088280894727
:1058600011456398F6001C3214220145A207D58F1A
:105870001EA382809A21D947AE8663F9E7000147CB
:105880000D4697050000938505F471BC094582809B
:105890001145639DA6001C3214220145A207D58F35
:1058A0001EA33C323422A207D58F3EA38280BC21A6
:1058B0000547FD1793F7F70F6361F7049E2195CF16
:1058C000011122CC2A84C84106CE2EC615C18945B5
:1058D00097B0FB1FE780A0962A8722856244B246D4
:1058E000F2401546970500009385C5EE056125BC7D
:1058F000F2406244094505618280094582809547EE
:1059000063F0D706411122C426C24AC006C61C3223
:105910003A841822A207B284D98F1EA03C323822C2
:1059200093854400A207D98F3EA089475CA0094611
:1059300013055400368997B0FB1FE78060A519470F
:1059400081476304E90093876400691923142401E3
:10595000B2405CC422449244024901454101828024
:10596000114582809E2195CF011122CC2A84C84105
:1059700006CE2EC615C1854597B0FB1FE780208C4B
:105980002A8722856244B246F2401D4697050000F0
:10599000938525E6056141BAF240624409450561F7
:1059A0008280094582809947B2856388F600D14795
:1059B000114541466384F60082800946411106C6BE
:1059C00050A39C31942113055700A207D58F1EA325
:1059D000BC31B4219105A207D58F3EA397B0FB1F20
:1059E000E780009BB2400145410182809E219DCF0E
:1059F000011122CC2A84C84106CE2EC61DC189457C
:105A000097B0FB1FE780A0832A8722856244B246B5
:105A1000F240254697050000938545DE05616FF04D
:105A20009F90F24062440945056182800945828069
:105A3000894711456398F6001C3214220145A207DC
:105A4000D58F1EA38280011122CC2A84C84106CEA4
:105A5000AE8601C92EC6854597A0FB1FE780207E34
:105A6000B2462A8722856244F2402D4697050000FF
:105A7000938505DA05616FF01F8B19BD011122CCEA
:105A80002A84C84106CEAE8601C92EC6854597A098
:105A9000FB1FE780C07AB2462A8722856244F24023
:105AA0003546970500009385E5D605616FF0BF8701
:105AB00093F71600114581EB89476386F6008582CE
:105AC00056A310C301458280011122CC2A84C8410B
:105AD00006CE2EC61DC1854597A0FB1FE780207608
:105AE0002A8722856244B246F2403D46970500006F
:105AF000938585D205616FF01F83F24062440945AA
:105B0000056182809E219DCF011122CC2A84C8414B
:105B100006CE2EC61DC1894597A0FB1FE7802072C7
:105B20002A8722856244B246F24045469705000026
:105B30009385C5CE05616FF00FFFF24062440945C1
:105B40000561828009458280854763F4D70208A7F2
:105B50000CB71C320C220945A207CD8F8145638406
:105B6000A60093052600F9161EA336A34CC30145D3
:105B7000828011458280014781464D4681456FF004
:105B80008FFA8D47114563F5D7021C320C22A2070C
:105B9000CD8F1EA33C322C22A207CD8F814563847A
:105BA000A60093054600F1163EA356A30CC7014577
:105BB0008280011122CC2A84884506CEAE8601C996
:105BC0002EC6954597A0FB1FE7806067B2462A87DF
:105BD00022856244F2405D4697050000938545C5E5
:105BE00005616FF04FF4854711456395F6001C225F
:105BF00001451CA3828001478146654681456FF0BF
:105C00008FF2011122CC2A84C84106CEAE8601C98A
:105C10002EC68D4597A0FB1FE7806062B2462A879B
:105C200022856244F2406D4697050000938525C2A7
:105C300005616FF02FE4011122CC2A84C84106CE01
:105C4000AE8601C92EC68D4597A0FB1FE780205F59
:105C5000B2462A8722856244F240754697050000C5
:105C60009385E5BE05616FF0EFE0011106CE2EC60B
:105C7000EF90703D19C5B245F2402A2105616FD001
:105C8000F078F24049450561828097E7FB1FA381C8
:105C900007FA97E7FB1F238D07F897E7FB1F23A75A
:105CA00007F897E7FB1F23A107F897E7FB1F23AB34
:105CB00007F697E7FB1F23A507F697E7FB1F23A728
:105CC00007F497E7FB1F23A107F497E7FB1F9387D0
:105CD00027173706840390D33707B40037C6070069
:105CE00098C3130606B83747A000D8C3D0D33707E8
:105CF000100041669306070AB70550009308060195
:105D000094C723A4170393860501930816F8D4C7F4
:105D100023A61703B706D007B7087F0013080705A7
:105D200013850601410723A81703B0C39308160083
:105D30009386060513861500D8CBF8C323A8070160
:105D400088CF23AE070023AA170323AC070223AE94
:105D5000070223A40704F0C7B4CB23AA0704ACCFDF
:105D600023AE0705B8D33707A000F8D71307000AFA
:105D7000B8DB1307C01CF8DB37071400B8DF054792
:105D8000F8DFE8D323A40706930710F817E7FB1FF3
:105D90002328F7128280011152C42A8A214522CC7D
:105DA00026CA4AC84EC606CE2E84B2893689BA841F
:105DB00097A0FB1FE780C04D05C9930700FD1CA1FC
:105DC0009947A30045013CA12303250164B1231297
:105DD0003501AA8522856244F240D2444249B24943
:105DE000224A05616FE06F90F2406244D24442491A
:105DF000B249224A0561828097E7FB1F23A8A7E2E8
:105E0000828097E7FB1F23A1A7E2828097E7FB1F11
:105E100023AAA7E0828097E7FB1F23A3A7E0828045
:105E2000011122CC26CA4AC806CE4EC62A89AE84A3
:105E30000144B309890063699400F2406244D2448A
:105E40004249B24905618280EFE04F94B3470508AB
:105E5000A1832380F9009307140093F7F70F8509B6
:105E600063F89700CA97090488A31374F40FD1B795
:105E70003E84D1B7411122C417E4FB1F13048404EC
:105E80006A20C16706C6FD17630EF50017E6FB1F03
:105E90000346462597E5FB1F938585D7EF90A07BAA
:105EA000FD577EA0B24022444101828009C92515D8
:105EB0001375F50F1335850E1345150082800145C6
:105EC000828023900500C9C2797122D426D252CC97
:105ED00056CA5AC806D64AD04ECE5EC62A8B2E8ADD
:105EE000B28A3684814463FF5405B307940083C9A2
:105EF0000700138914003349090863850904B3872F
:105F0000290163C1FA04B307240183CB07005E852E
:105F1000713F0DC99387F9FF2310FA0063906B035B
:105F2000050933052401B250225492540259F24912
:105F3000624AD24A424BB24B45618280CE94B3C48E
:105F4000040855B70145C5B701458280011122CC2F
:105F500026CA4AC84EC606CE97E4FB1F938484F631
:105F60002E89D0C88CC8C8C42A8441469305F00F36
:105F70004A8597A0FB1FE780405C8549631935037C
:105F80008848C145713D41469305F00F228597A091
:105F9000FB1FE780805A0549631525036244C84406
:105FA000F240D2444249B249C145056195BD4146DE
:105FB00081454A8597A0FB1FE7802058E31535FDF2
:105FC000C1B741468145228597A0FB1FE780E05677
:105FD000E30625FDF2406244D2444249B2490561DC
:105FE0008280411122C426C22E84AA841306000294
:105FF000814517E5FB1F1305E5EC06C64AC097A0CF
:10600000FB1FE780603F17E9FB1F1309A9EB97E728
:10601000FB1F238B870CA3019900EFD070418547AC
:1060200019C1814749452300F900B24022449244F6
:106030000249410182809DC91DC985476318F50049
:10604000DC3193E707FCDCB10545828089476316A4
:10605000F500DC3193F7F703FDB78D47E316F5FE46
:10606000DC3193F7F70393E70704F1BF0145828022
:106070008DC10DC1DC311307000C054593F7070CEA
:10608000638AE7001307000409456395E7000D459F
:10609000828001458280411122C4005D06C626C26D
:1060A0001DC8AA84085009C597A0FB1FE780A00B54
:1060B000485009C597A0FB1FE780E00A085409C5AE
:1060C00097A0FB1FE780200A228597A0FB1FE7808F
:1060D000800923AC0402B2402244924441018280F0
:1060E00019ED97E7FB1F83C707DE17E5FB1F1305B5
:1060F000E5DE91CB17E5FB1F130505B2828017E59E
:10610000FB1F1305A5DD828017E5FB1F0345A5DBFB
:10611000828017E5FB1F0325A5DB828017E5FB1FA7
:10612000032545DB828097E7FB1F83A7E7DA8843D7
:10613000828017E7FB1F1307E7D8544B9C42850763
:106140009CC228339307F00F6305F50091656FD06B
:106150007FED8280011122CC06CE2E8432C6EF90D4
:10616000007F9147B245631EF50097E7FB1F83A7A9
:1061700027AB99CF9C4389CF22856244F2400561C9
:10618000828797E7FB1F83A727AA99C3DC43E5B75C
:10619000F2406244054505618280797122D42A84E7
:1061A0004A214ECE06D626D24AD097C0FB1FE780A2
:1061B000A07F97E9FB1F9389A9A729E983C4090058
:1061C0009307F00F639DF40097E5FB1F83C555A669
:1061D0002685613C09E597E7FB1F238B07A44A202E
:1061E000EF90E0769147631CF50097E7FB1F9387DC
:1061F00067CD5620FA236394E6007D57FAA3B25088
:10620000225492540259F249456182805825042152
:106210002A893AC649354A85EF9030324A20EF90B4
:10622000406E83C70900324799C3E38F97F89307FD
:10623000F00F5220E385F4FA74202820A685A13EB1
:1062400079BF79715AC82A8B2E854ECE52CC56CA48
:1062500006D622D426D24AD05EC62E8AB28AB68903
:1062600097C0FB1FE780407475C5045D2A89FDC097
:106270009C501305400391E361459C5489C79307E3
:10628000450133C50708638609009307C50133C577
:106290000708DC5089C79307750133C5070897A025
:1062A000FB1FE780E0FE2A8455C56146814597A023
:1062B000FB1FE780601497EBFB1F83CB6BBB6394E2
:1062C0000B00834B0900930700FD1CA0A947A30006
:1062D00064013CA0230354018C5023124401130594
:1062E000840191C908C47146130A440397A0FB1F97
:1062F000E780000A52858C5491C948C45146130A5C
:10630000450197A0FB1FE780A0085285638C090018
:1063100008C87146CE85130AC50197A0FB1FE78008
:1063200020075285CC5099C548C85D4697A0FB1FF1
:10633000E7800006A2855E85EFD03FBB2254B250B5
:106340009254F249624AD24A424BB24B4A850259B0
:10635000456191B3B250225492540259F249624AB3
:10636000D24A424BB24B4561828001114EC6AA8986
:106370002E8526CA06CE22CC4AC8AE8497C0FB1F03
:10638000E780806221C917E9FB1F034969AE6314E6
:10639000090003490500194597A0FB1FE78040EF5E
:1063A0002A840DC98145194697A0FB1FE780C004C8
:1063B000930700FD1CA0B947A30034013CA046A0F0
:1063C000A2856244F240D244B2494A8542490561FD
:1063D0006FD0BFB1F2406244D2444249B249056134
:1063E0008280797162C42A8C2E8526D24ECE52CC00
:1063F00056CA5AC85EC606D622D44AD0AE84B28BDC
:10640000368BBA8A3E8AC28997C0FB1FE780C05983
:1064100035C52A89414597A0FB1FE78060E72A849C
:1064200031CD4146814597A0FB1FE780E0FC17E591
:10643000FB1F0345E5A319E103450900930700FD90
:106440001CA0BD47A30084013CA023047401A30445
:10645000640123055401A305440146A02326340109
:10646000A2852254B25092540259F249624AD24A49
:10647000424BB24B224C45616FD03FA7B2502254E1
:1064800092540259F249624AD24A424BB24B224CD0
:1064900045618280011126CAAA8439454AC84EC680
:1064A00052C406CE22CC2E8AB289368997A0FB1F11
:1064B000E78000DE15CD9307000D1EA1B1472A84A9
:1064C000231245013CA1CE851905194697A0FB1F53
:1064D000E78000EC23062401A2856244F240424991
:1064E000B249224A13F5F40FD24405616FD0FF9FE1
:1064F000F2406244D2444249B249224A0561828054
:10650000411126C206C622C44AC097E4FB1F9384E9
:10651000649BB8309307F00F6308F7042A89394564
:1065200097A0FB1FE780C0D62A841DCD930700FDEE
:106530001CA1A30025012301050097E5FB1F9385FE
:10654000E5990D05194697A0FB1FE78060E49E249E
:10655000A285A8303EA49C305CA42244B240924460
:10656000024941016FD07F98B240224492440249CF
:1065700041018280011156C2AA8A314526CA4AC801
:106580004EC652C406CE22CC5AC0AE84328AB689D8
:106590003A8997A0FB1FE780A0CF2DCD2A842685BE
:1065A00097C0FB1FE780404009C55825A1476311EC
:1065B000F70417EBFB1F034B1B91930700FD1CA077
:1065C0009D47A30054013CA046A02313440123147B
:1065D000340123152401A2856244F240D244424989
:1065E000B249224A924A5A85024B05616FD0FF8F09
:1065F00017EBFB1F034B5BAFE3910AFC97D7FB1F25
:1066000083A707779C47D5DBCA864E86D285268529
:10661000829765B7F2406244D2444249B249224A65
:10662000924A024B05618280411126C2AA8421450B
:1066300022C406C62E8497A0FB1FE78060C515C53F
:10664000930700FD1CA1C5473CA13C30AA853CB185
:106650005E205EA17C207CA17C307CB12244B240D3
:106660002685924441016FD05F88B2402244924413
:106670004101828041114AC02A89714526C206C65D
:1066800022C4AE8497A0FB1FE78080C03DC593075E
:1066900000FD1CA1F5473CA1BC302A849385C400B1
:1066A0003CB1DE2031051946231CF5FEFE20231DDA
:1066B000F5FE9E24231EF5FEBC24230FF5FEBC34FC
:1066C000A30FF5FE97A0FB1FE78080CCBC28A28516
:1066D0004A853CA8DE285EA8FC287CA8FC387CB84B
:1066E0009C2C1CAC9C3C1CBCBC2C3CAC2244B24042
:1066F0009244024941016FD04FFFB240224492447C
:1067000002494101828001114AC82A89614526CA8D
:106710004EC606CE22CCAE89B28497A0FB1FE7807E
:1067200020B725C1930700FD1CA1BC302A849385A6
:1067300084001CB195473CA1FC3011051946A30FFC
:10674000F5FE97A0FB1FE780A0C4DE2023063401DE
:10675000A2853EA4BE2C4A857EA4DE2C1EA8FE2C5B
:106760003EA883C704025CA883C714025CB8BE308D
:10677000F240D2447EA862444249B24905616FD0DA
:10678000CFF6F2406244D2444249B2490561828068
:10679000411122C406C617D4FB1F1304A4723C2067
:1067A0009DCBAA85194617D5FB1F1305E54697A073
:1067B000FB1FE780E0BD282097D5FB1F9385C545CB
:1067C000EFF07F872244B24017D5FB1F1305C54465
:1067D00041016FD0A046B240224401454101828070
:1067E000411126C206C622C44AC097D4FB1F938417
:1067F000646DB8309307F00F6302F7042A892945C6
:1068000097A0FB1FE780C0A82A840DC9930700FD4D
:106810001CA1A147A30025013CA1BC2097D5FB1FCB
:106820009385853F1105A30FF5FE194697A0FB1F21
:10683000E78000B6A830A285EFD02FEBB8208D47B7
:10684000631FF70097D7FB1F83A7C73D89CB9C47E2
:1068500099C72244B2409244024941018287B24022
:1068600022449244024941018280797122D406D6A1
:1068700026D24AD04ECE52CC56CA09444DCD2A8992
:106880000A212E8A514497C0FB1FE780E011AA8499
:106890005DC197EAFB1F938AEA8483C74A000547D4
:1068A0004944FD1793F7F70F6377F7085825A14779
:1068B0006314F70063110A089C5C4544ADEF9165D1
:1068C000938545711305C0029790FB1FE780807C7C
:1068D00088DCAA894D4425C11306C002814597A0D2
:1068E000FB1FE78060B18357090093864900368516
:1068F0002391F90071469305490036C697A0FB1F06
:10690000E78000A989472380F900DC24B2460356BA
:10691000090083C50A00E11713B51700EF90507AFC
:106920002A8463060A00D2852685EF90207001C470
:106930002685EFF04FF6B250228522549254025928
:10694000F249624AD24A4561828097D7FB1F83C7CA
:10695000A779FD1793F7F70F05476377F70801113C
:106960004AC806CE22CC26CA4EC652C432898947AE
:106970002DC22A8AAE89368497C0FB1FE780C002E9
:10698000AA84D14739C5485509C59790FB1FE780B0
:10699000807DF1454A8597A0FB1FE78000ADC8D4F4
:1069A000AA85CD471DC5D824A147631DF70209C894
:1069B000382D1229930625015285EF90806D2A8487
:1069C000D820936747006384090093676700DCA0C1
:1069D000A287F2406244D2444249B249224A3E85EB
:1069E000056182800144E9BFC9473E8582809307E3
:1069F000000463EAA70097D7FB1F938767443325FA
:106A0000F5200A21828041657D158280011122CC0A
:106A10002A842E8526CA06CEAE8497C0FB1FE78047
:106A2000A0F80DCDB7470F009387F723094563E220
:106A3000870281450A85414697A0FB1FE780C09BDE
:106A4000A68560800A8541804081A3010100EF9006
:106A5000F047F2406244D244056182804945D5BF87
:106A600097D7FB1F2381A76882806F90D05F7971D1
:106A700052CC2A8A328526D24AD04ECE56CA5AC81D
:106A80005EC662C406D622D42E8CB28A368BBA8BEE
:106A90003E89C289C68497C0FB1FE780E0F005C924
:106AA0002A84631A0A1893774B000343450085CF65
:106AB0001363230163940B1663100914639F090881
:106AC00085E81C5C1373B3FF23026400C5EBB2506E
:106AD000225492540259F249624AD24A424BB24B72
:106AE000224C456182801373D3FF13630301D9B72E
:106AF00013634300230264009C484146A6851CD4CE
:106B00001305840197A0FB1FE780808863130C1294
:106B1000638C0B0A485409C59790FB1FE780A0645B
:106B2000F1455E8597A0FB1FE780209448D4005C68
:106B300059DC1C5091EB91659385357171459790A7
:106B4000FB1FE780205508D008500DC17146DE8537
:106B500097A0FB1FE780C08311A8136343002302A3
:106B60006400D9F8005C630C0C0235D0639A09020A
:106B7000A5E029A0005C21DC639409022254B250F4
:106B80009254F249B24B224CCA865A860259424B61
:106B9000D6855285D24A624A45616FF08FEA05D8A0
:106BA0005C5091EB9165938525715D459790FB1F36
:106BB000E780404E48D0485045DD5D46CE859790F1
:106BC000FB1FE780E07C6DB7005C11D0E39A09FC05
:106BD0001C5491EB91659385157151459790FB1F5E
:106BE000E780404B08D4085451D95146A685979068
:106BF000FB1FE780E07959B7136343002302640069
:106C0000E39C04EEE3080CF6485405EDF1454A8593
:106C100097A0FB1FE780608548D431A81363430029
:106C200023026400E39A04ECE3060CEEE31E09FC85
:106C3000FDBDE31B09FC005CE30B04E8E39B0BEEEA
:106C400035B79790FB1FE7800052C9B7011126CADC
:106C500052C406CE22CC4AC84EC62A8AAE8497C0F9
:106C6000FB1FE78060D435C12A8939459790FB1F07
:106C7000E78000622A8431C997D9FB1F83C9491F65
:106C800063940900834909009307000D1EA0AD47D6
:106C90003CA0930569001305340019469790FB1F2B
:106CA000E780006F93F714005CA493D4144844B4B5
:106CB00023154401A2856244F240D2444249224A4B
:106CC0004E85B24905616FD04FA2F2406244D24472
:106CD0004249B249224A0561828001114EC652C41E
:106CE00056C206CE22CC26CA4AC8AA8A2E8AB289A1
:106CF00097C0FB1FE78040CB35CDAA841305C002A7
:106D00009790FB1FE780C0582A842DC517D9FB1F19
:106D1000034909166314090003C904009307000D11
:106D20001EA0E9473CA09385640013053400194672
:106D30009790FB1FE780C065D2852315540113058A
:106D4000C40041469790FB1FE7808064CE85130501
:106D5000C40141469790FB1FE7808063A28562448F
:106D6000F240D244B249224A924A4A8542490561D8
:106D70006FD0AF97F2406244D2444249B249224AAE
:106D8000924A0561828017D5FB1F0325E5E711CDE7
:106D9000411106C69790FB1FE780E03CB24097D7B1
:106DA000FB1F23A307E6410182808280411122C498
:106DB00006C626C24AC02E8497C0FB1FE780C0BE0D
:106DC00029CD00D517D9FB1F0349890AAA8463146A
:106DD00009000349050041459790FB1FE780404BA0
:106DE0002A8405CD9307000D1EA1A5473CA1DC30E8
:106DF000938564001105A30FF5FE19469790FB1FBC
:106E0000E78000599C54A285B2405CC4224492445D
:106E10004A85024941016FD04F8DB24022449244CD
:106E20000249410182805D71A2C4A6C286C6AA84BD
:106E30002E8497C0FB1FE78020B70DC9542511474A
:106E4000AA874945639FE6009C5F91C3E02B97B6F4
:106E500000009386A6910A86894526854080EF909A
:106E6000E013B64026449644616182805145D5BF07
:106E700097D7FB1F83C74727FD1793F7F70F0547E2
:106E8000637AF704411126C206C622C44AC0B284FE
:106E9000894715CA2E8997C0FB1FE780E0B02A8476
:106EA000D14715C1630609005C2193E727005CA167
:106EB0004146A685130584019790FB1FE780404D4E
:106EC0009C481CD48147B2402244924402493E85EA
:106ED00041018280C9473E858280011122CC26CAA9
:106EE00006CE2A84AE8497C0FB1FE780E0AB19C9A9
:106EF0006C0022854486EF900010F2406244D24438
:106F0000056182805145D5BF6F807019C1671387B5
:106F1000E7FF6393E50297D7FB1F83A7E7D091EBC9
:106F2000494582804945B240224492440249410188
:106F300082809C43F5D78287411122C426C24AC071
:106F400006C6FD172A892E84B284639AF50297D764
:106F5000FB1F83A767CD89C79C4399C3829711C53F
:106F6000A6854A85EFE07FD05DFD97D7FB1F238183
:106F700027CD97D7FB1FA38D97CA01456DB72E85E7
:106F800097C0FB1FE78040A251DD1C210D45E39C0B
:106F900027F922852244B2400249A6859244410144
:106FA0006FC0D0469307000463E1A7064111C16793
:106FB00022C426C206C6FD172A84AE840945638012
:106FC000F502C5476312F4022E85EFC0D04B97D768
:106FD000FB1F9387E7E63324F420014506A0B24067
:106FE00022449244410182809307A0036316F40077
:106FF0002E85EFC07042E1BF9307B003E319F4FCA4
:1070000013F5F50FEFC09041D9B709458280011102
:1070100006CE2AC6EFE07FC7EF20404EEF10C07CBF
:10702000EF501235324597D7FB1F9387A7E9130717
:1070300000F0BAA3238207007D5797D7FB1F9387E1
:10704000670AB8A388A3F240954505616F70E028F0
:10705000757126C306C722C54AC1CEDED2DCD6DA98
:10706000DAD8DED6E2D4E6D2EAD0EECEAE8493977A
:10707000556063D1075817DAFB1F130AAA060345A8
:107080000A00130B200A930BF00F9790FB1FE78069
:107090002026C167FD172A84130C1009954C394D21
:1070A00097DDFB1F938D0DE23ECC15E01395F46840
:1070B000BA402A449A440A49F659665AD65A465B57
:1070C000B65B265C965C065DF64D496182801C20AD
:1070D000639A670103C93D00E2452A202286EFF04A
:1070E0006F87E1A003492A00639A87091C306390E7
:1070F00097032285EFF06F8A2285EFC0FFD9034501
:107100000A009790FB1FE780A01E2A8479BF639B2B
:10711000A7194A208567A507631AF5040C4497D977
:10712000FB1F938929DA882115E51946850517D5AE
:10713000FB1F1305A5DA9790FB1FE780602503C7A7
:1071400009008547631CF70289472380F900EFC0D7
:10715000B02E5DB703C7090085476311F70297D7C3
:10716000FB1F238107D6EFF0AFB979B70967930703
:10717000C70063EFA7040507636BA702E30E79F767
:10718000A2854A85EFC07FD69DBF37070018130739
:10719000F770B357F748E5CB97D7FB1F83A787A8AE
:1071A000A1DF9C43B1DB2285829739F5C1BFF97716
:1071B000F917AA972947B3C707086366F70C17673B
:1071C00002001307E75FB3C7E7209C43BA978287A3
:1071D000F9779387A7FCAA97F146B3C70708E3F6A8
:1071E000F6FA3907E31CE5F897D7FB1F83A7C7A377
:1071F000E38407F0DC43E38107F00965A2853905E4
:10720000A5A883298400E38B09F603C7090097D753
:10721000FB1F938727CB19EB03C7290083C61900EF
:107220002207558F9AA703C7390098B394230947BB
:10723000E396E6F403C7090001CB97D7FB1F23832E
:1072400007C803C5090005B78C338A270D4798A3E3
:10725000EF70400BFDB71C448823EFF06FD869BD79
:1072600097D7FB1F83A7879CE38807E89C43E385A8
:1072700007E80965A2852D05829705BF1C449C235C
:10728000E39E07EE95BD896793871704E318F5EE33
:1072900097D7FB1F83A78799E38007E69C43A285C6
:1072A000E1FF99BD3D476394E7064A20896713874C
:1072B000D7006306E50013879701631AE50097D7A7
:1072C000FB1F83A76796E38907E2DC43C9BFCD07AD
:1072D000E316F5EAC16717D7FB1F035707BFFD1772
:1072E000631FF70097D7FB1F83A70794E38607E088
:1072F000DC43E38307E00965A2854D05B5BF97D759
:10730000FB1F83A7E791E38907DE9C43DDB71307E3
:10731000E003E395E7E63C2005476398E7127C200D
:1073200097DAFB1F938A4A8E6390071083A70A009F
:107330006387070E83C907002149683093078400DB
:10734000BE853ECEEFE0DFD268B013064002814535
:1073500068109790FB1FE780200A3C301946930580
:107360008400A307F1027C304818A309F10297902A
:10737000FB1FE780E0015E207010CA852318F10230
:107380007E244E852313F1041E282314F1043E2885
:107390002315F1045C282306F104FD57A306F1042C
:1073A0002317F104EFF02FB63C309DE3DD478358FF
:1073B00004010358E40074304E203EC23E281307F7
:1073C00084003EC0CA8705464E85EF80806F28B096
:1073D00083A70A0081C71145EFF0FF9A97D9FB1FD9
:1073E0009389098503C50900E30805D097D5FB1FDC
:1073F00083C51584EFE07F87E30005D03430930721
:1074000010036389F600522083C509004A87368538
:10741000EFE07F9897D7FB1F238C0780F1B997D9AE
:10742000FB1F83C959AA09BF97C7FB1F83A7877F83
:1074300097D9FB1F83C939A999C3DC4399E3114943
:10744000EDBD814501458297DDBFF91793F7F70F31
:1074500013077002E364F7D21767020013070739B6
:10746000B3C7E7209C43BA9782877C2097CAFB1F4B
:10747000938A8A79A9EB83A70A00A9C383C9070065
:107480002149683093772500A5C305891307440176
:1074900068B02286CA854E853ACEEFF0CFA63C3042
:1074A00072479DF7DD478358C4010358A401743027
:1074B0004E203EC27E2C3EC0CA8731B797D9FB1FF3
:1074C00083C979A075BF97C7FB1F83A7A77597D9F5
:1074D000FB1F83C9599F99C3DC4399E3114955B7F1
:1074E000814501458297DDBF13078400BA853ACEF6
:1074F000EFE01FB8724769BF97C7FB1F83A70773E9
:10750000E38C07BEDC43E38907BE22858297EDB694
:1075100097C7FB1F83A78771E38007BE9C47E5B72A
:1075200022868D454A2065BE9305A10213051031C0
:10753000EF50E26B6C1013052031EF50426B72205C
:107540008357C1024A2063E7C70016240357A102EC
:1075500063F7E60093050002EFC0E07171BE63734C
:10756000E6007AA063F3D7001EA45A24362412241E
:107570006E2001488147EFC0C06FBDBE2286B14575
:1075800055B797C7FB1F83A7676AE38707B6DC4732
:107590009DBF2285EF00607B85B697C7FB1F83A741
:1075A000E768E38B07B49C4BB9BF2285EF00F0037B
:1075B000A1B60145EF00301381B697C7FB1F83A723
:1075C0006766E38D07BADC43E38A07BA8145054560
:1075D00082976DB697C7FB1F83A7C764E38007BA7E
:1075E000DC43E38D07B8A2850945DDB72286930504
:1075F00060020DBF93F7150089CF97C7FB1F83A7C4
:10760000E76289C7DC4399C30145829713C514001B
:1076100045B493F7250091CF97C7FB1F83A78760D9
:1076200091C7DC4381C781450545829713C5240076
:1076300041B413F54500E30D05A697C7FB1F83A7CB
:10764000E75C17D4FB1F1304E48789CF85475CA050
:1076500097C7FB1F83A7075D91C7DC4381C781459F
:107660000545829748446C10EF80D0726810EFF0A7
:107670002F9297C7FB1F83D7C77E81CF1306006465
:107680003386C702914517D5FB1F0345A5A5EFC05B
:10769000BFAF13C5440029BC011122CC2A84554533
:1076A00006CE26CAEFF0AFB4AA8413054002EFF06D
:1076B0000FB42AC613055002EFF06FB3AA862285D5
:1076C00062443246F240B3359000D24405616FC047
:1076D0006062397122DC06DE0D472E84631AE500F4
:1076E000BA259625F2212830CE21EFE0BFE899A8EF
:1076F00009679306D700AA87631BD504BC21B9C3C9
:1077000017C4FB1F130444500C408DCDDC87BC31E3
:10771000194691054808A309F1009790FB1FE780DF
:1077200020C7930700F03ED61C4023180100231306
:10773000010202D4882370008145EFE0DFFC05459B
:10774000EFF06FE40545F2506254216182809306A8
:10775000E700E309D5FE930637016319D500A82198
:1077600075D1014781460146814541B76507E30B65
:10777000E5FC31476319E50017C5FB1F0345B574E8
:10778000EFE09FEAC1B7130760026319E50017C570
:10779000FB1F03455573EFE0FFED6DB741677D17A4
:1077A0000145E392E7FAD831C947E31DF7F8F6251A
:1077B000D2250A24AE25EFC0805B854711C55D4503
:1077C000EFF0EFA2B337A0004C202A2030007C84D9
:1077D000EF70D0693C84BDF79305A100130510310B
:1077E000EF50E2406C0013052031EF5042403C85E1
:1077F0001A246373F7001EA43C863A2463F3E7005F
:107800003EA41E243A246373F7003EA42A20EF40CE
:1078100061107A24562432240E242A2001488147FC
:10782000EFC0004305B741114AC006C622C426C2B4
:1078300017D9FB1F1309098B034779009307F00F32
:107840006302F706AA8439CD682551059790FB1F7E
:10785000E78000A42A8439C59307000D1EA1D947EB
:107860003CA1DE205EA1FC207CA1FC307CB19C24EC
:107870001CA5DC345CB5F02470A515C28C485105FC
:1078800008C89790FB1FE780A0B0A285224403455B
:107890007900B2409244024941016FC00FE52328AC
:1078A0000500E5B7B240224492440249410182807A
:1078B000C1679386E7FF2A87639DD50097C7FB1FA3
:1078C00083A787348DC39C230D45639FE7006FC05A
:1078D0006037FD1749456399F50097C7FB1F83A7DC
:1078E000A732F5F7828049458280397122DC06DEB5
:1078F00026DA4AD84ED652D456D25AD018218547C5
:107900002A84630BF7001025930695009305E10187
:107910000545EFE00FDB0DED8147014514201147D0
:10792000638FE60217C7FB1F0327473118338D46C5
:107930006307D7028DC705C711ED0145F2506254A8
:10794000D2544259B259225A925A025B2161828022
:107950001C21E9B785466311D7048D8BF9DF083008
:10796000930524002EC6EFE0AFF008B017C9FB1F47
:107970001309092D83270900AA8981449DC3B245B3
:1079800017CAFB1F130A0A2C130BF00F83470A00B8
:1079900063EBF400814481A08946E310D7FA858B1C
:1079A00075BF054561BF83270900939A4400D697A8
:1079B0009823630C670598336319370519461385B7
:1079C00027002EC69790FB1FE78000AFB24515CD6C
:1079D00083240900D69418209147C1E8E30FF7F4F7
:1079E00083240900B9D883460A0081471306F00FA3
:1079F000E385F6F403C8040013850401630BC80093
:107A0000850793F7F70FAA84E5B7850493F4F40F7D
:107A1000B5BF98A01C301385240019469CB09790E0
:107A2000FB1FE780E096082491659385F5710505B5
:107A30009780FB1FE780006605C1182091476314FB
:107A4000F702C8C41024930594000505A30FC5FED2
:107A50009790FB1FE780C0931C24A1F708207D1599
:107A600013351500E1BD88C4F1BF6311F706C844A2
:107A70001C2405C11021630DF604182091476317DB
:107A8000F706C84419C59780FB1FE780C06D23A681
:107A90000400082491659385E57105059780FB1F17
:107AA000E780405F05C118209147631AF704C8C4F6
:107AB0001024930594000505A30FC5FE9790FB1FA6
:107AC000E780008D08243335A0008DBD88444DB774
:107AD0009305940005059790FB1FE780E09D85477F
:107AE000E31DF5F85545EFE09FF09DBF884455D163
:107AF0009780FB1FE780206723A4040059BF88C438
:107B000045BF397122DC4AD84ED652D406DE26DA79
:107B100056D25AD05ECE2A84130925000831CA8570
:107B200017CAFB1F130A8A11EFE08FD408B083270E
:107B30000A000D47AA899C336391E70217CAFB1F0D
:107B4000130A0A1083270A00814497CAFB1F938AED
:107B50006A0F6393071005452DA0EDD3144C7038C0
:107B60009305E1000545EFE0CFB5AA841DC90327C1
:107B70000A0085461C2118336310D7028D8BDDFF68
:107B80000145F2506254D2544259B259225A925A83
:107B9000025BF24B216182808946858BE310D7FA24
:107BA000F9BF1C2011476385E7002D47E39AE7FCE6
:107BB00097CAFB1F938ACA0883A70A00014A97CB7A
:107BC000FB1F938B2B08CDDF03C70B00B3470A08BD
:107BD00063E4E700A5F46DB703A50A00131B4A0090
:107BE0001C205A9518216310F7021C31639D370140
:107BF0001946CA8509059790FB1FE780E08B01C5F0
:107C000083A40A00DA94050AC1B783A9840059A89D
:107C10000C4C138519009790FB1FE780E08985477E
:107C20006317F5085545EFE09FDC4DC191BF1C205F
:107C300011476385E7002D47639DE700C8C470388E
:107C40000505A30FC5FE0C4C9780FB1FE780407411
:107C5000B5A888C4EDB7850403C70A00B3C70408F4
:107C600063F8E70603250A00139B44001C205A957D
:107C70001821E312F7FE1C31E39F37FD1946CA8530
:107C800009059790FB1FE780208371D583240A00A4
:107C90001C201147DA946385E7002D47E397E7F648
:107CA00083A9C4007C3803C60900E303F6F64E85B9
:107CB0009780FB1FE780204B683891659385E571BD
:107CC00005059780FB1FE780E03C35F1E39504E86C
:107CD00003C70A0083240A0081479306F00FE3FCE0
:107CE000E7E68C20138604016387D5008507B284FC
:107CF000B3C70708EDB7E38004E61C20CA851385E7
:107D000024009CA01C3019469CB09780FB1FE78084
:107D10002068683891659385F57105059780FB1F8C
:107D2000E7804037E30905E218209147631DF7001B
:107D3000C8C470380505A30FC5FE0C4C9780FB1F07
:107D4000E780006509BD88C4EDB701114AC806CEB9
:107D500022CC26CA17C9FB1F1309C938034779006B
:107D60009307F00F630DF706AA8435C96145978024
:107D7000FB1FE780E0512A843DC19307000D1EA13F
:107D8000D5473CA1BC30938584002EC63CB1DE2093
:107D90005EA1FC207CA1E830EFE08FADB24568B079
:107DA0001946130584009780FB1FE780605EFC2462
:107DB000A285034579007CA49E281EA8BC283CA867
:107DC000BC383CB8DC285CA8DC385CB8FC287CA853
:107DD0006244F240D244424905616FC00F91F240C3
:107DE0006244D244424905618280411126C206C6DE
:107DF00022C497C4FB1F9384E42EF8309307F00F3E
:107E00006309F7022A8415C519459780FB1FE7808F
:107E10002048AA8519CD9307000D1EA1DD473CA17E
:107E20005E202244B2405EA1E830924441016FC01E
:107E3000CF8BB2402244924441018280011126CA74
:107E400097C4FB1F9384C4DF9C4006CE22CC4AC853
:107E50004EC652C49DC32A89AE89131A45000144F7
:107E6000884063144403638C09049780FB1FE780F8
:107E7000802F97C7FB1F23A507DCF2406244D24442
:107E80004249B249224A05618280B307850088478A
:107E900009C99780FB1FE780002D9C40A29723A46F
:107EA00007009C40A297C84709C99780FB1FE7803D
:107EB000802B9C40A29723A60700410455B755DDAF
:107EC000228681459780FB1FE780005394408147BD
:107ED0007D5613F7F70FE37227FB1397470036978A
:107EE00010A38507FDB7797152CC17CAFB1F130A7F
:107EF000EAD483270A0006D622D426D24AD04ECE10
:107F000056CA5AC85EC6E9C72A8997CAFB1F938A10
:107F10006AD3814419ED97C6FB1F83A666D291CA26
:107F200003C60A0081479305F00F13F7F70F636943
:107F3000C7021395340021059780FB1FE780403569
:107F40002A8415E921459780FB1FE78060342A8445
:107F500035C1C5679387073D1CC123220400A9A032
:107F600013974700369718236305B700850493F4E9
:107F7000F40F85075DBF930700FD1CA18547A30093
:107F800025013CA124B1F1D8130985002322250144
:107F9000814917CBFB1F130BABCA930BF00F83C7A1
:107FA0000A0063F3F900A1E083270A00A285882371
:107FB000EFB0BFF303C50A008145493503250A0028
:107FC0009780FB1FE780201A97C7FB1F23A807C6CF
:107FD000B250225492540259F249624AD24A424B58
:107FE000B24B4561828083250B0093974900BE9573
:107FF0009C21638377032300F9009C31130529003A
:10800000FD14A300F9001946890593F4F40F978035
:10801000FB1FE780E0372109850993F9F90F41B784
:1080200097C7FB1F83A787C1A9C7411122C406C6F2
:108030002A8415E10945EFE09F9B2A8601C9854501
:1080400017C5FB1F0345050AEFC00F940545EFF068
:10805000AFE42A8411C9854517C5FB1F0345850870
:10806000EFC0EFBB22854135B240224405454101B6
:1080700082800145828089679386B7006315D500A9
:108080009C45882371BF9386C7006317D5009C4524
:108090008546882319C9FDB793861704E302D5FEE8
:1080A000938727048146E304F5FE3685828001111B
:1080B00006CE22CC26CA4AC84EC652C456C261C198
:1080C0003C312A898DC3444199CC5945EFE03F9218
:1080D000814997CAFB1F938A6AB6131A4560834782
:1080E000390063EBF900F2406244D2444249B2499C
:1080F000224A924A056182808387840263C84707C7
:1081000083A70A00A5C72685EFF02FFE25C1882486
:1081100051059780FB1FE780A0172A8421C9930788
:10812000000D1EA1B5473CA19C2019469385240053
:108130003CB18387840215057CA19C30A30FF5FE1A
:108140009780FB1FE780C024902450A415C6130518
:10815000440108C8938594009780FB1FE780402363
:1081600083A70A00A2858823EFB03FD885099384AE
:10817000940293F9F90FA5B723280400D5B797C740
:10818000FB1F83A7A7ABA5D3B93B6244F240D244FF
:108190004249B249224A924A014505616FF0CFCF68
:1081A000797106D622D426D24AD04ECE52CC56CAA7
:1081B0005AC85EC655CD3C312A898DC744419DC001
:1081C0005945EFE0DF828904814997CAFB1F938AF2
:1081D000EAA6130B00FDC14B131A45608347390013
:1081E00063EDF900B250225492540259F249624AA6
:1081F000D24A424BB24B456182808387D40063C42C
:10820000470783A70A00A5C351459780FB1FE78056
:1082100020082A8429C923006501A3000500230141
:10822000750183C7E4FF1946A6853CB18387D40056
:1082300015055CB583C7F4FFA30FF5FE9780FB1F00
:10824000E7800015FC20938574001305C4003CB43E
:1082500019469780FB1FE780A01383A70A00A28519
:108260008823EFB09FC8850993F9F90FC104BDB702
:1082700097C7FB1F83A7879CB5D7B5312254B2504F
:1082800092540259F249624AD24A424BB24B0145DA
:1082900045616FF06FC0797106D622D426D24AD0DC
:1082A0004ECE52CC56CA5AC85EC662C466C2630C71
:1082B00005223C312A8985CB404115C45945EFE060
:1082C0000FF30904814917CAFB1F130A2A97914B20
:1082D000354C175B0200130B6B5B931A45608347A9
:1082E000390063EFF900B250225492540259F24916
:1082F000624AD24A424BB24B224C924C4561828038
:108300008307A40063CA571583270A0063860714EE
:10831000834CE4FF93F70C01CDC793870CFF93F7D1
:10832000F70F6369FC00B3C767219C43DA97828724
:10833000230F04FE1305E4FFEFF0AFFC630E0510FE
:108340008347E4FF63EFFB1005476398E70A514555
:108350009780FB1FE780C0F3AA84630F050E930785
:1083600000FD1CA1C147A30005003CA18347E4FF19
:108370001946A2853CB18307A40015055CB5834767
:10838000F4FFA30FF5FE9780FB1FE78060007C24BD
:1083900019469305F400BCB41385C4009780FB1FF5
:1083A000E78000FF65A08547230FF4FEA30A0400C1
:1083B00051B78947230FF4FEB5BF8D47E5BF9147FD
:1083C000D5BF93F78C0099C3AD47EDB713F71C00E9
:1083D00093F74C0011C799C39547F9B7A147D9BF87
:1083E00013F72C0011C799C3A5477DBF9947D9B78B
:1083F00099C3A947C1B79D4775BF483851059780B4
:10840000FB1FE780E0E8AA8421C99307000D1EA1A5
:10841000B5473CA18347E4FF1946A2853CB18307D9
:10842000A40015057CA18347F4FFA30FF5FE9780F8
:10843000FB1FE780E0F55038D0A419C6138544012E
:1084400088C88325640199BF23A8040083270A00F4
:10845000A6858823EFB07FA9850993F9F90F7104E8
:10846000BDBD4838130505029780FB1FE78040E239
:10847000AA847DD19307000D1EA1C9473CA1834763
:10848000E4FF93FC0C061946B3E797013CB1834720
:10849000F4FFA2851505A30FF5FE9780FB1FE7806B
:1084A00020EF7C2019469305F400BCB47C30138582
:1084B0003401DCA41C24DCB41C34FCA48307A40019
:1084C000FCB45E249EA87C24BCA89780FB1FE78098
:1084D00020EC503890BC09C613850402C8CC95B76F
:1084E00023AE0400A5B797B7FB1F83A72775E38CBE
:1084F00007DEEFF05F9F2254B25092540259F249C6
:10850000624AD24A424BB24B224C924C01454561E1
:108510006FF08F9817B7FB1F0327477205CB1823FF
:10852000AA870D456315F7024111854517C5FB1F45
:10853000034545BB06C6EFB09FEE13050003EFF001
:108540009F9AB240014541016FF00F9549458280E5
:1085500079714AD017B9FB1F1309496E83270900A7
:1085600006D622D426D2CDEB17C4FB1F130484B742
:108570005820C947298B51CB9165AA849385D57121
:1085800011459780FB1FE780E0B02320A900CD476D
:108590002DCD78309307F00F6314F7009C207CB04A
:1085A0001146A6859780FB1FE78080DE9305310189
:1085B0001305F041EF20723497C7FB1F9387879014
:1085C000A023034731013334800011C3090413058C
:1085D0001002EFE0CFC11376F50F0589E14715C50D
:1085E000154532C6EFE0AFC0BC20E8841945230A28
:1085F000F100EFE0CFBF3246AC30E8867C083808A7
:1086000054082285EFB0C06EAA87B250225492540B
:1086100002593E8545618280C547C5BF1971A2DCFC
:10862000A6DA86DECAD897C4FB1F9384A4ABDC20ED
:108630004944A18BB9CF97B7FB1F83A7276041445B
:10864000A9EB2A89EFE05F8C9C2455446373F50401
:1086500097B4FB1F9384445B9C4045449DEB91651C
:108660009385C57129459780FB1FE780A0A288C02C
:108670004D4405C12946CA859780FB1FE78040D13C
:1086800013056002EFE0AFB61374F50F058909E931
:108690006144F65022856654D65446590961828059
:1086A00013060003814588009780FB1FE780C0D434
:1086B0004145EFE0CFB32316A1043D45EFE02FB3D2
:1086C0002319A1043545EFE08FB2231CA1043945DD
:1086D000EFE0EFB1231FA1042145EFE04FB12312DA
:1086E000A1061D45EFE0AFB09C402315A106136421
:1086F00024009C33F1C72D45EFE06FAF2310A10498
:108700003145EFE0CFAE2313A1041305C002EFE023
:108710000FAE2317A1041305B002EFE04FAD231AEB
:10872000A10413059002EFE08FAC231DA1041305F3
:10873000A002EFE0CFAB2310A10613058002EFE00B
:108740000FAB2313A10613057002EFE04FAA9C4064
:108750002316A106A83393854700EFD0DF8D2AD6D4
:108760009305F1031305F041EF20321997B7FB1F72
:1087700093874775AC230347F1033256B335B000F6
:1087800011C389059440FC002287A8223EC89307A4
:1087900021053EC6BC083EC49307E1053EC2DC107D
:1087A0003EC09308A106130861049C009106EFB037
:1087B000A0542A84E30F05EC0D45EFE0CFDCD1BDDA
:1087C0002545EFE0CFA22310A10429451DBF97C77F
:1087D000FB1F83C76791A18B17B5FB1F1305854549
:1087E00091E301456FD0EFE197B7FB1F238C07445E
:1087F000FD5717C7FB1FA30AF78E97B7FB1F23A1CF
:10880000074497B7FB1F23AB074297B7FB1F93871C
:10881000676D170700001307478698C31707000006
:1088200013072789D8C3170700001307A79798C70E
:1088300017070000130767A6D8C717F7FFFF13072E
:10884000C7FE98CB97B7FB1F9387C73E17F7FFFF6D
:108850001307470698C317F7FFFF1307C7E7D8C3E7
:108860008280411122C426C206C617B4FB1F13041E
:10887000643DAA8408208545EFF04FDC97C7FB1FB5
:1088800083C78786A98BBDC717B5FB1F13058565F1
:1088900004A0EFD06FD697B4FB1F9384643A9C403A
:1088A00099C74D45B240224492444101828008203C
:1088B00019E10145C5BF91659385B57112059770A2
:1088C000FB1FE780207D88C069DD102081451206EE
:1088D0009780FB1FE78040B2142090408147FD55F0
:1088E00013F7F70FE377D7FC1397470032970CA3E2
:1088F0008507FDB7014597B7FB1F23850734EFD0E8
:10890000AFCF45BF17B5FB1F0325453011CD411132
:1089100006C69780FB1FE7800085B24097B7FB1F14
:1089200023A6072E41018280828001111305700366
:1089300006CEEFE0CF8B2AC613058003EFE02F8B26
:108940002AC413059003EFE08F8A2246B245F24015
:10895000AA86054505616FB0E0385D711305D00347
:1089600086C6A2C4A6C2CAC0EFE06F882A841305D7
:10897000C003EFE0CF87AA841305E003EFE02F8761
:108980002A891305F003EFE08F868A871377F50FA6
:108990009376F90F13F6F40F9375F40F0545EFB0C6
:1089A000A036B64026449644064961618280011192
:1089B00022CC06CE26CA0D472E846317E504B831B3
:1089C000E947CA2197B4FB1F9384C44F6315F7008E
:1089D000FE206387A70497A0FB1FE780E0FC7220BE
:1089E00011C172A53A2416244E202830EFD09FB82A
:1089F0005A20FE206314F700FD57FEA00545F24003
:108A00006244D2440561828009674D07AA87631CCE
:108A1000E500BC2131476385E7004547E390E7FE69
:108A2000EFD04FC5E1BF31476319E50017B5FB1F14
:108A30000345956BEFD05FBFD1B713076002631991
:108A4000E50017B5FB1F0345356AEFD0BFC27DB700
:108A500041677D170145E394E7FAD831C947E31030
:108A6000F7FACC212A20300023140100EF60103BDC
:108A700071B71971A2DC17B4FB1F130424191C4031
:108A800086DEA6DACAD8CED6D2D4D6D2DAD005457A
:108A9000638A070C9305F1051305F041EF20E265A9
:108AA0009305F1051305F041EF20226597B7FB1FF1
:108AB00093874741BC230347F105B337F00011C347
:108AC00089071840BEC6283393054700EFD0AFD6BC
:108AD0001840AAC40D452C23AEC2EFD05FF1AAC046
:108AE0001145EFD0DFF0832A04002ADE654503C775
:108AF000AA0003CBBA003ADCEFD07FEF2A846945A5
:108B0000EFD0FFEEAA847145EFD07FEE2A896D4544
:108B1000EFD0FFEDAA897545EFD07FED2A8A794520
:108B2000EFD0FFEC2648B6476257F2560646964508
:108B30001375F50F137AFA0F93F9F90F1379F90FEB
:108B400093F4F40F2ACC1314446002D002CE52CA1C
:108B50004EC84AC626C422C25AC093884A00054558
:108B6000EFB02013F6506654D6544659B659265ADB
:108B7000965A065B09618280411122C44AC006C62A
:108B800026C217B9FB1F1309790D83470900130784
:108B9000E00F2E846382E7041307F00F6385E7027A
:108BA00011459770FB1FE780A06EAA8509CD93073A
:108BB00000FD1CA189473CA1854700B13CB103459C
:108BC0000900EFB08FB2F9572300F900B2402244F8
:108BD0009244024941018280AA8411459770FB1F8B
:108BE000E780006BAA857DD1930700FD1CA1894712
:108BF00000B13CA124B12244B2409244024917B5CD
:108C0000FB1F0345A50541016FB02FAE79714AD016
:108C100017B9FB1F130989FF8327090022D406D641
:108C200026D24ECE52CC4544C5EB97B4FB1F93845D
:108C3000644BDC204944958BC5C32E8A916597B758
:108C4000FB1F238DA700AA89938575713145977005
:108C5000FB1FE78020442320A9004D4435CD23008D
:108C60003501A30005002946D28509059770FB1F31
:108C7000E78000720327090091463C2363E7F6066C
:108C8000CD4691CF0546F546638BC7000946C946D8
:108C90006387C7000D46C1466383C700D54634A32A
:108CA000930571001305F041EF2022459C83C5E335
:108CB00017B7FB1F034727218D47631AF708EFD02B
:108CC0004FC52C00EF70100D2800EFD07FAC45454C
:108CD000EFD0FFD125E50144B250228522549254B1
:108CE0000259F249624A45618280ED1793F7F70F06
:108CF00095460544E3E2F6FE97560200938686BC4D
:108D0000B3C7D7209C43B697828789473CA319A055
:108D1000230107006545EFD09FCD9307F007E301DE
:108D2000F5F8032709003C2393E707043CA38DBF14
:108D30008547E9BF9947D9BF9147C9BF130600646A
:108D40003306C50288209145EFB00FC469B71533CB
:108D50002A8451D1EFF01FBB41B7011126CA97B445
:108D6000FB1F9384A4EA9C4022CC06CE4AC8494407
:108D7000A1C79C230D446391A70417B9FB1F1309D6
:108D80006936034509008945EFB06FE903450900DD
:108D9000914597B7FB1F239107ECEFB04FE89C403C
:108DA0000147814680B31306F1008547854501459B
:108DB000DC87EFA0F0722A84F24022856244D2441C
:108DC000424905618280011106CE22CC26CA4AC8DA
:108DD0004EC68547631EF50617B4FB1F1304C4E790
:108DE0001E20B1CB17B7FB1F0347070E29E7130758
:108DF000B003636EF70297B4FB1F9384A42E882000
:108E00008945EFB0CFE11220930700648820330634
:108E1000F6028945EFB04FB797B7FB1F239E07E2D5
:108E2000F2406244D2444249B2490561828093874C
:108E300047FC1EA0F5B797B7FB1F83A727DDEDD32F
:108E40006244F240D2444249B2498823056131B7B5
:108E500097B9FB1F938989DB83A70900F1D317B961
:108E6000FB1F1309292883474900918BD5DB8947CC
:108E70006311F5062D45AE849770FB1FE7804041D6
:108E80002A8459DD930700FD1CA1E547A3000500D6
:108E90003CA1BC3015051946230FF5FEDC20938557
:108EA0005400A30FF5FE9770FB1FE780604E03454B
:108EB00059009307F00F6315F50083A70900882375
:108EC000A2856244F240D2444249B24905616FB082
:108ED000CF81034509008945EFB06FD46244F24069
:108EE000D2444249B24997B7FB1F239707D6056181
:108EF0006FF05FA197B7FB1F83C7071F958B89CFC3
:108F000097B7FB1F83A787D491CB854717B7FB1F64
:108F1000A305F7D46FF07FA1494582804145828047
:108F200097B7FB1FA38B07D2854501456FA0105C47
:108F300097B7FB1F83C7471B958B81CB854717B717
:108F4000FB1F230CF7D06FF05FA14945828097B7D4
:108F5000FB1F238407D0814505456FA0305B97B781
:108F6000FB1F83C76718958B638B0712011122CCF7
:108F700006CE26CA4AC84EC69307C01C328463FA7E
:108F8000C7000945F2406244D2444249B2490561F2
:108F9000828097B7FB1F83A767C76384071097B7C3
:108FA000FB1F9387B7CBB68994231307E00F639A0F
:108FB000E60E88A31305860033450508ADC9916503
:108FC000938565719770FB1FE780C00CAA8455D903
:108FD00017B9FB1F130909C80325090009C59770B4
:108FE000FB1FE78040181385840088C022868145D6
:108FF000232099009770FB1FE7800040832709001A
:109000002286CE8588439770FB1FE78060388327D0
:109010000900A286F240C2A36244D2444249B24946
:10902000984305468D45054505616FA0F04A916559
:10903000938555719770FB1FE780C005AA8431D1D5
:1090400017B9FB1F1309C9C00325090009C597708B
:10905000FB1FE78040111385840088C0228681456C
:10906000232099009770FB1FE780003983270900B0
:109070002286CE8588439770FB1FE7806031832767
:109080000900A286F240C2A36244D2444249B249D6
:10909000984305468D45054505616FA03044494517
:1090A00082804945C5B59307C01C63FCA7000945EC
:1090B00082800945F2406244D2444249B249056186
:1090C0008280011122CC06CE26CA4AC84EC62A8406
:1090D00025C1AE89916521059385657133450508E4
:1090E0009770FB1FE78000FBAA8461D517B9FB1FAF
:1090F000130949B60325090009C59770FB1FE780CE
:1091000080061385840088C022868145232099002B
:109110009770FB1FE780402E832709002286CE85AB
:1091200088439770FB1FE780A02683270900C2A30E
:1091300097B7FB1F83A787AD85CF97B7FB1F83C763
:10914000A7FA958B85CB97B7FB1F83A7A7B091CFC5
:109150009843D6236244F240D2444249B24905467C
:109160008D45054505616FA0303701478146DDB764
:10917000014589B749453DBF9307C01C63FCA70063
:10918000094582800945F2406244D2444249B249CD
:1091900005618280011122CC06CE26CA4AC84EC67D
:1091A0002A8425C1AE899165210593855571334582
:1091B00005089770FB1FE780E0EDAA8461D517B919
:1091C000FB1F1309E9A80325090009C59770FB1FB8
:1091D000E78060F91385840088C0228681452320BA
:1091E00099009770FB1FE7802021832709002286C2
:1091F000CE8588439770FB1FE7808019832709007D
:10920000C2A397B7FB1F83A767A085CF97B7FB1FA4
:1092100083C787ED958B85CB97B7FB1F83A747A3A4
:1092200091CF9843D6236244F240D2444249B24996
:1092300005468D45054505616FA0502A01478146C9
:10924000DDB7014589B749453DBF9307C01C63F4AD
:10925000A70009458280797122D406D626D24AD049
:109260004ECE2A842DC1AE899165210593857571F5
:10927000334505089770FB1FE780C0E1AA840945C4
:10928000A9C817B9FB1F1309699C0325090009C563
:109290009770FB1FE78020ED1385840088C022862D
:1092A0008145232099009770FB1FE780E0148327F6
:1092B00009002286CE8588439770FB1FE780400D0A
:1092C00083270900C2A397B7FB1F83A7279489EBC5
:1092D0000145B250225492540259F24945618280AC
:1092E00097B7FB1F83C747E0958B4945FDD36C00BB
:1092F0001305D030EF30B20FB24793F7070FE9DB19
:1093000097B7FB1F83A787949443D2238D450545C8
:10931000EFA0901D7DBF97B7FB1F83A7A79389CFB1
:10932000D2238C43411106C69770FB1FE78040068D
:10933000B2400145410182800945828097B7FB1FF9
:1093400083A7479185C717B7FB1F032767908947F6
:1093500019CF52230C43411106C69770FB1FE780BB
:109360002003B24081473E854101828089473E8586
:10937000828097B7FB1F83A7E78D85C717B7FB1FB1
:109380000327C78C894719CF52230C43411106C6C6
:109390009770FB1FE780C0FFB24081473E854101C7
:1093A000828089473E858280797126D206D622D472
:1093B0004AD04ECE97B4FB1F9384C4B08D4783C967
:1093C000240063FAA7000945B2502254925402596E
:1093D000F2494561828098202A844145E316F7FED0
:1093E0009307F4FF93F7F70F854663E8F60A2E8993
:1093F000B1ED99452800EFC0BFA2A0A0914517B5D7
:10940000FB1F034525CEEFB08F812800EFD04FB86A
:1094100055E9930571001305F041EF10124E9C833E
:10942000D1EB8D476318F4084545EFD04FDC59C1A7
:1094300037761800130606A03306C502914517B506
:10944000FB1F034525CAEFA09FF5ADA01946814536
:1094500028009770FB1FE78020FA19462C004A85E8
:109460009770FB1FE780400539FD19469305F00F03
:1094700028009770FB1FE78020F819462C004A85CA
:109480009770FB1FE78040031DFD1946CA85280021
:109490009770FB1FE780C0EF8DB7630FE400914525
:1094A00017B5FB1F034505C497B7FB1F238D07A006
:1094B000EFA0FFF6014509BFC8442C00EF70800DF6
:1094C000A0A00DDD2381340101B797B7FB1F83C72F
:1094D000A7C1918B8DC3411117A5FB1F1305C5763D
:1094E00006C6EFC05F93B240FD5717B7FB1F231EA0
:1094F000F79C4101828001456FC0FF91FD5717A77E
:10950000FB1F230DF774F95717A7FB1FA308F77468
:1095100097A7FB1FA383077497A7FB1F238F0772CF
:1095200097A7FB1F239A077297A7FB1F23A4077215
:1095300097A7FB1F23AE077097A7FB1F23A80770F1
:1095400097B7FB1F9387479B170700001307E72078
:1095500098C31707000013074787D8C317F7FFFF03
:109560001307675198C717F7FFFF1307473CD8C782
:1095700017F7FFFF1307A73E98CB97F7FFFF9387D7
:10958000474317A7FB1F2321F76C8280411126C296
:1095900097A4FB1F938484679C4006C622C495CB86
:1095A0002A840D459770FB1FE78080CEAA8519C9D4
:1095B000930700FD1CA18D4700B13CA19C4088236E
:1095C000EFA0BF9219C42244B240924441016FF00F
:1095D0006FB3B240224492444101828079714AD0F3
:1095E00017A9FB1F130989628327090006D622D415
:1095F00026D24ECE6383070E98338547AA8497B947
:10960000FB1F9389298C6301F70483C749008DE709
:109610000D459770FB1FE780A0C7AA8501CD930772
:1096200000FD1CA1914704B13CA1832709008823B8
:10963000EFA0BF8BEFF00FAD0545B250225492540E
:109640000259F2494561828097A7FB1F83A7876073
:1096500089CB9443D2239305E1000545EFC07F8673
:1096600011ED0145EFD0AFB82A8621C6894517B55F
:10967000FB1F034525A7EFA03FB125A81C21858B23
:10968000EDD30545EFD0AFB69307B0032A8463F15D
:10969000A7045D6613060670894517B5FB1F0345D1
:1096A00065A4130444FCEFA09FCF97A7FB1F23954D
:1096B000875A83270900094798B383C7490091C790
:1096C00097B7FB1F2382078085BF2685C135ADB7BD
:1096D000930700643306F50249BF0145B9BF411144
:1096E00022C42A840D4506C69770FB1FE78040BA46
:1096F0000DC1930700FD1CA1CD4700B13CA1224440
:10970000B240AA8517A5FB1F0345455541016FA02F
:10971000CFFDB240224441018280411122C42A84FB
:109720000D4506C69770FB1FE78080B60DC19307F5
:1097300000FD1CA1ED4700B13CA12244B240AA8526
:1097400017A5FB1F0345855141016FA00FFAB240D9
:109750002244410182805A210111896606CE22CC21
:1097600026CA13866600AA876316C7009C47014570
:109770008C2371A8138606046365E60413865603DA
:10978000636FE60013869600630BC7081386A60076
:10979000630DC712A1066309D7060145A5A8F9768E
:1097A0009386A6FC3697A94633470708E3E7E6FE0B
:1097B00097460200938686123347D7201843369780
:1097C0000287138616056307C71893862605E316D6
:1097D000D7FC1C45802397A7FB1F83C7074822851A
:1097E000639D07160D459770FB1FE78060AAAA8549
:1097F0000DC1930700FD1CA1F14700B13CA117A5C5
:10980000FB1F0345A54591A29C4705458C23EFF01E
:10981000AFB60545F2406244D2440561828017A785
:10982000FB1F0327A73E014575D79C47882359E9AD
:1098300085471CB30545EFA0A040E1BF1C4597A498
:10984000FB1F9384B4411307E00F80239C20638B9C
:10985000E7021307F00F6384E70211459770FB1FBF
:10986000E78000A3AA8501CD930700FD1CA18947CD
:1098700000B13CA1A30105008820EFA00FE7F95734
:109880009CA041BF97A4FB1F938444389C40014592
:10989000D1D305E805447D454085EFD04F956886D6
:1098A00013050002EFD0AF949C40C8851307B100A8
:1098B00080B374001306A10085450545EFA0404222
:1098C00089BF2285EFF09FCCA9B79C476244F24044
:1098D000D244882305616FF07FD01C4509458C2355
:1098E0003DB71C4588232DE56C001305D030EF30C3
:1098F0000230B247414793F7070FE38CE7F0930537
:10990000B10013056031EF30822E88858545EFA0C8
:10991000E03D01B71C45802397A7FB1F83C7F733A2
:1099200022859DE70D459770FB1FE7806096AA850D
:10993000E30105EE930700FD1CA1D14700B13CA156
:1099400097A7FB1F83A7872C8823EFA00FDAD1B539
:109950007933C1B51C45882319C1C1335DBD854527
:109960000545EFA0A03A75B5411122C417A4FB1F0D
:109970000344847706C6158809CC17A5FB1F130579
:10998000A557EFC0AFC84D44B240228522444101E3
:1099900082800145EFC08FC7C5BF9821937625000F
:1099A0009377D70F99C29367270093F6F70713179A
:1099B00045606354070093E607081378850093F722
:1099C000760F6304080093E786009376050299CE2C
:1099D00093E707029CA1635707001C2293E7C70087
:1099E0001CA282801375A5026DF9828093F7F7FDA2
:1099F0009CA1E34407FE9377A502E5F37DF11C22C9
:109A0000CD9BF9BF2D45631C0710011126CA4AC81A
:109A10004EC606CE22CC9821BE8989472E89B684AF
:109A2000631EF704DC413284983394232207558F58
:109A30008D66938746A01316576063C9C702938645
:109A4000F69F63DDC602F5779387F75F3E978D47F4
:109A5000C8453347070863E7E70297460200938645
:109A6000A6EA3347D7201C43B6978287938766AA16
:109A7000630EF608938686B8630FD6082390040019
:109A8000054525A09770FB1FE780009B334605081E
:109A90003356360B92A08325C9001DA01E2109470D
:109AA0009AA01CA0A1831CB00145F2406244D2449C
:109AB0004249B2490561828099479EA01946AA850C
:109AC00022859770FB1FE780A08CF9BF85479EA079
:109AD0001C211CA0D1BF05C9A1479EA01E211CA00E
:109AE0001E21A1831CB03E213CA03E21A1833CB09D
:109AF0005E215CA05E21A1835CB07E217CA07E21E2
:109B0000A1837CB055B72390040079BF85479EA000
:109B1000DC459C237DBFE1479EA06146ADBF8280AE
:109B2000797122D44AD006D626D24ECE52CC56CA0D
:109B30003A89982189472E84631DF7025C40B684D8
:109B4000B28503C8170094238D6722083368D800B4
:109B5000938627A013185860630BD8102A8A63CC09
:109B60000601938607A0630BD802938717A06300B2
:109B7000F80A854711A8138737A0630FE80A1387EF
:109B800067AA8D47E317E8FEB25022549254025957
:109B9000F249624AD24A3E8545618280484432C6D3
:109BA0009770FB1FE78040899D4733450508E36DAB
:109BB00025FD97AAFB1F938AAA0B83C70A00B30946
:109BC0009900B24563D43701B5477DBF4844268626
:109BD000B3C909084A959760FB1FE780607B03C6FD
:109BE0000A00484481450506330636414E95977074
:109BF000FB1FE780608097A7FB1F83A7A70799E358
:109C0000814759B79C438145E5DF528525A0AD4783
:109C1000E31C09F6E39AE4FA1C321822A207D98F52
:109C200058441EA397A7FB1F83A7C704F1DB9C43DF
:109C30008545F9D78297E9B717A7FB1F0347F702B6
:109C40008D4739D3AD47E31109F49947E39EF4F604
:109C5000484419469760FB1FE780807397A7FB1F56
:109C600083A74701D1DF9C43C1DF8D4579BF17A78B
:109C7000FB1F034707EF218B8D4719D7AD47E3152E
:109C800009F08547E392F4F4182293070008E3ED06
:109C9000E4EE5C4498A3ADB7411122C4094497A7F0
:109CA000FB1FA38187EC97A7FB1FA38C87EA97A7CD
:109CB000FB1F238887EA97A7FB1F23AD07FA97A707
:109CC000FB1F238E07F897A7FB1F238307FA97A78D
:109CD000FB1F239E07F897A7FB1FA38807F8A14740
:109CE0001946814517A5FB1F1305C5F706C617A71B
:109CF000FB1FA307F7E69760FB1FE780E06F97A7BE
:109D0000FB1F238F87E4B707A00017A7FB1F1307CC
:109D1000A7E4938707051CC3B707E8035CC397A7AD
:109D2000FB1F238987E285476146814517A5FB1FF5
:109D30001305C53017A7FB1FA30DF7E097A7FB1F5F
:109D4000238987E097A7FB1FA38487E097A7FB1FC2
:109D5000238807F09760FB1FE780006A97A7FB1F27
:109D6000238887DE97A7FB1FA38B07EE97A7FB1F10
:109D7000938747D8B2402244170700001307C7C88B
:109D800098C3170700001307E7D9D8C323A4070017
:109D900041018280797122D426D206D64AD04ECE95
:109DA00052CCA1472E84B28463EBA7001747020070
:109DB000130787B63345E5201C41BA97828793077E
:109DC00010086304F51C63ECA70093072004630EDE
:109DD000F516930700086303F518094591A093074A
:109DE0002008E31CF5FE8547639BF5020822937764
:109DF000250095E797A7FB1F83C727E71387F7FF82
:109E000097A5FB1F93858510120792072E97A10730
:109E10005047BE9585AA9307800F63FBB700614545
:109E2000B250225492540259F249624A45618280EA
:109E300017AAFB1F130A0AD383470A0017A9FB1F9F
:109E40001309C90C9207CA97C84709C99760FB1F35
:109E5000E780603197A7FB1F238C07E013061400EF
:109E60001376F60F916593850571328583490A0053
:109E700032C69760FB1FE780E02183470A00920902
:109E8000CA99920723A6A900CA97C84749D932465A
:109E900081459760FB1FE780205683470A00228692
:109EA000A68592073E990325C9009760FB1FE780AE
:109EB000204E97A7FB1F238D87DA014595B7894769
:109EC000E39FF5F41E2217A7FB1F2312F7DAF5B75D
:109ED0008547E396F5F41C2217A7FB1FA307F7D8C5
:109EE000E9BF9947E39DF5F21946A68517A5FB1F23
:109EF000130545D79760FB1FE78080497DBFA147C9
:109F0000E39FF5F02146A68517A5FB1F1305C5C4E1
:109F1000D5B78547E395F5F01C2217A7FB1FA30AC9
:109F2000F7C261BFE147E39CF5EE6146A68517A540
:109F3000FB1F1305A5107DBF8547E392F5EE1C229C
:109F400017A7FB1FA30DF7D08DBF8547E399F5EC4D
:109F50001C2217A7FB1F2306F7C085B78547E39090
:109F6000F5EC97A7FB1F83C7E7BF1387F7FF97A5FC
:109F7000FB1F9385A5F912072E979207504788205B
:109F8000A107BE95EFF07FA10DBF8547E399F5E8E6
:109F900097A7FB1F83C787CDC9BFAA8721472E85F7
:109FA000636DF7001747020013074799B3C7E7200F
:109FB0009C43411106C6BA97828713072004638B1E
:109FC000E70889473E85828017A7FB1F034787B9AB
:109FD000120797A7FB1F938767F3BA97CC47894768
:109FE00085C117A6FB1F0346A6C89760FB1FE78025
:109FF000203A31A097A7FB1F83D767C79EA181474F
:10A00000B2403E854101828097A7FB1F83C7F7C5F9
:10A010001CA1F5B7194697A5FB1F9385A5C4F1B7F9
:10A02000214697A5FB1F938525B3EF907FD7C1BF2E
:10A0300097A7FB1F83C7F7B1E1BF614697A5FB1F39
:10A040009385C5FF5DB797A7FB1F83C757C1C9B7E6
:10A0500089477DB797A7FB1F83C7A7B09CA18147FE
:10A0600095B76300053A97A7FB1F938747BF9823CF
:10A0700063190738054798A397A7FB1F938707E93C
:10A08000894698A717A7FB1F231707E817A7FB1FE9
:10A09000130747AF94A397A6FB1F938666B2D8C752
:10A0A000D4C37D57630CE53413771500854529C764
:10A0B00017A6FB1F231906E6094797A6FB1F9386E1
:10A0C00066AF17A6FB1F1306F6A998ABD4CBD0CF6B
:10A0D000854617A6FB1F2307E6A82380E70217A7DC
:10A0E000FB1F1307A7ACD8D394AF2384D70217A7BD
:10A0F000FB1F231207E48D451377250025C3139713
:10A1000045003E9797A6FB1F9386C6AA094654C3EF
:10A1100017A8FB1F1308F8A4854610A314A723262D
:10A12000070123150700138715003347070817A8F1
:10A13000FB1F230DE8B212073E9710A314A717A622
:10A14000FB1F130666A697A6FB1F938646B28905DA
:10A1500050C32315070054C7B3C50508137745003E
:10A1600025C3139745003E9797A6FB1F938686A4A9
:10A17000094654C317A8FB1F1308A89E854610A3C1
:10A1800014A723260701231507001387150033475B
:10A19000070817A8FB1F230AE8AC12073E9710A375
:10A1A00014A717A6FB1F1306E69F97A6FB1F93860F
:10A1B000D6AB890550C32315070054C7B3C505089E
:10A1C0001377850021CF139745003E9717A6FB1FF5
:10A1D0001306469E50C30546894610A717A6FB1FC7
:10A1E0001306169814A32315070050C713871500EC
:10A1F0003347070812073E9714A397A6FB1F9386C1
:10A20000269A54C3A14614A797A6FB1F938686A53A
:10A2100089052315070054C7B3C505081377050141
:10A2200021CF139745003E9797A6FB1F93868698EC
:10A23000094654C317A8FB1F13088892854610A32C
:10A2400014A723150700232607011387150033479A
:10A25000070812073E9710A314A717A6FB1F1306A3
:10A26000E69397A6FB1F9386268F890550C3231577
:10A27000070054C7B3C505081377050221CF13970C
:10A2800045003E9797A6FB1F9386C692094654C386
:10A2900017A8FB1F1308088C854610A314A72315C5
:10A2A0000700232607011387150033470708120705
:10A2B0003E9710A314A717A6FB1F1306A68D97A6FB
:10A2C000FB1F93861689890550C32315070054C7C1
:10A2D000B3C505081377050421CF139745003E97B2
:10A2E00097A6FB1F9386068D094654C317A8FB1F2C
:10A2F00013082886854610A314A7231507002326D4
:10A300000701138715003347070812073E9710A36C
:10A3100014A717A6FB1F1306268897A6FB1F938674
:10A320002694890550C32315070054C7B3C50508F3
:10A330001377050821CF139745003E9717A6FB1FFB
:10A340001306468750C35146894610A717A6FB1F20
:10A350001306168014A32315070050C71387150092
:10A360003347070812073E9714A397A6FB1F93864F
:10A37000268254C3854614A797A6FB1F938606CC56
:10A3800089052315070054C7B3C5050813750510C3
:10A3900039C9139745003E9797A6FB1F9386868180
:10A3A00054C3094685461795FB1F1305657A10A30C
:10A3B00014A72315070048C713871500334707085C
:10A3C0001207BA971797FB1F1307877CD8C317A7E5
:10A3D000FB1F1307D788890590A394A7239507002F
:10A3E000D8C7B3C505089796FB1F9386A67041464C
:10A3F00017A5FB1F130585B16F300042130530030D
:10A4000045B9014582800111FD1522CC06CE32846A
:10A4100026CA3E864AC813F8F50FAD4763E8070B16
:10A420003A89173702001307A7533348E8208327D8
:10A430000800B684BA9782878545EFB09FBA01E5D8
:10A44000EFF08FD20145F2406244D24442490561A7
:10A4500082808945EFB0FFB87DF52285EFE06FC0BF
:10A46000D5B7914532C6EFB0DFB7324669FDCA8530
:10A470002685EFB0BFADEFF02FCFEFF00F85EF6087
:10A48000A078C9B7A14532C6EFB0BFB5324645FD89
:10A49000CA852685EFB09FAB2285EFE08FBCEFE049
:10A4A0000FB3EF60407479BFB14532C6EFB07FB3F0
:10A4B000324651F9CA852685EFB05FA92285EFE0C3
:10A4C0004FBAEFE0CFB0EF60007275B70945A5BF96
:10A4D00079714ECEAE896C0022D426D24AD006D6EF
:10A4E0002A89B284EF00306E2A840DE1CE854A8538
:10A4F000EFB04F8E2A8419E93245268797B6FFFFC1
:10A500009386C60C2D468145EF100006B250228579
:10A51000225492540259F24945618280397126DAF7
:10A52000AE844C0022DC4AD84ED652D406DEAA892C
:10A530003289368AEF0030692A8421E9A685630DC5
:10A5400009009E202C007C84BE207C85930720304F
:10A550007C86930780025C874E85EFB0CF842A8487
:10A560000DE55946A6851305A10023042101976036
:10A57000FB1FE780E0E11245528797B6FFFF938605
:10A58000060025462C00EF00307EF25022856254F2
:10A59000D2544259B259225A21618280797126D20D
:10A5A000AE846C0022D44AD04ECE06D6AA89328917
:10A5B000EF0070612A840DE1A6854E85EFB04F83D0
:10A5C0002A8419E932454A8797B6FFFF9386C60168
:10A5D0003546A685EF005079B25022852254925418
:10A5E0000259F249456182807547AA876365B702BF
:10A5F000114701456378B702ED1593F5F50F6147F3
:10A600006361B7029736020093868638B3C5D520BA
:10A6100098413697028793F5F50713072005638A5B
:10A62000E50001458280C847828088438280884750
:10A630008280C84382809307F00F630FF5060111F3
:10A6400026CAAA841305000222CC4AC84EC652C4A8
:10A6500056C206CE2E8AB28AB6893A899760FB1F07
:10A66000E78000C32A844D450DC8930700FB1CA05A
:10A67000A300540123114401230234011305840073
:10A68000614663050902CA859760FB1FE78040D0D9
:10A69000A2852685EF907F850145F2406244D24431
:10A6A0004249B249224A924A0561828081459760B7
:10A6B000FB1FE78060D4E9BF09458280011122CCED
:10A6C00006CE2A844C86D0869780FB1FE780C02D5B
:10A6D00005C15425214797A7FB1F9387A7A0639D1A
:10A6E000E600E82378009306E0070146A285A1373B
:10A6F000F240624405618280C83378009306E00727
:10A700000146A285EDB7930700643306F6026F9009
:10A71000FFBC15C1411122C406C62A840821930733
:10A72000D00F63E6A700EF903FD9FD571CA0B240C1
:10A730002244410182808280797122D406D626D2B9
:10A740004AD04ECE9E2509448DEBAE846C00AA897A
:10A750003289EF0050472A840DE1A6854E85EFA08F
:10A76000FFF42A8419E932454A8797B6FFFF93869A
:10A77000A6F34D468145EF00305FB250228522544A
:10A7800092540259F249456182801A219307000BC5
:10A790006310F7025C214947639AE700183985473F
:10A7A0006398E7002A2185456F30902A6D47CDBF19
:10A7B000828001116C846C0022CC26CA4AC806CE65
:10A7C0002A89B6847085EF0010402A840DE12C00A0
:10A7D0004A85EFA01FD42A8419E93245268797B607
:10A7E000FFFF9386C6CE15462C00EF00F057F240CF
:10A7F00022856244D244424905618280797193077F
:10A8000020306C8470857C862C0093078002014682
:10A8100006D65C87EFF09FD0B25045618280C17749
:10A82000797185073EC4894726D27C86AE8493071A
:10A8300080024C0022D44AD006D62A895C87EF00D9
:10A8400090382A840DE12C004A85EFA09FE32A84EA
:10A8500019E91245268797B6FFFF9386C6DF45465E
:10A860002C00EF007050B2502285225492540259AD
:10A8700045618280B28605466FF05FCA797126D243
:10A88000AE846C0022D44AD04ECE06D6AA89328934
:10A89000EF0070332A840DE1A6854E85EFA01FBF1F
:10A8A0002A8419E932454A8797B6FFFF9386C6BCCA
:10A8B0000D46A685EF00504BB2502285225492548B
:10A8C0000259F249456182807971930720206C8496
:10A8D00070857C862C0093078002014606D65C8733
:10A8E000EFF0DFC3B25045618280011122CC26CA4D
:10A8F0004AC806CE2A84AE84328936C69780FB1FAA
:10A90000E780800A15C95025A14632479797FB1F5B
:10A910009387477D631DD600E823CA862686A285D5
:10A920006244F240D244424905616FF0DFD0C8333F
:10A93000CA862686A285EDB7F2406244D2444249D7
:10A940000545056182806FF0BFB86FF07FB86FF08A
:10A95000FFC46FF0BFC479714ECEAE896C0022D4B3
:10A9600026D24AD006D62A89B284EF00D0252A847E
:10A970000DE1CE854A85EFA07FC92A8419E93245C9
:10A98000268797B6FFFF9386E6C73D468145EF00D1
:10A99000B03DB2502285225492540259F249456189
:10A9A0008280B28601466FF07FB7011122CC2E84DF
:10A9B0006C0026CA06CEAA84EF00F020DD476309AA
:10A9C000F500930710101EA4A2852685EFA01FCEC8
:10A9D000F2406244D24405618280239405006FF006
:10A9E000BFD5E5BF1797FB1F0347472D854763F882
:10A9F000E702011122CC2E846C0026CA06CEAA845E
:10AA0000EF00701C01E9930700101EA4A2852685A3
:10AA1000EFA0DFC9F2406244D2440561828059450B
:10AA200082809797FB1F23ABA72482809797FB1FF9
:10AA300023A4A7248280011122CC26CA06CE2A8410
:10AA4000AE849780FB1FE78020F6A6852285EFA0C5
:10AA5000EFF705E9228564869780FB1FE780C0F445
:10AA60000DC1542521479797FB1F9387A767639FC5
:10AA7000E600E82378009306F0070146A285EFF090
:10AA80009FBBF2406244D24405618280C833DDB787
:10AA9000797122D44AD0AE8706D6BA8526D24ECE58
:10AAA0007547328436896364F7042147636CF70085
:10AAB00015476388E7021947638DE708C167FD17EB
:10AAC00085441DA037061400DD1713060620B317B2
:10AAD000F0287D8E49EE19677D8F25EB93F71710CF
:10AAE000F1DFC167FD1789446316F40221A813F74B
:10AAF000F70793062005E313D7FC41677D17631E14
:10AB0000E6048D442EC6EFA02FF0B24533049540E5
:10AB1000334404083385840033450508EF30D00002
:10AB2000AA87B3C9040821C9630409002310890056
:10AB30002254B25092540259B3053041F2493E8535
:10AB400045611753FB1F6700836FC167FD1795446D
:10AB500061BFC167FD179D4441BF1307200D8D44A0
:10AB6000E39AE7FA1304C6003344040865B7C167E3
:10AB7000FD178D4495BFB250225492540259F249A8
:10AB800045618280011122CC26CA06CED0212E84B6
:10AB90001307000281469945AA84DD3D2AC621C5D6
:10ABA0001E205020930554007C803E207C818947E4
:10ABB0007C82930780025C839750FB1FE780407D77
:10ABC0005C208A8526857C84EFA05F972A8411C546
:10ABD00032459750FB1FE7800059F24022856244BE
:10ABE000D244056182804D44CDBF397122DC26DA22
:10ABF0004AD806DE89472A84AE8436896306F60081
:10AC0000C14709456315F60432C6A9C04C08228520
:10AC1000EF00607B324605EDC1778507A6851305F9
:10AC2000D1013ECC230EC1009750FB1FE780407638
:10AC30002C082285813F01ED52454A8797B6FFFFD8
:10AC40009386668E1D462C08EF0010120145F250C7
:10AC50006254D254425921618280397126DA4AD82D
:10AC60004ED63289AE893686BA84814613071002E1
:10AC7000D94522DC06DE2A8432C6EFF07FE12ACEF7
:10AC80001DCD3246A685231A3101F084231B2101F4
:10AC90009750FB1FE780C06F22854C08EFA0BFAA2A
:10ACA0002A8411C572459750FB1FE780C04BF250B4
:10ACB00022856254D2544259B259216182804D4456
:10ACC000FDB7011122CC06CE26CADD472A84639F38
:10ACD000F5085439B1441C49B38696023287B697B9
:10ACE000904314436306D6020A20230601006C0039
:10ACF000EFA01FA90824B165938505B8EF90EFBABE
:10AD0000E5473CA097B7FFFF938747A75CC091A892
:10AD10005623D223E31AD6FC88470C479750FB1FD3
:10AD2000E7808079AA870A2089E7230601006C0062
:10AD3000C1B75C385828850793F7F70F5CB863F400
:10AD4000E702B38797021848BA979847D623B223E9
:10AD50008E23213751F90824B165938505B8EF900A
:10AD6000CFB4D94431A87C285C86D1B70A21AE84FF
:10AD70006C0023060100EFA0BFA08547E39CF4F61A
:10AD8000F24062442685D24405618280011122CCC2
:10AD900006CE26CADD472A840A216398F508EFA06B
:10ADA000AFC6522C3E284E286D162A96334606080A
:10ADB0003307F64052ACAA86334707080A2063726D
:10ADC000B7061388C6FFB388E54063D40803AE977F
:10ADD000918FB3C607081C4C0E283E97EFF0FFE793
:10ADE00009ED0824B165938505B8EF900FACD944FF
:10ADF000B1A0ED16B3C60608F9BF0A20230601006C
:10AE00006C00EFA0FF970824B165938505B8EF901B
:10AE1000CFA9E5473CA097B7FFFF938727965CC073
:10AE2000F9B785475C866C00E9BFAE846C002306E9
:10AE30000100EFA0FF948547E397F4FCF2406244E1
:10AE40002685D24405618280397126DAAE842C00D1
:10AE500022DC4AD84ED606DE2A89B289AD232A845E
:10AE600031E54A85EFA04FBAD6206D1563C4A60020
:10AE7000B34605089844B2208E204A85EFF0FFDDE6
:10AE80002A840DE53146A68508082306010097505F
:10AE9000FB1FE780E04FBE2022454E8797B6FFFF9D
:10AEA000938666875D466C00FC867D2DF250228578
:10AEB0006254D2544259B2592161828071B769B744
:10AEC000797122D406D626D24AD04ECE52CC56CA5A
:10AED0005AC80944C1CD3289094449CAAE84BA8AE4
:10AEE0002A8A368BEFA04FB2138744008147711531
:10AEF000162363DEA608850793F7F70F3107E319DA
:10AF0000F9FE8A855285C1212A842DE13145330518
:10AF1000A9029165938515704D449750FB1FE780FA
:10AF20006017AA8921C531463306C902A685975004
:10AF3000FB1FE780E0459844D620B2208E20528542
:10AF4000EFF0BFD12A8415ED02458547568797A6B5
:10AF5000FFFF9386467C5D464C005C824EC4230610
:10AF60002101A306010023076101FD2BB2502285B8
:10AF7000225492540259F249624AD24A424B4561E4
:10AF800082804E859750FB1FE780E01DC5B76D445A
:10AF9000F1BF79714ECEAE89C16526D20147AA8430
:10AFA00089461796FB1F130666BEFD15054522D47C
:10AFB00006D64AD0EF101001054429C92A89130783
:10AFC000300281461146F5452685EFF07FAC2AC652
:10AFD00055440DCD0357A900CE860146788411470C
:10AFE0007885054718A1B2472C002685A380070065
:10AFF0003247FD573CA332473CB3EF10E0712A843F
:10B0000011C532459750FB1FE780E015B2502285ED
:10B01000225492540259F24945618280411106C678
:10B02000EFF08FDC19C5B24041011753FB1F6700D9
:10B030008313B24041018280011106CE2AC6EFA0DF
:10B04000EF82324591459797FB1F23A907C2979737
:10B05000FB1F23A307C29797FB1FA385A708EF3009
:10B06000C027F24005616F20700F79714AD006D673
:10B0700022D426D201499397556063D807041795C7
:10B08000FB1F034535062E899750FB1FE78040269E
:10B090002A845DC518219307000A6310F70A8547C3
:10B0A0004C08DC85EFA00F8AAA841DC59C8599C732
:10B0B000084409C59750FB1FE780E00A2A20854510
:10B0C000EF300019CD47639AF406B25022549254DF
:10B0D0004A850259456182808347610191CF71475A
:10B0E0006363F7064D476378F7069386C7FE130739
:10B0F00030143357D74825C31797FB1F0327C7B70B
:10B1000001C7034751012DCB9C8599C7084409C548
:10B110009750FB1FE78020055247B7070001938730
:10B1200007F07D8FB7071200938707106307F700BA
:10B1300003476101ED476302F70A2285EF80DFD5FF
:10B140001319F96859B7138717FE1377F70F93068A
:10B150000002E3F3E6FA858B9DCB9797FB1F83A74D
:10B16000E7B1A5C72A201306B1004C0882979C8539
:10B17000AA84ADEBD5D099B75C8699472308F10036
:10B180002A206C0023170100EFA06F9EB5BF979790
:10B19000FB1F83A767AE85CB2A201306B1004C089E
:10B1A0008297AA8435D183475101E39107F02308A0
:10B1B0009100834761012A206C005C8623170100FF
:10B1C000EFA0EF9AE5B59944F9BF9C8599C708446B
:10B1D00009C59750FB1FE78000F92A208545EF300D
:10B1E0002007A1BF084459D59750FB1FE780A0F75F
:10B1F00051B75D71A2C4A6C286C6CAC04EDE52DC7B
:10B2000056DA5AD85ED6A5472A84B2846392F50EE0
:10B21000834745021A22322285072302F50293074B
:10B22000F7FFB307F602D440B3C70708B697542513
:10B2300003CB070003C917008547638BF6049317F8
:10B240008900B3E7670141677D17638AE70A1A2817
:10B2500063F7E70A50248507B3C7070885467EA42D
:10B260000A209305E400631BD6007C8493072030FA
:10B270007C869307800278855C872C00EFA0AFB2B4
:10B280000824B165938505B8EF803FE259458DA844
:10B290003307C702239004008149014A930B35010B
:10B2A000B34A0708E3FD59F9B620DC402C28138681
:10B2B0005900ED163E965E85B3C60608EF901FE076
:10B2C0001DC1630B3A01C840B220B3053501529548
:10B2D0009750FB1FE780C00BBE203E9A9E20334A4A
:10B2E0000A0885079EA0BE20BE99B3C909085DBFA4
:10B2F0005822A9476311F7028347450289CF0145C8
:10B30000B640264496440649F259625AD25A425BE4
:10B31000B25B616182803428130934014A86894511
:10B320001795FB1F1305C589EF905FD939ED3428B8
:10B330004A8689451795FB1F13054588EF901FD84E
:10B3400029E534284A8689451795FB1F1305C586CC
:10B35000EF90DFD61DE934284A8689451795FB1FF3
:10B3600013054585EF909FD50DE1DC2009476380EB
:10B37000E702ED1793F7F70F29476368F700130704
:10B380009048B357F700858B99E3054595BF8347F0
:10B39000440285072302F402BE2075B5411122C480
:10B3A00006C62E849770FB1FE780C05509C93C254F
:10B3B000138717006315E40093F707F83CA5B24024
:10B3C000224441018280411122C406C62E84977016
:10B3D000FB1FE78020531DC111C008C01C251307A7
:10B3E000E00F5D456388E7001307F00F594563934D
:10B3F000E7000145B2402244410182800945DDBF9A
:10B40000411122C42A84210526C206C64AC0EFF093
:10B410004FB02420A51493F4D40F81E85824854715
:10B42000631DF7041C483149A1E3FD5723010400C3
:10B430001CB4230204021305C4002244B240924407
:10B4400002496146814541011753FB1F6700C3FA5A
:10B45000B38724033E95084509C59750FB1FE78035
:10B4600080D0850493F4F40F5C280848E3E2F4FEEE
:10B470009750FB1FE78020CF4DBF084C75F975B77B
:10B48000411122C4416406C626C29307E4FF63014A
:10B49000F502AA849DE19770FB1FE780A04609E9A9
:10B4A0001305F4FF9770FB1FE780C04511C106A18B
:10B4B000B240224492444101828085476392F50460
:10B4C0009770FB1FE78000442A847DD1FD571EA1A1
:10B4D0001C241307F00F6382E7021307E00F638950
:10B4E000E7003420083401475146A685EFF0AF94B9
:10B4F0002285EFF0FFF0FD571CA4230504004DBF8B
:10B500008947E397F5FA8545EF40004655F12685D2
:10B510009770FB1FE780003F2A845DF951BF21C56A
:10B52000011122CC06CE18259307F00F2A84630858
:10B53000F70234210E21083501475D46EFF0AF8F49
:10B540003820E1476318F7000A206C002306010049
:10B55000EFA00FA3F9571CA42285EFF07FEAF24079
:10B5600062440561828082809307F00F6306F706CC
:10B57000011122CC26CA2A844AC84EC652C4B689B2
:10B58000328A3A8993068500AE847946AA851705E2
:10B590000000130505F906CEEFF0EF96A304240191
:10B5A000230144012322340185C01305C4006244F1
:10B5B000F2404249B249224AA685D2446146056119
:10B5C0001753FB1F6700C3DCF2406244D244424978
:10B5D000B249224A0561828082809787FB1F2383BC
:10B5E000A76A8280411122C406C695472A846391C6
:10B5F000F50683474502854685072302F5021E228C
:10B6000058423022FD17B3C70708631ED602B3C7DE
:10B61000E72098239C330145A207D98F7A2463F051
:10B62000E7020A2085075EA49305C400EF907FEE31
:10B630000824B165938505B8EF803FA75945B2400E
:10B64000224441018280C946B387D702BA97D1B755
:10B650005822A9470545E314F7FE03454402133574
:10B660001500F1BF411122C406C69D472A84639686
:10B67000F5048347450285072302F5021E2258423E
:10B68000FD17B3C7E72098239C33A207D98F7A25EB
:10B69000014563F0E7020A2085075EA49305C40014
:10B6A000EFF04FCE0824B165938505B8EF80FF9F7A
:10B6B0005945B2402244410182805822A94705459C
:10B6C000E319F7FE0345440213351500DDB74111B8
:10B6D00022C426C206C6B5472A84B2846394F50400
:10B6E0008347450285072302F5020A21EF90DFB167
:10B6F0009E201307F5FF014563C1E7027A240A2063
:10B700009305C400BA977EA4EF909FEE0824B1651C
:10B71000938505B8EF807F995945B2402244924401
:10B720004101828058229D470545E318F7FE0345F5
:10B73000440213351500D5B7411122C406C6C547CA
:10B740002A846390F5061E223A22FD17B387E7028A
:10B750000347450205072302E5025842B3C707081D
:10B760003E973C333823A207D98F41677D176397F3
:10B77000E7000145B240224441018280138717004F
:10B780005AA57A25E3F7E7FE9305C5000A21EF9055
:10B790005FEF0824B165938505B8EF801F91594587
:10B7A000D1BF5822A9470545E316F7FC03454402DB
:10B7B00013351500C1B7011126CA4AC84EC656C274
:10B7C00006CE22CC52C4BC211547AA8A2E89B28942
:10B7D000B684639EE7023686CE854A85EFF09FE009
:10B7E0002A84631E05108547034599006393F91069
:10B7F000D820A9476319F70C054A83462900034559
:10B80000990001476946D685EFE0FFE2F9A8354780
:10B81000638CE7086361F7041D47638BE7062547E0
:10B82000638EE706A547638FF90A0544034599002F
:10B830002687CE860146D685EFE0FFDF054A19E56B
:10B84000CE852685EFE05FDA133A15005DD4D9473F
:10B850006306F40259A84547638EE7045D47E39306
:10B86000E7FCD82585473686CE854A85631AF704D6
:10B87000EFF02FC58547054AE306F5FAF24062442A
:10B88000D2444249B249924A5285224A0561828095
:10B890003686CE854A85EFF0FFDC99B73686CE85B1
:10B8A0004A85EFF01F952DBF3686CE854A85EFF08D
:10B8B0001FE23DB73686CE854A85EFF0FFE70DB72C
:10B8C000EFF0CFCC45BF268785460146D685EFE011
:10B8D0009FD6E31305F285452685EFE0FFD0133AA6
:10B8E000150021BF9E20B1F3054A4A85EFF05FB1F4
:10B8F00071B7A547E39CF9F29E208DFBF5BDA547E6
:10B90000E396F9F29E20E39307F2054A89B79E2158
:10B91000639F071C397126DA4ED652D406DE22DC2C
:10B920004AD8A021ED47AA89AE84328A6315F40271
:10B930001787FB1F034707359307F00F0144631F69
:10B94000F7049947F2506254D2544259B259225ADC
:10B950003E8521618280F5476311F4089786FB1FBD
:10B9600083C646321307F00F9947E38DE6FC9770C4
:10B97000FB1FE78020F92A8415C1302505C29317E3
:10B98000466063D40700814775BFF5454E85EFE0FB
:10B99000FFD23C2493E707F83CA4F5B7D6209044A7
:10B9A0008C3088203800EF90BFDEAA8741FDB4209C
:10B9B00038000146CE851785FB1F0345A52CEFE017
:10B9C0009FC7AA8741F1B24799C323000A00BC2050
:10B9D0007547E39AE7FA69F07DB79770FB1FE78038
:10B9E00060F22A894DD185476317F404CE2088443C
:10B9F0003000EF905F83AA8731F583472900154710
:10BA00006382E702E51793F7F70FC14663E1F60497
:10BA10003317F0281377574411E7639AD702832727
:10BA2000090195C7B0203400CA854E85EFF0BFD814
:10BA30002300AA0089BF38219147E31587F05841B8
:10BA4000E30207F0CE208844300002976DB703452B
:10BA500099009787FB1F83C7F7686381A702B4200B
:10BA600038000146CE85EFE01FBD2A8409E9AC20ED
:10BA70002800EFE07FB719C123000A000144034703
:10BA800029008D476318F7043C840357C90063F409
:10BA9000E7002316F9008355C9004E85EFE0BFF992
:10BAA0001787FB1F03578733ED4763F5E70283577B
:10BAB000C900DD4663F0F6029386370063D1E602E3
:10BAC00011669385470013060629B3C505084E8500
:10BAD000EF8040144A85EFF0BF92A287A5B51166AA
:10BAE0009305B00F13060629B355B70ACDB799478A
:10BAF0003E858280011106CE26CA4AC822CC4EC697
:10BB000052C49784FB1F9384E45D882493078002CA
:10BB100091653305F502938565701789FB1F13093D
:10BB20002916334505089740FB1FE780A05690244F
:10BB30009307800281453306F6022320A90097501F
:10BB4000FB1FE780608B832709004D459DCB014497
:10BB5000130A8002FD599C24636DF402170500004E
:10BB6000130525DBEFE0FFEB170500001305458308
:10BB7000EF900FDC170500001305C590EF30F0556E
:10BB80000145F2406244D2444249B249224A056129
:10BB90008280B307440303250900614681450504FB
:10BBA0001374F40F3E95231035012301050023146F
:10BBB0003501230505002302050231059750FB1FBF
:10BBC000E780808349BF014582801787FB1F0347B9
:10BBD000F751814763E4E700014582809221938613
:10BBE00045006314A6002E8582808507B685DDB7E3
:10BBF0001DC5411122C406C638219307D00F2A84DF
:10BC000063EBE7000E2128310147F9465D46EFE07E
:10BC10009FA2F9573EA0B240224441018280828017
:10BC20001787FB1F0347974C8147FD5663E3E700E7
:10BC3000828016A12301050085071105C5BF0145B6
:10BC400082809785FB1F9385F5F293070002854656
:10BC50009CA1FD571787FB1F230EF7F01787FB1FCB
:10BC6000A309F7F01787FB1F2305F7F09787FB1F42
:10BC70002390D7F09787FB1F239407029787FB1F1A
:10BC800023AE07009787FB1F23A807009787FB1F9A
:10BC900023A207001786FB1F130606ED9787FB1FDD
:10BCA000938747F25CC29787FB1FA38D07FC97879A
:10BCB000FB1F9387A7E5094718A298A398AB238099
:10BCC000E7022388E7021787FB1F130767EE94A795
:10BCD000D0C794AFD8DB1785FB1F130565EE0D4762
:10BCE0001786FB1F130606ED9786FB1F938606EA51
:10BCF000238CE702C8C323950700D0CB239D070000
:10BD0000CCCFD4D3238407022395070223A60702AE
:10BD1000239D07021787FB1F032707F7D8DF9787A5
:10BD2000FB1F9387E7DD170700001307870B23A08E
:10BD30000700D8C323A407008280411106C6EFF094
:10BD4000DFE809C52821B240410182800145E5BFF5
:10BD5000411122C426C24AC006C6AA842E89328452
:10BD6000EFF0BFE6AA8711E94165CA857D15EFF0BE
:10BD7000DFE5AA87454581C786A3A0A30145B24058
:10BD80002244924402494101828021E30948354717
:10BD9000639E0603011106CE22CC18221032220621
:10BDA000598E32C6B377F64085E7CC452A842EC437
:10BDB000EFF0BFF832460147630EC50022856244AA
:10BDC000A245F24005616FF0BFF82D473A858280A9
:10BDD00013070008F24062443A850561828083C8F7
:10BDE0000500094863910803DC4103C807009C3340
:10BDF000A207B3E707010D681308289063950701B0
:10BE000089476FF09FF80545828001114EC606CE26
:10BE100022CC26CA4AC89789FB1F938999D503C7A4
:10BE200009009307F00F630FF7022A892945AE84B2
:10BE300032849740FB1FE780A045AA8505C593077C
:10BE4000100B1EA12302050002A562442311250147
:10BE500066A1F24003C50900D2444249B2490561D6
:10BE60006F80AF88F2406244D2444249B2490561D2
:10BE70008280411126C2AE849785FB1F83A5C5E051
:10BE800022C406C62A84EFF05FEB098909C922851E
:10BE90002244B240A685924441016FF08F8FB24098
:10BEA00022449244054541018280411122C426C2A8
:10BEB0004AC006C6AA84130445001309850B1E2038
:10BEC0009DC3084409C59740FB1FE780C029228510
:10BED000314681459740FB1FE78000523104231A09
:10BEE00004FEE31E24FDB2402244FD579EA00249F9
:10BEF0009244410182809786FB1F83C6361F978735
:10BF0000FB1F83A7E7D801476394E60001458280C1
:10BF10008E231386870B6394A5003E8582800507D8
:10BF20001377F70FB287CDB7AA871785FB1F0325B5
:10BF3000A5D601C95A216314F7000845828008413B
:10BF4000CDBF8280411106C6EFF01FFE09C508452E
:10BF5000B240410182800145E5BF797122D413844A
:10BF6000450026D24AD052CC5AC82E8A06D64ECE8A
:10BF700056CA5EC622892287014B81448146814789
:10BF8000BD45122345CAB5EE46233E23B286A69789
:10BF9000B3C70708050B3107E315BBFEADC49165B8
:10BFA0009385457026859740FB1FE780A00EAA8BDE
:10BFB00039C90C44D1C9814A8149522033853B019A
:10BFC0009740FB1FE780C03C5E200844BE99B3C980
:10BFD00009089740FB1FE780001963980A003109A0
:10BFE000854A832589004A84E9F9314681452285BD
:10BFF000850A9740FB1FE780204063826A0531096C
:10C00000CDB7630ED6000145B25022549254025966
:10C01000F249624AD24A424BB24B45618280322396
:10C02000E313F6FE5223B294B297B3C40408B3C725
:10C0300007088DB78547E3E367F70545F1B7232682
:10C040007A0123149A00D5BF1309C400854A814997
:10C0500049BFAA871785FB1F0325C5C311E182804D
:10C0600018453A276314F700110582800841FDB78F
:10C07000411106C6EFF0FFFD09C50A21B24041019A
:10C0800082800145E5BF411106C6EFF09FFC09C55E
:10C090002821B240410182804145E5BF4111178608
:10C0A000FB1F130626BF22C40042AA8606C62E85A1
:10C0B00001471DCC1C44AE271C406396D5021DC70A
:10C0C0001CC301C92146930544009740FB1FE7802C
:10C0D000202C22859740FB1FE780E0080145B240F5
:10C0E00022444101828022873E84E1B71CC2D1BF35
:10C0F0000545F5B701119786FB1F9386E6B926CA59
:10C10000AA84884222CC06CE2E8401470DCD52212E
:10C110001C416315960215C71CC39740FB1FE7809F
:10C1200080042C002685EFF07FF701E519C0B247A7
:10C130001CC0F2406244D244056182802A873E8559
:10C14000F1B79CC2D9BF0545EDB7411122C42A847D
:10C15000090506C6EFE0EFDBFD573CB0B2402244D4
:10C1600041018280411122C4416406C626C2930760
:10C17000E4FF6301F502AA849DE19760FB1FE7805D
:10C18000807B09E91305F4FF9760FB1FE780A07A25
:10C1900011C106A1B24022449244410182808547E8
:10C1A0006392F5049760FB1FE780E0782A847DD1D5
:10C1B000FD571EA13C201307F00F6382E70213070F
:10C1C000E00F6389E70028300147F9465146A6850C
:10C1D000EFE06FC62285EFF05FF7FD573CA023022A
:10C1E00004004DBF8947E397F5FA8545EF30C077E6
:10C1F00055F126859760FB1FE780E0732A845DF97F
:10C2000051BF5D71A2C4CAC086C6A6C24EDE52DC52
:10C2100056DA5AD82E84AC21F9472A896392F5045C
:10C220009760FB1FE78020712A8405C1382193079E
:10C23000D00F63ECE70028310147F9460146CA8573
:10C24000EFE06FBF2285EFF05FF00145B640264476
:10C2500096440649F259625AD25A425B6161828021
:10C26000832A0400B7070001938707F037071200FD
:10C27000B3F7FA0013070710B28981446388E70215
:10C280002EC69760FB1FE780006BB245AA8419CDCC
:10C29000502109CE93174660E3C907FA4A85EFE0BB
:10C2A000EFC1DC2093E707F8DCA045B7178AFB1F36
:10C2B000130A4A8C03470A009307F00F1945E30756
:10C2C000F7F8E147E3E4B7F893D71500FD17171720
:10C2D00002001307E777B3E7E72003A80700E307A7
:10C2E00008F603AB4700E3030BF6B3CA0A086385FD
:10C2F0000A00C947E39CF5F4562010440C3008208E
:10C300003808029821F52C084A85029B1DCD18306B
:10C3100015FF3820230AA100B9472308E100631460
:10C32000F702E24798239C33A207D98F0C084A856D
:10C33000FC81EF90CF8311D914080546D9454A8571
:10C34000EFE0AFDA21B7BC84D5B734209147E38E54
:10C35000F6EE03450A0038080146CA85EFE0AFADA6
:10C36000E31605EE2C202808EFE00FA819C1238062
:10C3700009001840B7070001938707F07D8FB707C2
:10C38000120093870710E302F7ECE38004EC3C20F3
:10C3900021BF411122C406C62E849760FB1FE7808F
:10C3A000805909C95C21138717006315E40093F7CE
:10C3B00007F85CA1B240224441018280397152D415
:10C3C0002E8A4ED69305E100AA89528522DC4AD8EE
:10C3D00056D25AD05ECE06DE26DA3289368BBA8B3A
:10C3E000BE8A9760FB1FE7808057054425C1AA8459
:10C3F00028873944EFF05FB331C90328450063074C
:10C400000804D6875E87DA864A86A6854E85029816
:10C410002A840DED9307E00F638AFA02982089477A
:10C420006316F702DC4098239C33A207D98F0D676F
:10C4300013072790639CE700834719000346090010
:10C44000D285A2075D8E4E85EFF03F9CF25022858B
:10C450006254D2544259B259225A925A025BF24B58
:10C4600021618280797122D422214ECEAA8922852F
:10C4700056CA06D626D24AD052CC5AC85EC662C424
:10C48000AE8AEFF05FA705E52285EF90CFF659441D
:10C4900011E10144B2502285225492540259F249CA
:10C4A000624AD24A424BB24B224C4561828003C75A
:10C4B000890085476307F700EFF03F9F03D5290008
:10C4C000E9B7AA85AA8413858900EFF01FA92A84F9
:10C4D00015CDFA209624D044CE2003D52900E1477B
:10C4E000EFF0DFEDD9472A846318F50023A6040096
:10C4F0002685EFF09F9B71BF19E1268575BFDE2071
:10C5000026852390FA00EFF05F9A69B713894400FB
:10C51000014AB94B594C3D4B8355090085CDE14744
:10C5200063077A010357C900D94711E3E14703576D
:10C530002900835649000326890003D52900EFF01E
:10C54000FFE72A846310850323240900050A3109C3
:10C55000E3146AFD2685EFF05F952DD0D947E31BE4
:10C56000F4F205BF65D5835709002390FA00F9BF9F
:10C57000011170879307E00F1306E1000147894618
:10C5800006CEEFF0BFE3F2400561828079714AD0B8
:10C590000359850022D426D22A84AE844A85930585
:10C5A000210106D69760FB1FE780603B79C51C25FB
:10C5B0002AC693F707029DC7A881EFF0BF98B2453E
:10C5C000AA8711E9239024013945B250225492548C
:10C5D0000259456182802A204946829701C51E245E
:10C5E0009EA0E5B7035924004A85EFF0DF9001EDE6
:10C5F00041657D15EFF03F9009E51E2425459EA07D
:10C60000E9B723102501130745008147BD461223D2
:10C6100039EE3147B387E7029305840031462EC6D1
:10C6200091073E959740FB1FE78080D6B245314683
:10C6300048089740FB1FE780A0D552242A20414795
:10C640008146DD45EFE0CFC42ACE09E51E244545ED
:10C650009EA0A5BF0C4852249740FB1FE78040D303
:10C660002A204C08EF90EFD42DD15945B9BF85074A
:10C670003107E39ED7F825459DB705458DB77971FC
:10C6800022D42A840A254AD02E899305E1004ECE71
:10C6900006D626D2B2899760FB1FE780402C2DC9B1
:10C6A0001C25AA8493F707028DEF183893072005FD
:10C6B00011E35C20362450440E242A200147EFF079
:10C6C000FFCF21E11C38B9E32A20EF90CFCAAA8717
:10C6D00059458DCFB250225492540259F2494561C6
:10C6E00082802887EFF01F86AA870DC52A20494639
:10C6F000A68582975DD91E242310F9001C3899E77E
:10C70000D1BFD947E319F5FE238009000145D9B708
:10C710000545D5B73945C5B7797122D44AD04ECE33
:10C7200052CC56CA06D626D2AA892E8AB28A368911
:10C730009760FB1FE780202009440DC53C211307AB
:10C74000E00FAA845D44638FE7001307F00F59449C
:10C75000639AE70063920A02D2854E85EF90AFCDCF
:10C760002A8421C1B2502285225492540259F2499E
:10C77000624AD24A4561828003550A009305E1006E
:10C78000231701009760FB1FE780601D2887EFF0EB
:10C790009F8FAA8505464E85EF20507C2A844DDD6B
:10C7A000D1B79307F00FE30FF9FA93862400794687
:10C7B000A68517F5FFFF1305E543EFD0DFF4A3814E
:10C7C00024014DB7797126D24ECE52CC56CA5AC8E2
:10C7D0005EC606D622D44AD062C466C2AA8A2E8B0E
:10C7E000B28B368ABA899774FB1F83A4A44AB9C056
:10C7F000804483DC44000149035CA4006314990174
:10C800008440F5B73E2463F75701050941043349D5
:10C810000908EDB7E36BFBFE63090A000C204840F2
:10C82000D2865E86EF809F896DD163840900239054
:10C830008901A284B25022540259F249624AD24A72
:10C84000424BB24B224C924C2685925445618280D9
:10C850009A21B621854763E3E60429C3D421011157
:10C860001386550022CC1775FB1F130565352E84E2
:10C87000894506CE32C6EF807F84C14719C954204E
:10C8800032462E200A200147EFF0DFF3A94711C1FD
:10C890008147F24062443E85056182803E85828008
:10C8A0002E860A22AE21854763E1A50219CD5422C6
:10C8B00041110147150606C6EFF0DFF0A94711C187
:10C8C0008147B2403E85410182803E8582802E862E
:10C8D0000A22AE21854763E1A50219CD54224111F8
:10C8E0000147150606C6EFF0FFEDA94711C18147C4
:10C8F000B2403E85410182803E85828039714ED6AC
:10C90000BE2183D9050006DE22DC26DA4AD852D4BD
:10C9100056D25AD05ECE62CC66CA63E437152A8AF4
:10C92000054563830912416BAE8A2314010002C6D8
:10C93000014401497D1B894B054CC94C83D52A0014
:10C940000147814601464E8523130100EFF09FE722
:10C95000AA8471C509EC13072002930661005A8668
:10C9600095455285EFE0CF922A84630E050E3884F8
:10C970009C2025C718856301870541476394E70A12
:10C98000BE244146130524001CA0BE24A1831CB074
:10C99000CC409740FB1FE780A09F49043C8485075B
:10C9A000B3C707087C8463FC2707BE246389670735
:10C9B0008509B3C9090859B763967707BE240946A4
:10C9C000130524001CA0BE24A1831CB0CC409740BA
:10C9D000FB1FE780E09B1104D1B722C60359610019
:10C9E000B82413052400638F770133599903230575
:10C9F000710118A0BE244146A1831CB0CC4013791C
:10CA0000F90F41BF2305810118A0BE241359290045
:10CA10001379F90FA1831CB0CC4009464DBF3C846B
:10CA200029459DC32C005285EF807FE809CD340055
:10CA30001546D9455285EFD05FEB11C53245973089
:10CA4000FB1FE78040720145F2506254D2544259B4
:10CA5000B259225A925A025BF24B624CD24C21617B
:10CA600082800545D5B74545C5B71777FB1F0347F6
:10CA7000E724854763F7E706011122CC26CA4AC896
:10CA800006CE2A84AE8432899760FB1FE780A0EA35
:10CA900011C538219307E00F6307F704631B0900F2
:10CAA00022856244F2404249A685D24405616F90D6
:10CAB0004F958A209305E100231701009760FB1F23
:10CAC000E780E0E92887EFF00FDCAA85054622859C
:10CAD000EF20D04871D5F2406244D244424905610A
:10CAE0008280594582805D45FDB7411122C406C64A
:10CAF00026C293F705022A84328585C3EFF0AFD8AA
:10CB0000AA8505462285EF20704595476305F50007
:10CB1000BD476315F502214515A093F78500B6843E
:10CB20009DC3EFF04FD6AA8505462285EF2010431E
:10CB300009C59C3481C79C2491C30145B24022445D
:10CB40009244410182809397456063D70700EFF0DC
:10CB50008FD3AA850146D1BF89890D45F9FDF9BF5B
:10CB60007971AE8622D42A848A229305E10106D601
:10CB700036C69760FB1FE78080DE11C90C25228531
:10CB80002254B246B087B25045616FF01FF6B250E2
:10CB90002254054545618280411122C406C693F79F
:10CBA00005022A8432858DC3EFF0EFCDAA850546B4
:10CBB0002285EF20B03A1547AA876305E5003D4777
:10CBC000631DE502A14715A893F7850099CBEFF007
:10CBD0008FCBAA85054622852244B24041016F20B1
:10CBE000F0371397456063570700EFF0CFC9AA8568
:10CBF0000146D5B7898991E18D47B24022443E85EF
:10CC0000410182807971AE8622D42A848A229305DA
:10CC1000E10136C606D69760FB1FE78040D4B246D6
:10CC200009C90C2522852254B087B25045616FF0A6
:10CC3000BFF6B25022540545456182803E25797188
:10CC4000416722D426D24AD04ECE06D62317010001
:10CC50007D17AA84328436898149638DE700942048
:10CC6000D040138517001307E10033450508EFF0A6
:10CC70007FB5AA899420D04089451775FB1F1305FD
:10CC800025F4EF80AFC315C5A2242285EFF04FBE77
:10CC900009C57D142A943344040863040900231051
:10CCA0008900B2502254925402594E85F24945618E
:10CCB00082809420D04089451775FB1F130505F02D
:10CCC000EF80CFBF71F19420D04089451775FB1FCD
:10CCD000130545EEEF808FBE11C9E38809FA3C8742
:10CCE000E39587FA03D4A9007D1475B7A22475B71C
:10CCF000397122DC26DA4AD84ED652D456D25AD0CE
:10CD00005ECE06DEBE8B9C252A8AAE84C18BB28A9B
:10CD100036843A89C289468B9DEF94208947638384
:10CD2000F6065685EFF04FA005CD832805006389F0
:10CD3000080222866254F250925A5A88CE87025BC9
:10CD4000B2595E87CA86F24B4259A6855285D254A3
:10CD5000225A216182883285EFF0CF9EAA8709EDA1
:10CD60003945F2506254D2544259B259225A925A19
:10CD7000025BF24B216182802946A685528582970B
:10CD800049DDC5B7DC4003C3170098238D67220334
:10CD90003363E3001386479013175360E343E6F8C9
:10CDA0001386F78F634BE60293862780630FD708BD
:10CDB00063C8E604F977938707803E93854733433A
:10CDC0000308E3E067F62D45E39D0BF8DC44902370
:10CDD000CC432310C90022851DA2F5779387F76FF6
:10CDE0003E938D473343030863E067121717020031
:10CDF000130747C03343E32083270300BA97828792
:10CE000093873780E31FF7F02D45E39C0BF48547AC
:10CE10002310F900DC4481459C231CA0AA240505AD
:10CE2000334505089760FB1FE78060B3835709000F
:10CE30004DE991072310F9001146814513051400AF
:10CE40009730FB1FE780405B41A82D45E39B0BF02B
:10CE5000DC446C0083C917009823A209B3E9E900F8
:10CE600011472310E9009C234E851CA0DC449C3311
:10CE70001CB09760FB1FE78080AEAA8425C1308676
:10CE8000C1659306E100FD158329C500EFF01FDBA6
:10CE900009ED9420D04089451775FB1F130505D275
:10CEA000EF80CFA119E1FD577C8703C709008947AF
:10CEB0006310F70283A54900094613054400973023
:10CEC000FB1FE780E04C8357090089072310F90016
:10CED0003C873CA0A1833CB0014561B523173101DB
:10CEE000C5BF18218907BA972310F9003E251CB049
:10CEF0003E25A1833CA010214C41130534009730FE
:10CF0000FB1FE780E048C9BF2D45E39C0BE42310DD
:10CF1000D900DC449C231CA0DC449C331CB06DBFB6
:10CF2000C8449730FB1FE7802051334705081D4553
:10CF3000E36977E36380EB02B386790163C6E600B9
:10CF400033077741B3490708CC44231039014E8693
:10CF5000DE9551B58149CDBF2D45E3940BE0CC441E
:10CF60005285EFE09FDD89472310F90008A0218159
:10CF700008B09DB72D45E3960BDE89472310F900D5
:10CF800049BF2D45E39F0BDCDC441D472310E9001E
:10CF9000982318A0983318B0BA2338A0BA23218355
:10CFA00038B0D82358A0FA2358B0FE23A1837CA020
:10CFB00025B75D71A6C2AA842A214EDE52DC56DA5C
:10CFC0005AD85ED662D466D26AD06ECE86C6A2C465
:10CFD000CAC0AE8AC16BEF802FA3130CF5FF2A8A5B
:10CFE0008149977DFB1F938DED06977CFB1F938CEA
:10CFF000ECCA177BFB1F130BABCAFD1B334D0C0890
:10D00000DE2463F6F90083D70D0063CD8701AA20E3
:10D010009775FB1F93850504EF801FAB2A841DCDF8
:10D0200059442DA89C449305E100B3A7F92003C9F6
:10D0300017009C2322093369F9004A859760FB1F7A
:10D04000E780E091AA851DE923902A0103A54D0000
:10D0500009C59730FB1FE78000110544B6402285C3
:10D06000264496440649F259625AD25A425BB25B50
:10D07000225C925C025DF24D6161828083C8440053
:10D0800083A60C003087AA206A8881475A87EFF070
:10D090003FC62A8419C923902A0103A54D005DDDEE
:10D0A0009730FB1FE780200C55BF83A74D0099EFF9
:10D0B000AA20514781465E86BD45EFD07F9D23A2C1
:10D0C000AD0009E523902A01454449BF83D70D00EF
:10D0D00003570B003E97634747013307FA407D171C
:10D0E0002310EB0003A54D0003560B0083A50C0095
:10D0F0003E9585099730FB1FE780802983D70D0077
:10D1000003570B00B3C90908BA972390FD00CDBDA2
:10D11000397126DAAA842A214ED65AD006DE22DCBC
:10D120004AD852D456D25ECE62CC66CA6AC82E8B1A
:10D13000EF808F8DAA89D424AE248A2478001386A8
:10D14000D400EFF02FE805C5938BB9FF2A84E519C9
:10D150000149177CFB1F130C6CB4977CFB1F938C4D
:10D160002CB433CA090863497901631B09109E2452
:10D1700029452310FB009DA8035DC10083C844001E
:10D1800083260C00AA205288814766876A86A2857A
:10D19000EFF01FB619C9AE2422859306E1006A8616
:10D1A000EFF0DFA92A8461F0C9B783D70C00922879
:10D1B000E313F6FE83250C00C8489730FB1FE78079
:10D1C000A02F71D99779FB1F9389C9E883A74900DC
:10D1D00095EFAA204166454781467D169D45EFD0D3
:10D1E0003F8B1DE19E2445452310FB00F250625405
:10D1F000D2544259B259225A925A025BF24B624CB3
:10D20000D24C424D2161828023A2A900AE24835AD0
:10D21000A40022859306E1006A86EFF03FA22A84EB
:10D22000E3830AF883A74900130719003347070867
:10D23000CA972380570183A7490093DA8A0093068F
:10D240002900BA972380570113073900110983A7D2
:10D250004900B3C60608334707083349090811C90E
:10D260003087B69790A383A749002182BA9790A3ED
:10D27000DDBDB697FD5694A383A74900BA9794A342
:10D28000AA209775FB1F9385E5DC1359290023908D
:10D290002501EF802FED39D9594589BF411122C4AD
:10D2A00006C693F705012A84328585C3EFE0BFDD0A
:10D2B000AA8505462285EF20604A95476305F5005B
:10D2C000BD47631DF502214515A893F7450099CB8D
:10D2D000EFE07FDBAA85054622852244B24041016A
:10D2E0006F20C04793F7050491C7EFE0DFD9AA8507
:10D2F0000146DDB713C5F5FF05890605B240224496
:10D3000041018280797122D426D252CC06D64AD0ED
:10D310004ECE56CA5AC82A8AAE840144DE206364BF
:10D32000F400014581A083AA040093191400138915
:10D330001900B327542103CB0700B3872A018823A0
:10D340009305E1002205336565019750FB1FE780D7
:10D3500000611DE123806A019C4005453E99034719
:10D36000090098B3B250225492540259F249624AC9
:10D37000D24A424B456182800C2530875285EFF0BE
:10D38000FFF101CD9C40BE9903C7090098A39C40C2
:10D390003E990347090098B3F1B7050433440408E4
:10D3A000B5BF0111AE8722CC2A848A239305E10000
:10D3B00006CE9750FB1FE780805A09C90C252285AD
:10D3C00062443087F24005616FF05FEDF2406244E5
:10D3D00005450561828039715AD02A8B2A2126DAC7
:10D3E0004AD806DE22DC4ED652D456D25ECE62CC6D
:10D3F00066CAAE84EF705FE12A898346CB0083550D
:10D40000AB0003558B0078001306DB00EFF08FBBF9
:10D4100063050516C16A130AA9FFAA8B014497790F
:10D42000FB1F9389A987977CFB1F938CACC2FD1AC5
:10D430006D19334A0A08035CC10083C58B0003558C
:10D440002B006286EFF09FE56318051483484B00BC
:10D4500083A6090003552B00528881471777FB1FCD
:10D46000130707846286DE85EFF09F886316051236
:10D4700005CC83D72C001777FB1F03576782110752
:10D480006395E700A29763C427079775FB1F9385F1
:10D4900065BCBE2103552B003354F40282A1EF80FA
:10D4A0006FE615C1594505A003552B004947814634
:10D4B0005686C545EFD0CFDD23A2AC0015E183D75A
:10D4C000AB0045459EA0F2506254D2544259B25925
:10D4D000225A925A025BF24B624CD24C21618280FA
:10D4E0009767FB1F83D7C77B91072391FC0083A716
:10D4F0004C0003D7AB006286A29798A383A74C0089
:10D500001307140033470708BA9703D7AB009306F5
:10D51000E1005E85218398A38355AB00176CFB1F48
:10D52000130C0C78EFF08FF103A74C003C87130627
:10D5300024003346060832971CA303A74C00930629
:10D540003400A183B3C6060836971CA3AA8B03A593
:10D550004C0011043344040803560C0083A5090051
:10D56000229563910B029730FB1FE78060E283579F
:10D570000C00A29733C4070809F883578B0029458C
:10D580009EA091B79730FB1FE78080E083570C0087
:10D590003E943344040845B583D7AB009EA0E31600
:10D5A00004EE83578B009EA039BF1D71A6CACAC85E
:10D5B000AA84035985002A21A2CCCEC6D2C4D6C2E1
:10D5C000DAC05EDE62DC6AD886CE66DA6ED6AE8AF5
:10D5D000EF709FC3130BD5FF01447115138CD4005A
:10D5E000976BFB1F938B8B6B176AFB1F130A4A6B9E
:10D5F000177DFB1F130D0DA6B3490508635D64116C
:10D60000D424AE241307E10162864A85EFF08F9B94
:10D61000AA8C630205100359A500B0870C25AA2027
:10D6200032C6EFF0BFC7631D050E83C8440083A652
:10D630000B003246AA204E8881475287E685EFF0DC
:10D640002FEB79ED15C483570A0003572D00890786
:10D650006302F7069775FB1F9385C59FBE21AA201D
:10D66000B357F4029EA1EF806FB80DC1594539A898
:10D67000AA2041664D4781467D16A545EFD04FC192
:10D680002322AD001DE123902A014545F640664462
:10D69000D6444649B649264A964A064BF25B625C36
:10D6A000D25C425DB25D2561828083570A008907A2
:10D6B0002311FD0083570A00A29763DE67058327C5
:10D6C0004D0003D7AC00930D2400A29798A38327A5
:10D6D0004D0003D7AC000504334404082183A2970E
:10D6E00098A303254D0003560A0083A50B00B3CD74
:10D6F0000D086E959730FB1FE78080C983570A009D
:10D70000BE9DC167FD1733C40D08E309F9EE050995
:10D7100033490908E5B5294515FC23902A01BDB711
:10D720006DDC0DBF1E21411126C206C622C44AC0AF
:10D73000444189EB8947B2402244924402493E85E4
:10D74000410182809420D0402A8489451765FB1FBF
:10D7500013050547EF709F9611C93C202547E51733
:10D7600093F7F70F637FF700E147F1B79420D040BC
:10D7700089451765FB1F13056544EF703F9471FDE4
:10D7800055BF1769FB1F1309A93E8356090085473A
:10D79000DDD21A203697C166E3CFE6F8916593850E
:10D7A000257031459730FB1FE780C08EAA84CD4796
:10D7B00059D1314681459730FB1FE780E0C31A20DD
:10D7C0008355090001468147B386F500B3C60608B4
:10D7D00063E9E70201C62E972310E90023A00400A5
:10D7E0002146A285138544009730FB1FE78040BA8D
:10D7F0001767FB1F1307074A1C4381CF3E879C43D3
:10D80000EDBF50401395470085072A9636A605467A
:10D8100065BF04C3814705B7011106CE22CC26CAD5
:10D820004AC809E90944F24022856244D244424987
:10D83000056182802AC6AA84280036896C845085B6
:10D84000EFF05FEE2A8465F1E30F09FCBE24F9DBFB
:10D8500091659385557031459730FB1FE780808334
:10D86000AA8715C1BA249766FB1F9386E642232038
:10D8700005005AA198422324250101C7BA861843FE
:10D88000EDBF9CC24DB74D4479BF9767FB1F93878F
:10D89000773F98230DE3054798A3058909CD97663F
:10D8A000FB1F9386E625414691451765FB1F13052F
:10D8B000E5256FF07FF6014582809767FB1FA38AFD
:10D8C000A72A828041677D176315E5002E856FE0EA
:10D8D0002FB5411106C6EFE04FAF09C5FD571EA198
:10D8E00023010500B24041018280011126CA06CE03
:10D8F00022CC4AC88547AA846392F5042685EFE0C6
:10D900008FDF31E941699305F9FF1307E10089468B
:10D910001766FB1F1306C6290545EFE0BFEA2A84F8
:10D920007D1905C44C442685EFF0DFF93087228548
:10D930008146CA85EFF08FB02A84E5B789476396A0
:10D94000F5008545EF20400255D9F2406244D244AB
:10D95000424905618280EFE04FD56DB7411122C485
:10D9600006C626C21764FB1F1304C47708349767E2
:10D97000FB1F23AF07309767FB1F23A9073097676B
:10D98000FB1F23A3073059C59307200C3305F5026D
:10D990009165938515709764FB1F9384642F190517
:10D9A000334505089720FB1FE780C06E10349307AE
:10D9B000200C81453306F60288C019069730FB1FFC
:10D9C000E78080A39C4018348145938647007D55AD
:10D9D00063EAE5069306800BB306D7020146050706
:10D9E000FD55B6979766FB1F23A2F62ABE868EA228
:10D9F000ACB2ACA22382060005069906E369E6FEF6
:10DA0000F95696A399463307D702BA971767FB1FB3
:10DA1000232CF72617E5FFFF1305E57EEFD00F81D6
:10DA200017F5FFFF13052597EF702FF117E5FFFF9F
:10DA300013058573EF10706AB24022449244014589
:10DA400041018280239EA6FE36861388460B231052
:10DA50000600232406003106E31B06FF8505938696
:10DA6000860BBDB7411106C622C42A84EFC0CFA2DF
:10DA7000EFE02F9D1765FB1F032505219767FB1F0F
:10DA80002389870EEFE0CF999767FB1F2384870ECA
:10DA90002244B24017050000130565E541016F10EF
:10DAA000D0639397556063DB072E79711765FB1F71
:10DAB0000345250C22D44AD006D626D24ECE2E8936
:10DAC0009730FB1FE780C0822A8441CD182193073D
:10DAD000000B6315F70885479764FB1F9384041CAC
:10DAE000DC849C402315010081EFEF00C075916537
:10DAF000938535709720FB1FE780C05988C031C9D6
:10DB0000614681451765FB1F1305C5549730FB1F00
:10DB1000E780808E8349440089476393F90825276D
:10DB20009764FB1F938404538AA02A20A685EF7074
:10DB30007FD4AA869E202A201A248DEE6363F700E4
:10DB40001EA40E24EFC03FEF2285EFC01FC49C84AB
:10DB500091C74C2013058400EFD04FCC2285EF6095
:10DB6000AFB3B25022549254F2491315F9680259D6
:10DB7000456182806363F7001EA41E24D945976621
:10DB8000FB1F9386264D0D469EA0EFC01FD68D45E8
:10DB900045DD1765FB1F1305E54BEFD02FC86DB7AB
:10DBA0009387A9FF93F7F70F4947E36FF7F8170734
:10DBB0000200130727E5B3C7E7209C43BA97828783
:10DBC0009305A1002285EFF0AFD4AA8435DDD947B3
:10DBD0006394F40A85092A2093F9F90F9766FB1FCD
:10DBE000938646474E86D945EFC03FD031DDCE857E
:10DBF0004DB79305A1002285EFF03F9BF9B78359FC
:10DC000084006C004E859750FB1FE78040D5AA84A6
:10DC10002DC12A2041669306E10055477D16AD458A
:10DC2000EFC01FE79769FB1F9389C94223A2A90090
:10DC3000AA8655CD834844000358E10030862A2047
:10DC4000A68581474E87EFF0AF8AAA846312050E3E
:10DC50002A20CE85EF703FDFE30805EE2A20D94564
:10DC6000CE862D46EFC07FC8AD45E30F05EC4E854F
:10DC70002DB72315310185441830D147E306F7EC61
:10DC80005C209769FB1F9389E93C2A202380F900D7
:10DC90003C85CE85238299002391F900EF702FED0A
:10DCA000E30405EA2A20CE860546D945EFC0FFC326
:10DCB000E30C05E8854565BF835984006C004E85FB
:10DCC0009750FB1FE780A0C9AA8445D52A2041664A
:10DCD0009306E10059477D16B545EFC07FDB976994
:10DCE000FB1F9389293723A2A900AA8609E51E24D0
:10DCF000C5447C8551B7834844000358E1003E2465
:10DD000030862A20A6854E87EFE09FFEAA840DE18B
:10DD10002A20CE85EF709FD6E30805E22A20D94558
:10DD2000CE863546EFC07FBCB545E30F05E081B731
:10DD3000D94703A549006397F4009720FB1FE780AC
:10DD4000804219B59720FB1FE780E0411E247C85A7
:10DD500025B79305A1002285EFF0AFA5BDB59305CA
:10DD6000A1002285EFF02FE78DB5130691009305F2
:10DD7000A1002285EFE0BF9089BD9305A100228517
:10DD8000EFE0DF80AA84E31405E4A30401006DBB87
:10DD90009305A1002285EFE0EFEC05BD01458280EF
:10DDA000F1CE011156C2AE8A854526CA4EC652C46E
:10DDB00006CE22CC4AC82A8AB284B689EF10D03A5D
:10DDC000D1471DC51767FB1F034757EF9767FB1F19
:10DDD00083C797EE014999E03E89BA871317490036
:10DDE0001764FB1F032484EC3A94636DF900D54754
:10DDF000F2406244D2444249B249224A924A3E85A4
:10DE00000561828036201307040191C60509137944
:10DE1000F90F3A84D9BFB1C89565938525C013051C
:10DE200000029720FB1FE780E02648C469D1130653
:10DE300000028145130909049720FB1FE780C05B9E
:10DE40002300040023112401231344019C34176789
:10DE5000FB1F0327E7E5998C1CA45C449184918007
:10DE6000C4AF23A08900814761B7232604002300A3
:10DE700004002313440123045401E5B785473E857C
:10DE80008280AA869765FB1F83C555E31767FB1F32
:10DE90000327C7E181476394F5000145828032235F
:10DEA0003A8519C2E30CD6FE850793F7F70F4107B1
:10DEB000DDB7AA861766FB1F034656E01767FB1FF0
:10DEC0000327C7DE81476314F600014582802E23B5
:10DED0003A8581C54C23E38BD5FE850793F7F70F71
:10DEE0004107D5B7AA869765FB1F83C505DD176770
:10DEF000FB1F0327E7DB81476394F5000145828020
:10DF000012233A8519C2E30CD6FE850793F7F70F63
:10DF10004107DDB7AA861768FB1F0348F8D9976742
:10DF2000FB1F83A7A7D801476314E800014582803F
:10DF3000B2233E8509CAF2236317D600D04701C633
:10DF40003222E306B6FE05071377F70FC107E9BFD4
:10DF5000411126C2444522C406C62A8495C0C8443D
:10DF600009C59720FB1FE7800020C84809C59720F6
:10DF7000FB1FE780401F26859720FB1FE780A01E20
:10DF80002285414681459720FB1FE780E046FD57EB
:10DF90001CB4B2402244924441018280011122CC3F
:10DFA0002A842A2106CE2EC6EF10606832462285CA
:10DFB0008145EF00905722856244F24005616FF081
:10DFC0003FF905C53E21411122C406C62A8491CBE2
:10DFD000DD45EF00905822852244B24041016FF0A8
:10DFE0003FF7B2402244410182808280411122C425
:10DFF000B1471304C5FFB307F40226C29764FB1FA1
:10E000009384C40606C6A697BA276315B702C84309
:10E0100015C19307F00F6305F6001C21639CC70030
:10E020009720FB1FE7802014B1473304F402A29429
:10E0300023A20400B2402244924441018280411153
:10E0400022C42E8426C24946AA848145228506C65A
:10E050009720FB1FE780403A8DCCD82C9767FB1F99
:10E0600083A707C51207BA979A231AA0BA23FE23DB
:10E070003AA01767FB1F0357E7C35AA09A207AA05C
:10E08000BA201AA4DA203AA4FA205AA49A241EA884
:10E090007AA4B24022449244410182802A86976544
:10E0A000FB1F83C5B5C11768FB1F032868C09766AF
:10E0B000FB1F83A6A6BF014701456393E50082804D
:10E0C0009C2281CFDC4691CBDC2F9207C29763164E
:10E0D000F6009307150013F5F70F05071377F70FF1
:10E0E000C106E1BF130600643386C502930695009E
:10E0F000AA8517050000130505ED6F602F9E4111DD
:10E1000022C406C62A840835EF600FBBFD571CB435
:10E11000B240224441018280011122CC4AC84EC63D
:10E1200052C456C25AC006CE26CA2A89AE890144B4
:10E13000176AFB1F130A5AB8976AFB1F938A0AB71C
:10E140001D4B83470A006369F404639D09029769C4
:10E15000FB1F9389B9B6176AFB1F130A2AB5930AE6
:10E16000F00F83C709006364F4061144A1442285BB
:10E170001306F00FCA850504EFF05FE73344040887
:10E18000E31794FEF2406244D2444249B249224A23
:10E19000924A024B0561828083A40A0093174400CF
:10E1A000BE949C208DC3FE20639F27016395690167
:10E1B000AA20EF10C04726854E868145EF00F03635
:10E1C0002685EFF0FFD805041374F40F9DBF832458
:10E1D0000A0093174400BE949C208DC39C34638F27
:10E1E0005701FE20639C27012685EFF05FF126850D
:10E1F000D145EF0090362685EFF09FD505041374C6
:10E20000F40F85B7C167F917630BF502411122C4FA
:10E2100006C685472A846399F50022852244B240C8
:10E22000814541016FF05FEF89476396F5008545B1
:10E23000EF1080737DD1B240224441018280828000
:10E240009D456FF07FED1765FB1F0355A5A68280E6
:10E25000011106CE68876C861767FB1F0347C7A5A9
:10E2600085476318F70070009305E1000545EF50FE
:10E27000301BF24005618280A947631DF6029C3184
:10E280009821A207D98F1EA1BC31B821A207D98F2E
:10E290003EA1DC31D821A207D98F5EA1FC31F82143
:10E2A000A207D98F7EA19C359825A207D98F1EA5DC
:10E2B00001458280054582809147631EF6009C31AE
:10E2C0009821A207D98F1EA1BC31B821A207D98FEE
:10E2D0003EA101458280054582809387C5FF0D4799
:10E2E000B3C60708636ED70031473387E7029767E5
:10E2F000FB1F9387A7D7BA97A8A38EA30145828057
:10E3000009458280930740203355F50A71159767B8
:10E31000FB1F2391A79A9767FB1F2381B79A9767E3
:10E32000FB1FA38CB79882809565411119059385D1
:10E3300035C006C6334505089720FB1FE78080D50A
:10E3400001C9B240E95541011723FB1F670023EFC4
:10E35000B240410182809767FB1FA38107969767B0
:10E36000FB1F238D07949767FB1F238807949767EC
:10E37000FB1FA38307949767FB1F238F0792854793
:10E3800041111767FB1FA308F79206C622C426C2D5
:10E390002A849767FB1F238007929767FB1F239BA5
:10E3A00007909767FB1F23A30790EF102031176595
:10E3B000FB1F1305A5CB1306000381459767FB1FC1
:10E3C000238F878E9720FB1FE78000031764FB1FB6
:10E3D0001304448D08209764FB1F9384F48D1DC99A
:10E3E0009565938545C012059720FB1FE78080CA7D
:10E3F0001767FB1F232EA78A11CD1C3010208145E3
:10E400009CA09767FB1F238AC78A12069720FB1FD1
:10E41000E78080FE9C201765FB1F034525CD176410
:10E42000FB1F1304B4893E951375F50F956508A07D
:10E43000938555C012059720FB1FE780A0C5976400
:10E44000FB1F9384A48688C035CD10208145120619
:10E450009720FB1FE78040FA98401420814725074A
:10E460007D56639BF604EF10A046B1473305F502D5
:10E470009565938565C0334505089720FB1FE780A8
:10E4800060C19767FB1F23A1A7822A8401CDEF10EB
:10E49000204431463306C502814522859720FB1F63
:10E4A000E78080F52244B24092441705000013052E
:10E4B000A5D541016F106042850710A393F7F70FB0
:10E4C000410745B79757FB1FA38A077E9757FB1F46
:10E4D000A384077E49BF411126C206C622C44AC092
:10E4E000AE849397556063D907081759FB1F13092A
:10E4F000097D034509009720FB1FE78060DF2A8420
:10E5000031C5182193070009631FF7021831CD4761
:10E510006312F7069756FB1F9386467A28219C22A2
:10E520001768FB1F0348788B130664008145014779
:10E530006316E50291C19CA29C2291C70345090084
:10E540008545EF503FAE2285EF501F951395F46837
:10E55000B240224492440249410182800E220507C2
:10E560001377F70FAE9793F7F70F09068545B3D7E3
:10E57000070B7DBFE529C1BF13F5150071D9EF0069
:10E58000905209CD9757FB1F83C7477381CB8545B1
:10E590001755FB1F0345A572EF50DFA813C51400E4
:10E5A00045BF0547637EC7029C319421A207D58FE2
:10E5B0001EA16399E700BC31B821A207D98F3EA103
:10E5C000014582800947E39DE7FEBC31B821A207DF
:10E5D000D98F3EA1DC31D821A207D98F5EA1CDB75A
:10E5E000054582809147631EF6009C319821A20761
:10E5F000D98F1EA1BC31B821A207D98F3EA10145F8
:10E600008280054582809147631EF6009C319821E7
:10E61000A207D98F1EA1BC31B821A207D98F3EA174
:10E620000145828005458280A1476318F6029C312E
:10E630009821A207D98F1EA1BC31B821A207D98F7A
:10E640003EA1DC31D821A207D98F5EA1FC31F8218F
:10E65000A207D98F7EA10145828005458280894726
:10E660006319F6009C319821A207D98F1EA101459C
:10E670008280054582803E2279714ECE06D622D414
:10E6800026D24AD01307F007AE896371F702094713
:10E690003AC47C86300093F5F50FEF003078B25025
:10E6A000225492540259F249456182805A22D94635
:10E6B0002A89328463F7E6007E2263F4F6006379E8
:10E6C000F70023140100300093F5F90F4A85F1B7E4
:10E6D0000A2202C4EFF01F81AA8435C5EFF01F9C07
:10E6E0009C246369F5001146A246CE854A85EF0059
:10E6F000B06975B7340026869305F00F4A85EFF0B0
:10E700002FEA75F1A2471A24DC479AA33A20BAA34C
:10E710005A20DAA37A20FAA3DA209AA7DC4495C714
:10E7200093F4F90F2286A6854A858297C167FD1763
:10E730002A86E31BF5FA22459947F9451CA144A115
:10E74000EFF05F9AA9BF094645B7014671BFA947D7
:10E75000631DF6029C319821A207D98F1EA1BC31FE
:10E76000B821A207D98F3EA1DC31D821A207D98FC9
:10E770005EA1FC31F821A207D98F7EA19C35982596
:10E78000A207D98F1EA501458280054582809C2164
:10E790001CA19C311CB1BC31B821A207D98F3EA16C
:10E7A000828023220500D82189476304F7000545AC
:10E7B0008280F62101114EC606CE22CC26CA4AC856
:10E7C0000D47AE896379D7049C4584339023A033E9
:10E7D000A204D18CB023220493874400518C639C03
:10E7E000D7029307C4FF2A89B3C707086361F702FA
:10E7F00003A589002311990023108900F155972062
:10E80000FB1FE780C0A32322A900014531A0228578
:10E81000EFF02FE771FD0545F2406244D2444249D2
:10E82000B24905618280797122D426D22E8406D61F
:10E830004AD01C201947AA84B2856390E70630208D
:10E840002800EFF03FDA0DE92884EFF08FE30C3079
:10E850002A890DC92E86171700001307A7D1340087
:10E860009D452685EF0090304A85094681457529EA
:10E870004A85EFF0EFED0145B2502254925402590F
:10E880004561828089477C803C840A867C813C8506
:10E890007C822685EF009058F9BF49476395E702CF
:10E8A00032202800EFF05FD861F91755FB1F1305E0
:10E8B000E57B5E25E9D3183068253C00C946014652
:10E8C000A685CD2C4DBF5147639DE700322028001F
:10E8D000EFF09F9A55F10C3030002685EFF0BFD94C
:10E8E00059BF5947639AE70432202800EFF0DF9CB4
:10E8F00041F52C842685EFF0EFE105C958453485B4
:10E900001E23B697B3C707081EA3B5D75C47A5D784
:10E910009757FB1F83C7873AB9DF85451755FB1FFC
:10E920000345E539EF500FF0B9B789473EC03C8445
:10E930000C300A867C82B1BF0C30231001000A869D
:10E9400091BF5D71A2C456DA86C6A6C2CAC04EDEA9
:10E9500052DCAA8A88312E8432C6EFF08FD5B245B8
:10E9600001ED0144B6402285264496440649F259F9
:10E97000625AD25A61618280230205002311050088
:10E98000834904008547AA846399F9003020280848
:10E99000EFF03FC12A8405491DA09D476391F9040A
:10E9A00018218D47E31FF7FA302028080549EFF0BA
:10E9B0009FC52A8409E5054681452685BD2626850D
:10E9C000EFF0EFF388243C080147CE862286D685F7
:10E9D000D522E30909F82685EFF08FD761B7CD4737
:10E9E000639BF90018219147E31DF7F630202808B2
:10E9F000EFF0FFC645B7D547E395F9F6034A0500A2
:10EA00008947E310FAF6302028080549EFF03FD493
:10EA10002A8455F583570102A1EBB8841306F0034D
:10EA2000DC44930607FCB3C60608636AD600B085CB
:10EA3000D94663F6C600B486D94563EDD500BAA3BE
:10EA40000145EF00D03E054903560102D2852685D7
:10EA5000AD2CB5B7AC87BAA3D2A38EA3F6A38547D6
:10EA60009CA0014A0149CDB7014AF9BF7971AA8535
:10EA700022D426D22221AA84280806D64AD0EFF032
:10EA80005FD2F24599E53DE185452285EFF04FFCE7
:10EA900075A0BC8415476395E706B8858D4763F775
:10EAA000E7046800EFF0BFCE0359E100DD4763FBE8
:10EAB00027018C86B70717008507100822853EC8F6
:10EAC000EF00D035BC851109638527012285EFF061
:10EAD0002FF71C8672466C00858B1106228591CF1C
:10EAE000EFF03FE601C52285EFF08FF5884449DD60
:10EAF0009710FB1FE780206741BFEFF0DFD2DDB743
:10EB000011476389E7001387A7FF85463347070846
:10EB100063ECE6023147F117B387E7021757FB1F93
:10EB20001307C754BA979A2371D3A8233008A28534
:10EB30000D204DFDB8849147E318F7F4B2502254EC
:10EB400092540259456182802C082285212E59FD5C
:10EB5000F5B701114AC82A89314526CA4EC606CEE4
:10EB600022CCAE89B2849710FB1FE780607229C166
:10EB70009307000A231135011EA12A84214611059D
:10EB800095C0A6859720FB1FE7808080A2854A85D7
:10EB9000EF50AFB50145F2406244D2444249B24918
:10EBA0000561828081459720FB1FE780E084F9BFE3
:10EBB0000545D5B701114AC82A891305000226CA9E
:10EBC0004EC652C456C25AC006CE22CCAE8A328B32
:10EBD000B6893A8ABE849710FB1FE780606B21C913
:10EBE000930720FA1CA1A3006501231155012302FC
:10EBF0004501A30235012A84614621059DC0A685F1
:10EC00009710FB1FE780C078A2856244F240D2448F
:10EC1000B249224A924A024B4A85424905616F50E5
:10EC2000CFAC81459710FB1FE780007DF1BFF2401C
:10EC30006244D2444249B249224A924A024B056197
:10EC400082805C45797122D406D62A84AE86A5C717
:10EC5000BA23F885130720066396E504FA231756AE
:10EC6000FB1F035626053357C70AB22B9E2B13777B
:10EC7000F70F918F93F7F70F01E6890793F7F70FD7
:10EC8000BA97FD17B3C7E702FC863E206E20082422
:10EC9000FC8401473C080146EFF0DFF1B2502254FA
:10ECA00045618280D82F9757FB1F83A76700120703
:10ECB000BA97FE23D1BF2EC6194681452808971062
:10ECC000FB1FE7806073B246C9B7797122D406D6BC
:10ECD00026D22A8491CD08242E866E202254B2504A
:10ECE0009254814701479306000645616FF09FECFF
:10ECF000B284280059469710FB1FE780E06F6484B8
:10ED000099E43E2048446C007C85EFF04FB36E20C0
:10ED100008243C000147930600060146EFF09FE9F6
:10ED2000B2502254925445618280797106D681474F
:10ED300099E53E2170867C845C4589EF3C002E86F7
:10ED40006E210825014793060006EFF0BFE6B2509A
:10ED500045618280BE237C85D5B7411122C406C699
:10ED60001C2111472A846392E7022E866E21082512
:10ED700081470147CD46EFF0FFE349466E2022442C
:10ED8000B240154541016FF06FA613F7B70F8946E2
:10ED90006317D7000146EFF05FF35146C5B70D4743
:10EDA0006398E7002244B240014641016FF0FFF74B
:10EDB000B2402244410182809A21B1477117330742
:10EDC000F7029757FB1F9387672ABA97D84301EB3F
:10EDD000D841AAA70145D8C3BA219AA7828059452C
:10EDE0008280797126D2444522D44AD006D62A841C
:10EDF0002E89B1C4C84419C59710FB1FE780A036FF
:10EE000023A604009E206E2008247C85BE20014796
:10EE1000930640067C869E244A867C879C483EC892
:10EE20003E207C843C00EFF0FFD8A38E240123A871
:10EE30000400B25022549254025945618280280045
:10EE4000314681459710FB1FE780005B3E206E2016
:10EE500008247C8401473C00930640064A86EFF074
:10EE60007FD5C1BF797152CC2A8A8A2126D206D693
:10EE700022D44AD04ECE56CAAE84EFF08F806302C1
:10EE8000051240452A89630E04107E21639B4711B9
:10EE90001E24638A0710542C975AFB1F938A4AE159
:10EEA00003A70A009206FD1736977A23B3C707080F
:10EEB0001EA46316F70093053006EFF09FD85C4858
:10EEC000B5EBC840834915001C21A209B3E9F9003C
:10EED000BE2013872900631AF702F9559710FB1F0C
:10EEE000E780E035C8C023913401034589002686B8
:10EEF000D285EFF01FC61DEDB25022549254025934
:10EF0000F249624AD24A456182809565938515C06F
:10EF10004E859710FB1FE780E01748C8C840231CA8
:10EF20003401F9559710FB1FE7806031BE20C8C03F
:10EF3000F917BEA048482DCDB220362C1E2C330820
:10EF4000D60063C90707582C83A70A009545120706
:10EF5000BA97BE2363CA0705CC4036959710FB1FAE
:10EF6000E78000433A2CBE20BA971A2CB3C7070893
:10EF70003EAC6398E702035729000345890030003F
:10EF800078845848D2857C853AC6EFF09FBC11C57D
:10EF900048489710FB1FE780001D232A0400232CFC
:10EFA0000400054591BF99454A85EFE03FFFD5BF75
:10EFB000A545DDBF9145CDBFBE21F9C3011126CACC
:10EFC00006CE22CC1757FB1F0357C7CEAA846D4528
:10EFD0006363F70A2E84484091459710FB1FE78032
:10EFE00000263E20AA861CA13E20A1831CB11E2023
:10EFF0003CA11E20A1833CB13220C167F917110644
:10F0000033460608639FF4022AC4314532C697107E
:10F01000FB1FE780E027AA854D45B1CD930700F996
:10F020003246A2469CA1F957BEA18947DCA1F2A1B4
:10F0300094C51755FB1F034585C8EF401FEB0145DD
:10F040001DA881452685EF40505211E91757FB1F37
:10F050001307C7C61C23E5D7FD171CA3CDB78947E7
:10F060006302F5029D476301F502C9476300F5029B
:10F07000FD47E30DF5FCF2406244D2440561828015
:10F080006D4582805145C5BF1145F5B70945E5B7C6
:10F09000011122CC4AC831441309C5FF3304890247
:10F0A00026CA9754FB1F938464FC06CE26945C40CA
:10F0B000A9C31757FB1F034767C00DC768843EC627
:10F0C0002A241E242C007C85EFF01FEF11C5484038
:10F0D0009710FB1FE7802009B1473309F902CA9452
:10F0E00023A204000545F2406244D244424905612E
:10F0F00082800145CDBF797126D244454ECE52CC97
:10F10000FE20BA289759FB1F83D9C9BA06D622D444
:10F110004AD056CAB3D9F90A2A8A9E282DCF998F88
:10F120004E8463D4370133C4070889452285EFF044
:10F13000AF9F2A89CD4A31C5BE202AC660857C840E
:10F14000BE2899EB9E28130925001CA19E28A183A7
:10F150001CB1637434058228BE28CC4422864A85BB
:10F16000BE959710FB1FE780A02203556A002C0074
:10F17000EFF09FE4AA8A15C54A859710FB1FE78028
:10F1800080FEB250225492540259F249624A568586
:10F19000D24A45618280890761B7791433440408F3
:10F1A00065BFBA289E203A949A28FD17B3C707086E
:10F1B000334404089EA0A2A86376E400F9F3FD5747
:10F1C000DCBCC1B781455285EFF0BFC15DBF79712D
:10F1D00022D44ECE56CA5AC85EC662C406D626D2BD
:10F1E0004AD052CC9759FB1F9389E9AC03CA090056
:10F1F000975AFB1F938A8AAB054B5284930BF00FEF
:10F20000175CFB1F130C5CAB83A40A00931744002C
:10F21000BE9403C90400631D6907DC44B5CBD8471D
:10F2200025CB9A2339CB9757FB1F83C727A999CFA3
:10F230002685EFF05FECAA8505ED05049757FB1FC7
:10F2400083C797A76351F40223808900B2502254E8
:10F250009254F249624AD24A424BB24B224C4A85FE
:10F260000259456182809757FB1F238607A4F9BF87
:10F270002685EFF01FB70149D1BFDC3F639A7701C4
:10F28000930520062685EFF0DF9BDC44A38E070064
:10F2900083470C0005041374F40F6363F400014406
:10F2A000E31444F7C9BF4111154506C6EFF05FDE10
:10F2B00009C50545B240410182801945EFF05FDD87
:10F2C0006DF91145EFF0DFDC6DF51D45EFF05FDC0A
:10F2D0006DF11755FB1F0345359E69DDB2404101B5
:10F2E0006FF0FFEE9E210D47F117B3C70708636368
:10F2F000F706DC41411122C406C626C22E84A9CFDE
:10F300008545AA84952539CD2685AD2BC167F9178A
:10F31000638FF40009ED3E2099CB162019476395C1
:10F32000E6041757FB1F0357E79863FFE702975759
:10F33000FB1F83C7A798A285268599C72244B240A0
:10F34000924441016FF05FC72244B24092444101B0
:10F350006FF09FA6094582800945B240224492443D
:10F36000410182805145D5BF6D45C5BF797126D217
:10F3700052CCAA842E8A5D4589454AD04ECE56CAC3
:10F3800006D622D4B289B68A3A89EFE0FFF925C5BC
:10F390002A84014563060900D685130544000299B5
:10F3A000935785003CB093074500230044017C85BA
:10F3B000954728A07C84A300340122C69757FB1FE1
:10F3C00083C7C78F2C00268585C7EFF0FFBEAA84B0
:10F3D00011C522859710FB1FE780E0D8B250225458
:10F3E0000259F249624AD24A268592544561828086
:10F3F000EFF09F9CE9BFCD44D5B7797126D24AD0B2
:10F4000052CC56CA2E8906D6BE8522D44ECE9947F6
:10F41000B284368ABA8A6314F9062A220944EFE0D4
:10F420005FA62AC625C55C4583596500BE239EA0FC
:10F43000B247154723805701BAA31757FB1F13077D
:10F44000978710239305160093F5F50F0CA3D0A30F
:10F4500099E1854614A351476317E9001547BAA0FF
:10F46000DC479A249AA75287A686CA854E85EFF074
:10F47000FFEF2A8432450DC4EFE09FAD01A842861C
:10F480007400AA89EFE0DF912A845DD1B250228511
:10F49000225492540259F249624AD24A456182800A
:10F4A000F945EFE03FC4DDB79E211CA19E21A18359
:10F4B0001CB1BE213CA1BE21A1833CB1114582807B
:10F4C0009E211CA19E21A1831CB1BE213CA1BE2175
:10F4D000A1833CB1DE215CA1DE21A1835CB1FE21D0
:10F4E0007CA1FE21A1837CB1214582809E211CA1AB
:10F4F0009E21A1831CB1094582809E211CA19E21D1
:10F50000A1831CB1BE213CA1BE21A1833CB1DE215F
:10F510005CA1DE21A1835CB1FE217CA1FE21A1833F
:10F520007CB19E251CA59E25A1831CB52945828002
:10F530009A218546AA8718A19A21218318B19A2178
:10F540006319D700BA2138A1BA21218338B11145F6
:10F5500082800945631DA700BA211945B8A3BA21C5
:10F560002183B8B3DA21D8A3DA212183D8B38280EA
:10F570009E211CA19E21A1831CB1BE213CA1BE21C4
:10F58000A1833CB111458280797126D24AD04ECEFA
:10F59000B2842A89AE8929468145480022D406D6FC
:10F5A00036849710FB1FE78020E564868DE43E20BB
:10F5B0007C829747FB1F83D7E76F7C845C4481CFB5
:10F5C000D42F1747FB1F0327A76E9E279206369757
:10F5D0003A237C8578834A8517070000130727F2B2
:10F5E000540013F6F90FD545EFF05FD82A8911C101
:10F5F00095E085471CA02302040001468145228531
:10F60000EFF0AFECB25022549254F2494A850259BD
:10F61000456182802285EFE0BF93EDB7B286170780
:10F620000000130727F12E8685456FF03FD40111A6
:10F6300068874165700001489307F00F0D479706F2
:10F6400000009386A6E699457D1506CEEFF0FFDA19
:10F65000F24005618280B28701482E8611479706E5
:10F660000000938626E6C9456FF03FD9B28617079A
:10F6700000001307E7E72E86CD456FF03FCF01115D
:10F6800022CC26CA4AC84EC606CEAA842E89175452
:10F69000FB1F1304A4A09759FB1F938929A31C40A7
:10F6A00081C7CA85268582971104E31A34FFF24088
:10F6B0006244D2444249B24905618280411122C468
:10F6C00006C626C21747FB1F130747707C2B783BE3
:10F6D0001754FB1F130404A11CB4BA9793F7F70F38
:10F6E0001CA4A5CB1305C0033385A702A56585051A
:10F6F0009744FB1F9384C45C9710FB1FE78080999D
:10F7000010249307C00381453306F60288C0971082
:10F71000FB1FE78060CE14249C4001477D56634167
:10F72000D7022244B2409244130600038145175584
:10F73000FB1F1305A59641011713FB1F6700C3CBE1
:10F74000B2A32382070023A6070205079387C703F6
:10F75000F9B7B2402244924441018280411122C44F
:10F7600026C24AC006C62A892E84B2849730FB1F5F
:10F77000E780802309EDC167F91751456313F9004C
:10F780000145B240224492440249410182805455CD
:10F790005C2195C213F727014146630BC700C18B5B
:10F7A0003D45E5D3BC2E0145E3FD87FC3145D1BF86
:10F7B0001545F5D4F9B7C18B0145E1F71545D1B72A
:10F7C00079714AD0416922D426D24ECE52CC56CA43
:10F7D0005AC806D6AA8401449759FB1F9389899079
:10F7E000174AFB1F130ACA4D930AC0037D19054B24
:10F7F00083C789006364F400014525A833075403D7
:10F8000083270A00BA97BA236316270105041374E5
:10F81000F40FF9BFC833300093856700EFB0D12EE5
:10F820001946A68528009710FB1FE780E0C8E31F54
:10F8300065FDB250225492540259F249624AD24AAA
:10F84000424B456182804166AA869755FB1F83C55E
:10F85000E5891747FB1F0327A74681477D16639459
:10F86000F50001458280035827003A856306C800E9
:10F8700003480700E308D8FE850793F7F70F13073F
:10F88000C703F1BF411106C69730FB1FE780C011C7
:10F8900009C54A29B240410182800145E5BF1747A9
:10F8A000FB1F0327E7419756FB1F83C626841107DA
:10F8B000814701456393F6008280102301C6050548
:10F8C0001375F50F850793F7F70F1307C703DDB718
:10F8D0001755FB1F0345858182801747FB1F1307C0
:10F8E000E77B81473A86B1460C4391E5B3C7C72011
:10F8F00088C30145828085071107E397D7FE4D45F0
:10F900008280411106C622C49730FB1FE780C009E0
:10F910000DCD2A842A218545EFF07FD6485409C5AC
:10F920009710FB1FE780208422851306C0038145C2
:10F930009710FB1FE78040ACFD573EA02302040058
:10F940000145B2402244410182800945DDBF411199
:10F9500006C69730FB1FE780200509C54825B24041
:10F96000410182800145E5BFC167F9176305F502D2
:10F97000411122C406C62E849730FB1FE780C002C7
:10F98000AA87014589C7DC237D8C33358000B240CE
:10F9900022444101828005458280411122C406C66D
:10F9A0002E849730FB1FE780200001CD5A29AA87BB
:10F9B000054563048700C2AB0145B24022444101C2
:10F9C00082800545DDBF39CD01114AC8416922CC8D
:10F9D00026CA4EC652C456C206CEAA8401449749CE
:10F9E000FB1F93892970174AFB1F130A6A2D930A7C
:10F9F000C0037D1983C78900634BF400F240624461
:10FA0000D2444249B249224A924A05618280B307F0
:10FA1000540303250A003E953E2163832701829407
:10FA20000504C9BF82809747FB1F83A76729C1666A
:10FA30001746FB1F0346866B890701450147FD16E4
:10FA400091456313E600828003D807006309D8005C
:10FA500003C8A7006315B80005051375F50F050762
:10FA60001377F70F9387C703E9BF9746FB1F83A65A
:10FA700026251746FB1F0346666791060147814707
:10FA8000631FE600858393C7F7FF0545B3C70708E3
:10FA90006361E5023315A0283345050882808C2276
:10FAA00099C1CE36CD8F05071377F70F9386C6031E
:10FAB000C1BF93F61700F9FE050585831375F50F91
:10FAC000C1BF797156CAAA8A2E8526D24AD04ECE97
:10FAD00052CC5AC85EC662C406D622D4AE84328BDB
:10FAE000368CBA8B3E8AC28946899730FB1FE780E5
:10FAF000A0EB3DED41657D159730FB1FE780C0EA27
:10FB00002A84554531C81946DE8513056400A302D1
:10FB100084019710FB1FE780A0878357010326A06D
:10FB2000230264013EA88357410323005401232686
:10FB300004025EA82306440123173401231824017C
:10FB4000EFF0BFF20AB8232A04022685232C040210
:10FB50008145EFF0DFB20145B25022549254025970
:10FB6000F249624AD24A424BB24B224C45618280F2
:10FB70004545DDB79746FB1F83C646571747FB1F12
:10FB80000327071481476395F60041657D15828040
:10FB90000E3B1306C7036394A5002A2382808507C2
:10FBA00093F7F70F3287C5B741661748FB1F034825
:10FBB000E8539746FB1F83A6A61001477D1695487C
:10FBC00011436314E80001458280BE223685638EAE
:10FBD000C702CC5A9DC9BC31AC2189CD938597FD14
:10FBE00093F5F50FE372B3FE9387D7FA93F7D70F28
:10FBF00089EF82809385F7FD93F5F50FE3F6B8FC66
:10FC00009387D7FA93F7D70FE1D305071377F70F49
:10FC10009386C6037DB741669745FB1F83C5054D97
:10FC20001747FB1F0327C70981477D1625486394A3
:10FC3000F5000145828036233A85638BC600545B0C
:10FC400081CAB4329386E6FD93F6F60FE374D8FECC
:10FC5000850793F7F70F1307C703D1BF011122CC14
:10FC60002A84494506CEEF609FD81DC12AC6228549
:10FC70009730FB1FE78040D301CD624432460E39F6
:10FC8000F2401745FB1F0345154605616F40CFCF76
:10FC9000F24062440561828079714ECE52CCAE89C9
:10FCA0002A8A93053005414526D24AD056CA5AC8F9
:10FCB00006D622D4328B3689BA8A9700FB1FE7809A
:10FCC000603DCD4429C92A848944638109044146A1
:10FCD0008145231261019700FB1FE780E071568682
:10FCE000CE8522859700FB1FE780806A2146630F3F
:10FCF0000902CA8528009700FB1FE7806069A28679
:10FD000050002C005285EF307075AA842285970030
:10FD1000FB1FE7804045B25022540259F249624A23
:10FD2000D24A424B26859254456182808145280003
:10FD30009700FB1FE780406CD9B7411122C440599E
:10FD400026C206C6AA8429CC085409C59700FB1F01
:10FD5000E7806041285809C59700FB1FE780A04055
:10FD6000685809C59700FB1FE780E03F285C09C57C
:10FD70009700FB1FE780203F685C09C59700FB1FC9
:10FD8000E780603E0325040809C59700FB1FE78054
:10FD9000803D22859700FB1FE780E03C23AA0402F8
:10FDA00022448E38B24092441745FB1F0345B533B9
:10FDB00041016F40CFE6411126C206C622C4AE847F
:10FDC0009730FB1FE78040BE21C9032345032A84E7
:10FDD000630403048328C307032883078327430797
:10FDE000032703078346630003560300834523006C
:10FDF0002685EF60DFC72285EFF03FF4EFF0BFE12B
:10FE000001CD2244B24092441745FB1F0345B52D56
:10FE1000854541016F400FA1B24022449244410107
:10FE20008280411122C426C206C6AA842E8497303D
:10FE3000FB1FE78060B75C5989CF9E23639B9700C7
:10FE400085476318F4002244B240924441016FF0A8
:10FE5000DFEEB2402244924441018280411106C645
:10FE600022C426C2EFF05FD429C144592A8495CC1C
:10FE7000BC209DC79747FB1F83A707E589C7DC43C5
:10FE800099C326858297B8309307F002631FF70065
:10FE90002A202244B2409244814541016FF0BFF1D3
:10FEA0009747FB1F83A707E2D1BFB2402244924489
:10FEB00041018280411126C24AC006C622C4AA84DA
:10FEC0002E899730FB1FE78020AE05CD405955C4E1
:10FED0001E206394970A3C30130710026395E708CD
:10FEE0003C20ADCF7C5403270408DE2B15E313F729
:10FEF000170019CF18545A23058B19CB93072002EA
:10FF00003CB0B240224492440249054541018280FE
:10FF100013F7270001CB18545A23098B01C7930705
:10FF20004002F9BF918B81CB1C54DE23918B81C79A
:10FF300093076002F1B79747FB1F83A7E7D8F1D378
:10FF4000DC43E1D32285829738309307F002814564
:10FF5000E319F7FA2685EFF01FE665B79747FB1F11
:10FF600083A747D6E9BF1307A0026398E70063049D
:10FF7000090013092003CA85F1BF631C0900268507
:10FF80009730FB1FE78040A209C55C2193E707017A
:10FF90005CA1A6854A85EF604FBDA5B7011126CAB1
:10FFA00099476C85AA842E858D4522CC4AC806CEF9
:10FFB000328936847C84EFE02FB72AC61DC9AA8512
:10FFC0004A8502942A8419E52C002685EFF08FB12A
:10FFD0002A8411C532459700FB1FE780C01826858B
:10FFE000EFF0DFC7F24022856244D2444249056106
:10FFF00082804D44EDB7411122C42E862E8497167F
:020000025000AC
:10000000000093864675894506C626C24AC02A89DD
:10001000EFF0DFF80C20AA844A85EFF0DFD9B24078
:100020002244024926859244410182809747FB1F62
:1000300083A747C985CB9C4395C71D71A2CC86CEAB
:10004000984110082A843AC8D84185453ACA82970F
:1000500011C548862A206C00EFF0FFF9F64066448F
:10006000256182808280AA872E8591CFFC5781CF1F
:10007000982398A1983398B1B82BB8A1982FDC4B4E
:10008000B8B1DCC18280414681451703FB1F670080
:10009000A3369747FB1F83A727C381C79C4791C3FC
:1000A0008287094582801747FB1F032727C81DC782
:1000B0005843AA8705450DC703A50708411106C681
:1000C000930605021306050C9305050613050504A2
:1000D0000297B2401375F50F410182800545828079
:1000E00082804DC9357122CD2A840A2126CB52C582
:1000F00056C35AC106CF4AC94EC7DEDE2E8AB28A1F
:10010000368B9730FB1FE780208AAA8431C50C18F4
:100110002285EFF05FF53C20938B6400A9CBEF5074
:10012000BFFE2A89014583C95400EF507FFBAA8492
:100130000C100818EF10604408542C10EF10804485
:10014000DE88A68B5AC04E88DE874A87141030108E
:10015000D6855285EF20A06BFA406A44DA444A49BA
:10016000BA492A4A9A4A0A4BF65B0D618280EF50DF
:10017000BFF9AA89014503C95400EF507FF62ACE82
:1001800008540C10EF10603F2C100818EF10803F3F
:10019000F2484DBF8280AA8701CD1855414511CB49
:1001A000FC5781CB28333D476375A700882F828099
:1001B000414582806DC5411122C406C626C2AA8768
:1001C0002E840945E1C998337D761306F67F98A100
:1001D000B8234D4598B1B833B8A1D823B8B1D433BA
:1001E000DA21858AA2061377F7EF558FDAA1D43387
:1001F000334707081377F7DF93D61648A606558FBF
:10020000DAA1D433334707081377F7BF93D62648CC
:10021000AA06558FDAA1D43333470708718F93D6D6
:100220003648AE06558FDAA1F42333470708799B89
:10023000858A558FDAA1F42333470708759B898A8D
:10024000558FDAA1F423334707086D9B918A558FA8
:10025000DAA1F823DE21218BDD9BD98FDEA1EF60AF
:100260000FF9AA845145EF608FF8383093F4F40FFA
:10027000AA8749456360970293F7F70F63ECE7009D
:1002800018209147614563E7E7001830854763E32D
:10029000E7000145B2402244924441018280094571
:1002A000828015C52A87AE87094585C5411106C6D6
:1002B000143313851700194694A19305270097005E
:1002C000FB1FE780E00CB2400145410182800945F7
:1002D000828082800DC9AA872E8709459DC541115C
:1002E00006C6B423903313052700A206D18E96A12B
:1002F0002146938537009700FB1FE7806009B240D5
:100300000145410182800945828082801DC12A8782
:10031000AE8709458DC141113E85414693051700C1
:1003200006C69700FB1FE780A006B24001454101C9
:100330008280094582808280AA87094591CB89C93C
:100340009C333D4761456365F7009CA10145828070
:10035000828005C52A87AE87094595C141113E8532
:10036000130600049305170006C69700FB1FE780DD
:100370002002B2400145410182800945828082808D
:100380001D71A2CC2A84084586CEA6CA2306010088
:10039000042135479387F4FF93F7F70F6362F70A59
:1003A00017D701001307C770B3C7E7209C43BA975C
:1003B00082870C08EFF01FE0C947631CF5049947DA
:1003C0005C862A206C00EFF01FC3F6406644D644DA
:1003D000256182800C08EFF03FF61DED2A20972062
:1003E000FB1FE780605CA14705C15825631CF7042B
:1003F0001747FB1F0327478D9D4719C7184309C798
:100400001008A6850297AA875C8629A00C08EFF041
:100410007FEC69D51C86D5F72A20EFF03F8475B7AD
:100420000C08EFF01FE8F5B71C312308F1007DB789
:100430000C08EFF01FF2F1BF0C08EFF03FEDD1BF59
:100440009D47BDBF1747FB1F0327C78775B74111DE
:1004500022C406C626C24AC01821930720092A844E
:10046000631AF7101C3139476395E70A562109676B
:10047000610781476398E6089744FB1F93840485CE
:10048000884049C10C4403C90500631D09001C21B3
:1004900085052146B9CB29059700FB1FE78040EF72
:1004A0009C40A5C349459700FB1FE78060DE2A8476
:1004B0001DC1930710FC1CA1A30025018C40090558
:1004C000414689059700FB1FE78080EC9C40A28590
:1004D0008833EF309FA188409700FB1FE780A0C8BA
:1004E0009737FB1F23A4077E29A809059700FB1F48
:1004F000E78000EAEF30407605495DF19C402380BB
:1005000027018547B2402244924402493E85410179
:1005100082801307E003639DE7063821954763193E
:10052000F7024A21EFF0AFC29147E31CF5FC973781
:10053000FB1F83A72779F1D79C47E1D772244A2074
:10054000930564002244B2409244024941018287EB
:10055000A147631BF7006C204A202244B24092441A
:10056000024941016FF01F95930600038147E31B89
:10057000D7F8D5B79306000A8147E315D7F8EFF00F
:100580003FE008443DDD9700FB1FE780C0BD95BFFD
:1005900081478DBF011122CC06CE26CA4AC8094424
:1005A00015CDAE8409449DC92A898D456800EF5058
:1005B0003F871C8726866C0093F7F70393E70704B1
:1005C0004A855C87EF20A01B2A8409E90D466C0050
:1005D000138534009700FB1FE78080DBF240228503
:1005E0006244D2444249056182805D714EDE86C616
:1005F000A2C4A6C2CAC052DC56DA5AD85ED689490D
:1006000055C9328989495DC6138B45002A8AAE8A4D
:10061000334B0B08930530055A859700FB1FE78085
:1006200060A72A84CD4959C5EF50FFAFAA845686EA
:10063000D28593DA840013DA040193FBF40F1305D7
:10064000440093FAFA0F137AFA0FE1809700FB1F28
:10065000E78040EBA301740123015401A30044018E
:1006600004A0EF50BFABAA85414608089700FB1FC6
:10067000E78040E9214734005A86A2850808EF2028
:100680008036AA891DE121462C0023007901A300B0
:10069000590123014901A30199001305490097005D
:1006A000FB1FE78020E6EF50DFA822859700FB1FA5
:1006B000E78060ABB640264496440649625AD25A57
:1006C000425BB25B4E85F25961618280011126CA9C
:1006D000AA842E854AC806CE22CC2E899720FB1FDD
:1006E000E780802C4DCD40594DCC5C30094793F6C6
:1006F000B70F6387E60011471305E00F639DE70618
:100700001E20094563992707130984004146A685E1
:100710004A859700FB1FE780A0C74146A6851305C1
:1007200084019700FB1FE780A0C6383085469307F9
:10073000F7FE93F7F70F63E6F6041306C40332855A
:10074000C14532C6EF50CFED32469306C402CA858A
:100750002285EFF01F993C2089CB22856244F2402C
:10076000D244424905616F1040073830C947E3065B
:10077000F7FE3CB00145F2406244D2444249056173
:10078000828093071005E317F7FE3C20E5D722850A
:100790006244F240D244424905616F10400A094563
:1007A000D9BF4945C9BF797152CC2A8A328522D432
:1007B0004AD04ECE06D626D2AE8932899720FB1F6C
:1007C000E780801E494405C9445949448DC49E2090
:1007D00063932703DC30A18B85EB0944B830930782
:1007E000B005631AF7002685EF104002BC20ADCBA0
:1007F0009307C005BCB0B2502285225492540259CE
:10080000F249624A456182801739FB1F1309095278
:10081000832709001304E00FF9DF9C47E9DF138405
:10082000840122854146D2859700FB1FE78040B6B0
:100830008327090083A5040822869C479385050425
:100840002E850A87814682972A844146CE850A856D
:100850009700FB1FE78040C649D11374F40FBDBF5A
:100860009307E00541BF39C9011122CC26CA06CE43
:10087000AA842E84094595CD0D468D052800970044
:10088000FB1FE780E0B01C8570002C0093F7F70396
:1008900093E7070426855C85EF10706E19E90D4615
:1008A000A28568009700FB1FE78000C17D153335E6
:1008B000A000F2406244D2440561828009458280F2
:1008C000011152C42A8A32854EC656C25AC006CE7B
:1008D00022CC26CA4AC82E8BB28AB6899720FB1F23
:1008E000E780800C09ED8944F24062444249B249F4
:1008F000224A924A024B2685D244056182805C5985
:100900002A89C544F5F34D45EF606F8E1374F50FDA
:100910005145EF60CF8DE38809FC03C78901E3648B
:1009200087FC9377F50FE3E0E7FC930530051305AB
:10093000400897F0FA1FE780E075232AA9022A846D
:10094000CD445DD11306400881459700FB1FE78029
:10095000A0AAA3010400230144012302640123107F
:1009600054012326340723240402A302040063074E
:100970000A002285EF00B060AA8419E18144ADB776
:100980004A85EFF08FBB8DB7397122DC06DE26DA9F
:100990004AD84ED652D456D25AD05ECE62CC66CA0F
:1009A0000944630A0610BA84094463060710AA8B37
:1009B0002E89328B368C9720FB1FE780E0FEAA8AB7
:1009C000514475C993053005414597F0FA1FE780FA
:1009D000606CAA894D4465C198309C2003CA3400DC
:1009E00022075D8FBC20620AC207D98F336AFA00E2
:1009F00083A78A0263E647017D5709446398E70AA3
:100A00006307090083C74A000544898BC5C3214693
:100A100081450A859700FB1FE780009E930C4C00E0
:100A200093053005B3CC0C08668597F0FA1FE78074
:100A300060662A894D443DC96286DA8511059700B2
:100A4000FB1FE78020AC1146A6854A859700FB1F57
:100A5000E78040AB414693858A014E859700FB1F96
:100A6000E78040AA21478A866686CA854E85EF10B0
:100A700090772A841DE521468A8528009700FB1F70
:100A8000E78040A821469385440028009700FB1F7B
:100A9000E78080A28547631EF502D2855E85EF6000
:100AA000EFB04A8597F0FA1FE780E06B4E8597F02C
:100AB000FA1FE780406BF25022856254D2544259AB
:100AC000B259225A925A025BF24B624CD24C2161CB
:100AD00082800544F9B7797122D406D626D24AD04D
:100AE0004ECE2E849397556063D607049734FB1F30
:100AF0009384445FA83097F0FA1FE780607F2AC68E
:100B000009CDEFF0DF94B24511E5A8209307F00F6F
:100B1000631FF5002E85EF302FB81319F468B2501B
:100B200022549254F2494A85025945618280EF303D
:100B3000CFBBE5B713F9150063070900EFF00FB25B
:100B400013491400E9BFE1DD854421A0850493F435
:100B5000F40FEFE0FFD7E3F4A4FCB3179028B3C978
:100B60000708E18FE5D74E85EFF0CF80C167FD170D
:100B70006305F500DD45EFF00FA43349340145B7B7
:100B80009737FB1F23A407149737FB1F23AE0712C9
:100B90009737FB1F23A807129737FB1F9387C7536D
:100BA000170700001307675998C3170700001307BA
:100BB000072DD8C317F7FFFF1307470E98C79737BE
:100BC000FB1F9387A750171700001307E73F98C331
:100BD00017170000130727FAD8C3171700001307C9
:100BE000A72398C782809737FB1F83C7E74FA18B46
:100BF000014789C71737FB1F1307074E9737FB1F9E
:100C000023A4E70C014582809737FB1F83C7C74D9C
:100C1000918B014789C71737FB1F1307274B97375E
:100C2000FB1F23A1E70A01458280011106CE2AC6D7
:100C3000EFF01FF5324599459737FB1FA385A74A6B
:100C4000EFD0AFE9F24017F5FFFF1305C51D0561B1
:100C50006FE0BFC81C5599C321458280011122CC89
:100C600026CA2A84AE84130500049305300506CEF7
:100C700097F0FA1FE780004208D469C51306000404
:100C8000A68597F0FA1FE780A0707454B82A93776E
:100C90008700F5C71C54BC23A18BF5C38327040828
:100CA000D5E3930530051305001097F0FA1FE78090
:100CB000603EAA872320A4080D45D1C774549C30F8
:100CC0009832D9C73337E0000E07936707016C5499
:100CD0005CB0B829058B19CB1854854638230D8B89
:100CE0006316D70078201367170078A0032704083D
:100CF00009C778201367870078A005476396E70C3B
:100D00009304840041468145268597F0FA1FE780C9
:100D1000A06E414681451305840197F0FA1FE780D4
:100D2000A06D1306C4033285C14532C6EF504F8F04
:100D3000832704083246BDC72285EF005030930751
:100D4000000525CD2145F2406244D24405618280F0
:100D5000A14735FFBC20918B91E7BC2A918B99E389
:100D60008547B5B79820942295473307F70297D760
:100D70000100938767D7BA97B6979C2389BF9C30A9
:100D800081C79032E14721F6BC205D8F118B69DB72
:100D90009820954794223307F70297D7010093874D
:100DA00067D6D1BF22859306C402A685EFF06FB344
:100DB0002285EF00902259F5C1470A203CB08145B9
:100DC000EF50DFE8014541B713F7870135CFC18BFD
:100DD000930484004146B1C78905268597F0FA1F20
:100DE000E780005B414681451305840197F0FA1FB7
:100DF000E78080607C201306C403328593E74700B8
:100E00007CA0C14532C6EF50AF818327040832462B
:100E100085C32285EF00B02215F5930720053CB06D
:100E200055B78145268597F0FA1FE780E05C5DBFE6
:100E30009306C402A6852285EFF0AFAA2285EF00B3
:100E4000D019CD4769DDFDBD094785456388E700B9
:100E500093F7D70F11476396E70089450A20EF50B3
:100E6000FFDE7C2093E747007CA08327040881C72E
:100E7000930710056DB7C5475DB73C216380072414
:100E8000797122D406D626D24AD03C3113075005B8
:100E90002A84639DE706034975001306C503C1450F
:100EA00093573900AA973285842732C6EF405FF7FF
:100EB0009737FB1F83A787E7A1C79C47B1C30325CB
:100EC0000408137979003246B3D62441858A930504
:100ED0000504180893E6060813050508829713759C
:100EE000F50F19ED41460C081305C40297F0FA1FDF
:100EF000E780004A2285EF00500E930760053CB062
:100F0000B250225492540259456182801307100254
:100F10006392E7021C5503270508DE2361E713F7F8
:100F2000071069C378555A2B1377071045CF9307DD
:100F300070023CB03C3013077002639BE70C3C58D6
:100F400085E393053005714597F0FA1FE78080141B
:100F500028D819C57146814597F0FA1FE780C04926
:100F60002458B1C4BC2C89E72285EFF0CFA2A8ACED
:100F700028588145414697F0FA1FE780E0472858F6
:100F80003D472C2D9387F5FF93F7F70F6364F70028
:100F9000EF401FE9EF209FFF3C58A1458AAB138526
:100FA0002701EF40FFE72C580A20EF00D0329307CB
:100FB00080020A203CB09720FB1FE780E09E41465C
:100FC00009C57E2513D617003E962254B25092547E
:100FD00002591735FB1F0345151106068545456166
:100FE0006F308F9A13F7072009CB78545A2B137759
:100FF000072001C7930790022DBF93F707409DDBA1
:101000007C54DE2B93F7074095D79307B00215B7B2
:1010100013078002639FE7023C5899C78E2B0A2072
:1010200013862701EF0090301C54DE2313F70720AE
:1010300011C778545A2B1377072035EF93F70740E1
:10104000A5CB7C54DE2B93F70740BDC39307B002BA
:101050008DB713079002639BE700EF508F8BAA8533
:101060000A20EF00B02B9307A002A1B71307A0023C
:101070006396E702EF504F89AA858547014563844F
:10108000F500814505452EC6EF508F852A86B2456D
:101090000A20EF0050251C54DE234DB71307B00281
:1010A0006398E700EF508F87AA850A20EF00702B26
:1010B0009307F002A9B593079002E5BD8280411124
:1010C00022C4405926C206C67C54AA84DE2B13F7DC
:1010D000071011C718545A23137707100DE313F79D
:1010E000072011C718545A231377072009EB93F7E9
:1010F00007408DCB1C54DE2393F7074085C7930729
:1011000010023CB02285EFF05FD738309307F00231
:10111000631EF7002244AA20B24092448145410157
:101120006FE07FC99307F0023CB0EDB7B2402244B4
:10113000924441018280397122DC405926DA4AD832
:101140004ED606DE2A89AE84B289630404382A2189
:101150001E20639FA7103C20638807389387E5FF14
:1011600093F7F70F2D476361F73817D7010013077F
:10117000279BB3C7E7209C43BA9782872285625496
:10118000F250D2544259B259B28521616FF09FACEE
:101190004146CE851305C40497F0FA1FE780401F2F
:1011A0002285AD25383093074005631AF700930771
:1011B00090053335A000931435003CB05DA893062C
:1011C0006005D147E317D7FE9307A005DDB71309E4
:1011D000C4054A854146CE8597F0FA1FE780401B3B
:1011E000032504084DC53C30130790056397E700BD
:1011F000228575259307E00595A81307A00563923E
:10120000E7087C3013D73700229714279D8BB3D67D
:10121000F640858A9737FB1F83A747B193E60608F8
:10122000A1CB9C47B1C79305050818084A8613054A
:10123000050482971375F50F05ED41460C0813055B
:10124000C40497F0FA1FE78020277C304D478507BC
:1012500093F7F70F7CB0E36DF7F885451735FB1F63
:10126000034575E8EF201FDC930750053CB031A81B
:10127000A144F25062544259B2592685D254216198
:1012800082801307C005E385E7F68144DDB7930943
:1012900084004A86CE8522851408EFE09FE441460B
:1012A0009305C404080897F0FA1FE780E02071D185
:1012B0008A861306C403CA854E85EF106069A1446F
:1012C0000DE12285EFE03FED2A870A209737FB1FCB
:1012D00083A707E1814601468A858297B334A0003F
:1012E0008E0493072002D1BD0C22EFE0DFAC71BF6A
:1012F0003830930720026319F71E7C5889EB930559
:101300003005714597F0FA1FE780C0D868D8685853
:10131000630C051C4146CE8597F0FA1FE780400715
:1013200064582285EFE03FE7A8AC930730023DBF49
:101330003830930730026319F71A1E226858214685
:10134000938529001EA9490597F0FA1FE7804004FC
:101350007C54DE2B13F727002DC718545A23098B12
:101360002DC39307400219B7383093074002631D1D
:10137000F7163C5C81EB85455D4597F0FA1FE780E9
:1013800060D128DC285CE30205F083C709004146F0
:10139000CE857CA997F0FA1FE78080FF9307500263
:1013A000F1B53830930750026310F714285C1946E2
:1013B00093851900410597F0FA1FE78060FD7C5482
:1013C000DE2B918B95CF1C54DE23918B95CB93070D
:1013D000600269BD7C5C89EB93053005514597F04F
:1013E000FA1FE78020CB68DC685CE30305E8414630
:1013F000CE8597F0FA1FE780A0F97C5C7D5798CBEB
:101400004A85EFF0DFCB51B503250408130600042D
:10141000CE851305050497F0FA1FE78060F7228553
:10142000EFE07FC83C30130700056395E7009307A2
:1014300040052DBD13071005E381E7E213072005E2
:10144000E395E7E49737FB1F83A7478EE38207E224
:101450009C47E38F07E08325040893048400180861
:1014600093850508814626862E8582970A201008D6
:10147000A685EF509F869307B005CDBB3830930704
:10148000E0056313F7068325040841464E8597F06F
:10149000FA1FE7806002AD44E30D05DC0325040874
:1014A0004146CE8597F0FA1FE78080EE2285EFE077
:1014B0009FCE2A872C580A209737FB1F83A747C245
:1014C000814601468297B334A0008E049307100230
:1014D000EDB1AD47E39BF5DA14222E21130665002A
:1014E0000821EF403FFB55B39D4461B3AA870945EE
:1014F00041C6D9C11CA29C211CB29C313CA2BC217A
:101500003CB2BC31A30206005CA2DE2193D787481F
:101510005CB2DA211377072001C793E727005CB29A
:10152000DE2193F7074089C75C3293E747005CB23E
:10153000DE211317B028F98F89C75C3293E7870043
:101540005CB223030600DE21858B7CA2DA21098BA5
:1015500001C793E727007CA2DE21918B89C77C22FB
:1015600093E747007CA2DE21A18B89C77C2293E709
:1015700087007CA20145828082802E86AA8505454F
:101580006FF0DFF62E86AA8509456FF03FF68DC510
:101590002A87094505C7411106C6AE878D4694A125
:1015A000138517004146BA8597F0FA1FE78040DEA1
:1015B000B2400145410182800945828082808DC50B
:1015C0002A87094505C7411106C6AE87914694A1F1
:1015D000138517004146BA8597F0FA1FE78040DB74
:1015E000B2400145410182800945828082808DC5DB
:1015F0002A87094505C7411106C6AE87994694A1B9
:10160000138517004146BA8597F0FA1FE78040D846
:10161000B2400145410182800945828082809DC996
:101620002A87094515CB411106C69D4694A116236C
:10163000AE871385370094B116232146A182B4A149
:101640009305270097F0FA1FE78080D4B240014548
:10165000410182800945828082808DC52A870945A3
:1016600005C7411106C6AE87A14694A11385170090
:101670004146BA8597F0FA1FE78080D1B240014514
:101680004101828009458280828085C92A87094577
:101690001DC7411106C6A54694A11423AE87138524
:1016A000270094B119469305170097F0FA1FE780B9
:1016B00020CEB2400145410182800945828082806E
:1016C0008DC52A87094505C7411106C6AE87A946BB
:1016D00094A1138517004146BA8597F0FA1FE78059
:1016E00020CBB24001454101828009458280828041
:1016F00095C52A8709450DC7411106C6AE87B14673
:1017000094A11385170013060004BA8597F0FA1FF9
:10171000E78000C8B24001454101828009458280CE
:1017200082808DC52A87094505C7411106C6AE8747
:10173000B54694A1138517004146BA8597F0FA1F64
:10174000E78000C5B24001454101828009458280A1
:101750008280AA87094581C999C7154798A19C230A
:1017600001459CB182808280AA87094581C999C7B9
:101770002D4798A19C2301459CB1828082800DC594
:101780005D718A8586C6A2C42A84EFE0DF8D0A20B7
:101790000A8697060000938686DE9D45EFE01F804F
:1017A000B640264461618280054582800DC55D7129
:1017B0008A8586C6A2C42A84EFE0FF8A0A200A86A8
:1017C00097060000938646DC9D45EFE02FFDB6406E
:1017D000264461618280054582805D71A2C49305C3
:1017E000C5022A8441460A8586C697F0FA1FE7801B
:1017F00020BA0A200A8697060000938686D9C54536
:10180000EFE0CFF9B6402644616182805D71A2C4E9
:101810009305C5032A8441460A8586C697F0FA1FB8
:10182000E78000B70A200A8697060000938666D9EB
:10183000C545EFE0AFF6B640264461618280972748
:10184000FB1F83A7A74EA9CB9C435D71A2C486C68C
:101850002A841305E00F8DCF032504089305050C9A
:1018600013050508829783250408130600040A85DA
:101870009385050897F0FA1FE78080B10A20970644
:101880000000938626E70A8693051004EFE00FF127
:10189000B6402644616182801305E00F8280317179
:1018A00022DD2A840A2126DB06DF4AD94ED752D50B
:1018B00056D35AD15ECF62CD66CB9710FB1FE7801F
:1018C000A00E3C58AA8489EB93053005714597E03A
:1018D000FA1FE780207C28D82858CD4715C97146C3
:1018E000814597F0FA1FE78020B10329040722857C
:1018F000EFE07F8A230DA9003C201729FB1F130965
:10190000E94263820712832709008DE39307E00F02
:10191000FA506A54DA544A59BA592A5A9A5A0A5BFE
:10192000FA4B6A4CDA4C3E852961828003AC070190
:10193000E30E0CFC032B0408EF400FFDAA8B0145BE
:10194000EF400FFADC303458130B0B029309C40339
:10195000130AC405938A64002A8736C0B337F0009F
:10196000930801045688B33670015286CE855A8595
:10197000029C1C54B8232307E1029833A306E1021A
:101980009C232306F10283270900C9D383AB4701B7
:10199000E38E0BF6DC30B337F0003ECEEF40CFF6EF
:1019A0002A8B0145EF40CFF303270408F2472AC0F2
:1019B0003AC2B338600156887810930684004E8688
:1019C000D2858800829B7C54B82B2305E102983392
:1019D000A304E1029C232304F1028327090003AB43
:1019E0004701EF406FF22A890145EF406FEF83C84E
:1019F00054009C082A883EC2B3381001B337200136
:101A00003810930684015286CE8556C08800029B0A
:101A10000A2097060000938606D19008C545EFE09E
:101A2000EFD7AA87F5B5D43083270900032B040824
:101A3000B336D00083AC070136CEEF40EFECAA8B73
:101A40000145EF40EFE93C58F246130B0B02130A35
:101A5000C4059309C403938A64002A889308010487
:101A60004E86D2853EC05687B33770015A85829C18
:101A70001C54930B0103B8232307E1029833A306F8
:101A8000E1029C232306F1028327090083AC47016E
:101A9000DC30B337F0003ECEEF400FE72A8B014534
:101AA000EF400FE4F2472AC0B3386001568878103F
:101AB000930684004E86D2855EC28800829C832570
:101AC000040841465E8597F0FA1FE780E09EAD4727
:101AD000E31B05EE35BD2E8697060000938666B1A2
:101AE000C5456FE0AFCB5D71B287A2C44C802A843C
:101AF000BE8513051100194686C697F0FA1FE780C8
:101B000020890A86228597060000938646B8A1455B
:101B1000EFE0CFC8B6402644616182802E869706EA
:101B200000009386C6B3C5456FE04FC75D71B287AD
:101B3000A2C46C802A84BE8513052100214686C676
:101B400097F0FA1FE780C0840A8622859706000076
:101B5000938626ADAD45EFE06FC4B6402644616183
:101B600082802E86970600009386C6B5C5456FE035
:101B7000EFC2797122D406D626D23C311307300544
:101B80002A84638FE706130750056390E7089307DD
:101B9000A0053CB17C31C14513D737002A971427E3
:101BA0009D8B1305C503B3D6F640858A93E60608D8
:101BB00036C6EF40EFA6B2469727FB1F83A707174D
:101BC0009DCB9C478DCB0325040818081306C4033E
:101BD000930505041305050882971375F50F01EDAC
:101BE0001305C40241460C0897E0FA1FE780407ACB
:101BF0002285EFF09FBEB2502254925445618280FC
